:020000040800F2
:1000000000000120694000082D2800082F28000862
:1000100031280008332800083528000800000000B7
:100020000000000000000000000000003728000869
:1000300039280008000000003B2800083D2800087F
:10004000B9400008B940000841280008B94000083C
:10005000B9400008B9400008B9400008B94000089C
:10006000B940000865280008B9400008B9400008F8
:10007000B9400008B94000084D2800085928000878
:10008000B9400008B9400008B9400008B94000086C
:1000900000000000B9400008B9400008B94000085D
:1000A000B9400008B9400008B9400008B94000084C
:1000B000B9400008B9400008B9400008B94000083C
:1000C000B9400008B9400008B9400008B94000082C
:1000D000B9400008B9400008B9400008B94000081C
:1000E000B9400008B94000086D280008B940000870
:1000F000B94000080000000000000000B9400008FE
:10010000B9400008B940000879280008B940000843
:10011000B9400008B9400008B9400008B9400008DB
:10012000B9400008B9400008B9400008B9400008CB
:08013000B9400008B9400008C5
:1001380010B5054C237833B9044B13B10448AFF319
:1001480000800123237010BDBC08002000000000BF
:10015800E839010808B5034B1BB103490348AFF35D
:10016800008008BD00000000C0080020E839010830
:1001780014214160704714207047406A704700009E
:10018800790100087F01000883010008990100082F
:1001980010B5044604F1100000F05CFCC4F8F80047
:1001A8000148C4F87C0110BD88010008F8B5E6B024
:1001B80004460D4616461F460A4906A800F0CAFE20
:1001C80070996F9A05910492009733466E996D9ACB
:1001D800039102922A466C990191214600F060F839
:1001E80067B0F0BD94010008F8B5E6B004460D46C6
:1001F80016461F46094906A800F0ACFE6F996E9A8C
:100208000491039200976D996C9A0291019233467A
:100218002A46214600F087F867B0F0BD940100082F
:1002280038B500281CBF01680029184A23D1184B8B
:100238001C684FF6F0710C404CF24025AC421FBFD1
:100248001B6819404CF27024A14212D1114D296843
:1002580079B911490B68C3F30B03B3F58A6F1FBF54
:100268000968C1F30B0140F28343994204BF01219D
:10027800117028B905E0094B994204BF012111709A
:100288004068BDE8324001F0D7BE00BFD808002062
:1002980000ED00E0002004E00010005C000037489A
:1002A8002DE9F04104460D46216816464A681F4666
:1002B80090478046B8F5403F2ED122680A99936846
:1002C800204698478046B8F5403F25D12368089ACC
:1002D8000799D3F80CC02046E0478046B8F5403F60
:1002E8001AD12368069A39461F692046B8478046BE
:1002F800B8F5403F10D1236829465D69324620464B
:10030800A8478046B8F5403F06D123680B9A09995B
:100318009D692046A847804621680A68204690477C
:100328004046BDE8F0812DE9F04104460D462168BC
:1003380016464A681F4690478046B8F5403F2ED17A
:1003480022680A999368204698478046B8F5403F46
:1003580025D12368089A0799D3F80CC02046E047AE
:100368008046B8F5403F1AD12368069A39461F6976
:100378002046B8478046B8F5403F10D12368294643
:100388005D6932462046A8478046B8F5403F06D109
:1003980023680999DD6900222046A847804621681C
:1003A8000A68204690474046BDE8F0814FF4403047
:1003B80070470000F0B50C4685B0114600281A4673
:1003C8001CBF0568002D0B4B11D082B104B971B95F
:1003D8000D9860B10F9E0E9F0A9B0290049603979A
:1003E8000B980C9E009001962046A8470346184695
:1003F80005B0F0BD020003002DE9F04F0646D0B06D
:100408000868F56DD6F860E0726EB76EF36E00BAE4
:1004180000906C46486800BA60600DF14008886832
:1004280000BAA060C86800BAE060086900BA206134
:10043800486900BA6061886900BAA061C86900BAF1
:10044800E061086A00BA2062486A00BA6062886A95
:1004580000BAA062C86A00BAE062086B00BA2063FA
:10046800486B00BA6063886B00BAA063C86B00BAB7
:10047800E063402058F80C1C58F820CC58F838ACE9
:100488008CEA010158F840CC8AEA01018CEA01099A
:100498004FEAF979401E48F8049BEBD187EA02003D
:1004A80000EA0E00784010EBF5610098DFF824C4EC
:1004B80041186144C81882EABE032B404FEAF06134
:1004C80053405918636859186144CF194FEAB50366
:1004D80083EABE01014081EABE0111EBF765A1681C
:1004E8004D196544A91883EAB0023A404FEAF1650C
:1004F8005A405519E26855194FEAB70282EAB0071F
:1005080065440F4005EBBE0E97EAB00717EBFE6592
:1005180027697D194FEAB10782EA0701654401EAB4
:100528000E01EB18514011EBF36561694D194FEA63
:10053800BE0187EA010E65440EEA030E15EBB00012
:100548008EEA070E0EEBF065D4F818E075446544A2
:10055800AA1881EAB30505404FEAF26E4D40AE4451
:10056800E569AE44E64477444FEAB00080EAB30E4A
:100578000EEA020E8EEAB30E0EEBF765D4F820E011
:1005880075446544691880EAB2053D404FEAF16E4A
:100598004540AE44656AAE44E6440EEBB3034FEA09
:1005A800B70787EAB20E0EEA010E8EEAB20E0EEB1C
:1005B800F365D4F828E075446544281887EAB1053E
:1005C8001D404FEAF06E7D40AE44E56AAE44E64415
:1005D8000EEBB2024FEAB30383EAB10E0EEA000E45
:1005E8008EEAB10E0EEBF265D4F830E0754465443E
:1005F800EF1983EAB00515404FEAF76E5D40AE4447
:10060800656BAE44E6440EEBB1014FEAB20282EAF2
:10061800B00E0EEA070E8EEAB00E0EEBF165D4F8B6
:1006280038E075446544EB1882EAB7050D404FEA97
:10063800F36E5540AE44E56BAE44E6440EEBB000B5
:100648004FEAB10181EAB70E0EEA030E8EEAB70E41
:100658000EEBF065D4F840E07544654481EAB30ECA
:10066800AA180EEA000E4FEAF2658EEA010E7544EA
:10067800DDF844E04FEAB000754480EAB30E654403
:100688000EEA020E15EBB7078EEAB30E0EEBF7650E
:10069800DDF848E04FEAB202754480EA020E65448C
:1006A8000EEA070E69188EEA000E0EEBF165DDF80A
:1006B8004CE07544654405EBB3034FEAB70E1427C5
:1006C8000DF1500CDFF810528EEA010B82EA0B0B89
:1006D8000BEBF36A5CF804BBDA44AA44504483EA9F
:1006E800B10B4FEAF06A8EEA0B0BDA445CF804BBF4
:1006F800DA44AA44524480EAB30B4FEAF26A8BEA1E
:10070800B10BDA445CF804BBDA444FEAB000AA44FF
:1007180080EA020BD6448BEAB30B0BEBFE6A5CF85B
:1007280004BBDA444FEAB202AA4482EA0E0B0AEB8F
:10073800B10180EA0B0B0BEBF16A5CF804BBDA44FD
:100748007F1DAA44282F0AEBB3034FEABE0EBBD382
:100758003C2F61D3502F4DD204EB870CC7F15407BF
:100768005E4CA7FB04A504465D4FA8088EEA010A63
:1007780082EA0A0A5CF804BB0AEBF3655D447D195A
:100788002C1983EAB10A4FEAF4658EEA0A0A55443D
:100798005CF804AB5CF804BB55447D19AA1884EADC
:1007A800B30A4FEAF2658AEAB10A55445D444FEA52
:1007B800B4047D1984EA020AAE448AEAB30A0AEB51
:1007C800FE655CF804AB55444FEAB2027D1982EA33
:1007D8000E0A15EBB10184EA0A0A5CF804BB0AEBBD
:1007E800F1655D447D1915EBB303401E4FEABE0E5B
:1007F800BCD12046F46D1B19F365336EC9183166F8
:10080800716E71447166B36ED218B266F16E40189B
:10081800F06650B0BDE8F08F4EEA010B0EEA010A0F
:100828000BEA020B4BEA0A0A0AEBF36554F827A015
:10083800DFF8B0C0554443EAB10B654403EAB10A96
:100848000BEA0E0B28184BEA0A0A7F1C0AEBF06524
:1008580054F827A0554440EAB30B654400EAB30AAC
:100868000BEAB10BAA184BEA0A0A7F1C0AEBF265DD
:1008780054F827A055444FEAB00040EA020B6544FB
:1008880000EA020A0BEAB30BAE444BEA0A0A7F1CE1
:100898000AEBFE6554F827A055444FEAB20242EA33
:1008A8000E0B654402EA0E0A0BEA000B15EBB101C8
:1008B8004BEA0A0A7F1C0AEBF16554F827A0554455
:1008C8007F1C65443C2F05EBB3034FEABE0EA3D350
:1008D80040E700BF9979825AA1EBD96ECDCCCCCC38
:1008E800D6C162CADCBC1B8F00B581B00168074A5B
:1008F800914200D110B9064801B000BD7C2112F028
:10090800D9FF4FF4003001B000BD00BFFC0900085A
:10091800030002002DE9F0410B4A92E8F85188B033
:10092800694681E8F8510268084B9A4200D118B923
:10093800074808B0BDE8F0811422083000F04FFBEA
:1009480008B0BDE8F08100BFDC090008FC09000818
:1009580003000200152904D20268044B9A4200D110
:1009680008B903487047083000F048BBFC09000884
:100978000300020010B481B013460268074CA2427B
:1009880000D118B901B010BC0548704701B000F19A
:10099800240210BC083000F035BB00BFFC09000879
:1009A8000300020010B481B013460268074CA2424B
:1009B80000D118B901B010BC054870470A4601B00B
:1009C80000F1240110BC083000F070BBFC090008DD
:1009D800030002000123456789ABCDEFFEDCBA981E
:1009E80076543210F0E1D2C300000000000000008D
:1009F80000000000F10800081D0900085D09000852
:100A08007D090008AD09000801040008790F0008F5
:100A1800C50F0008810F0008F0B5A3B004460B48C5
:100A280002900D4616461F46094B0822402104A88D
:100A380000F0D1FA28980190009733462A462146BB
:100A480002A800F01BF823B0F0BD00BFFC090008A5
:100A5800100A000810B5040008BF002408D0054893
:100A6800054B20600822402104F1080000F0B3FA89
:100A7800204610BDFC090008100A00082DE9F041C5
:100A880004460E46216817464A681D469047804628
:100A9800B8F5003F19D1226806999368204698470F
:100AA8008046B8F5003F10D123683146DE683A46E3
:100AB8002046B0478046B8F5003F06D12368079A1C
:100AC80029461D692046A847804621680A682046AD
:100AD80090474046BDE8F08110B500F033FA4FF476
:100AE800403400280EBF034C4FF4C07112F0E2FEF0
:100AF800204610BD0200030010B5044600F022FA9B
:100B080008B9054810BD0021A160D0F87C21116802
:100B180088474FF4403010BD0200030070B504460A
:100B28000D4600F00FFA064E40B1D0F87C0141683E
:100B38008847A84224BF65604FF44036304670BDF0
:100B4800020003002DE9FF4715000C4600D02CB128
:100B5800064600F0F7F95FEA000801D16448C3E0EF
:100B6800D8F8F80001684A689047B0F5003F17D1F7
:100B7800D8F87C118A68404690478146B9F1810FC0
:100B880080F09E80A94508F1FC0A17D2D8F8F80031
:100B98000368D3F80CC02A462146E047B0F5003F69
:100BA80040F08E80D8F8F8000368D3F810C06A4681
:100BB8005146E047B0F5003F76D10AE0002004E056
:100BC800215C0AF800100098401C00900098A84288
:100BD800F6D34FF0000C4749474A484B01AC009800
:100BE800844558D2D3E9007001ADC5E9007010788A
:100BF80000281ABF042086464FF0000E085854F803
:100C08000E5028443E4D05600127D0F800E087606B
:100C1800019D4F681AF80C007D408EEA050585F0A5
:100C2800040E65680F687D4085F0FC05754485F005
:100C3800A30568400AF80C000CF1010CCFE7D3E9D2
:100C4800004501A8C0E9004510782E4D002814BFC2
:100C58004FF0040E4FF0000E01A8744651F80EE054
:100C68000459A6440127CEF80050DEF80040CEF81B
:100C780008704D68019F40687D406C400D68684071
:100C880084F0040480F0FC00041984F057040AF886
:100C98000C400CF1010CCC45D1D3D8F8F800016810
:100CA8004A689047B0F5003F0AD1D8F8F8000368C1
:100CB800D3F80C804A465146C047B0F5003F01D0F2
:100CC800114811E0002006E05AF8201081F06A313E
:100CD8004AF82010401CB0EB990FF5D3B06840F0EB
:100CE8000100B0604FF4403004B0BDE8F08700BFA9
:100CF80002000300803A0108D8080020240F0008E9
:100D0800ADBE4ED70DBE75A10100030038B50C4627
:100D1800017A1546CA0702D500F014F908B908483F
:100D280032BDD0F8F80003682146DC682A46A0479F
:100D3800B0F5003F01D0034832BD4FF4403032BD1A
:100D480002000300010003002DE9F84191B00546B7
:100D58000E461746402101A812F0ACFD297AC807B3
:100D680004D5284600F0EEF8040002D1DFF8A4808C
:100D78004BE0D4F8F800DFF8A0800368D3F810C07F
:100D88006A4601A9E047B0F5003F3ED1D4F8F80023
:100D980001684A689047B0F5003F36D1D4F87C1115
:100DA8008A6820469047D4F8F830024618461B68EF
:100DB800D3F80CC004F1FC01E047B0F5003F24D1A2
:100DC800D4F87C0141688847D4F8F83002461846C0
:100DD8001B68D3F80CC001A9E047B0F5003F14D157
:100DE800D4F8F8000268696893689847B0F5003F3E
:100DF8000BD1D4F8F80003681C693A463146A0477D
:100E0800B0F5003F08BF4FF44038404612B0BDE887
:100E1800F08100BF02000300010003002DE9F84142
:100E2800A5B0074688461646402115A812F042FD8F
:100E380000220492402105A812F03CFD387AC1072F
:100E48005ED5384600F07EF8050059D0D5F8F80090
:100E58002D4C0368D3F810C06A4605A9E047B0F5E1
:100E6800003F3CD1D5F8F80001684A689047B0F5D2
:100E7800003F34D1D5F87C118A6828469047D5F8C8
:100E8800F830024618461B68D3F80CC005F1FC017F
:100E9800E047B0F5003F22D1D5F87C01416888478A
:100EA800D5F8F830024618461B68D3F80CC005A9D7
:100EB800E047B0F5003F12D1D5F8F800026879682C
:100EC80093689847B0F5003F09D1D5F8F800036852
:100ED8001D6904AA15A9A847B0F5003F01D020460E
:100EE8000FE00A4B0A490B4A0396029101924046C9
:100EF8001C68049B009415AA796800F0E5F900E0E5
:100F0800054826B0BDE8F08101000300883A0108D1
:100F1800936E030026C703000200030004B001011A
:100F280000170145E10A0008010B0008250B00081D
:100F3800B50300084D0B0008150D0008510D0008F9
:100F4800250E00080168024A914218BF0020704728
:100F58002C0F000810B5040008BF002404D0034873
:100F68002060204609688847204610BD2C0F0008DD
:100F780020225C3012F09CBCF0B58468A3080022E3
:100F880004F0030407E000F15C0555F8226035BA67
:100F980041F82250521C9A42F5D300220BE000F18E
:100FA8005C0502EB830755F82360D500C5F11805E9
:100FB800EE40CE55521CA242F1D3F0BD30B5C46804
:100FC80003690022E31AD5188C5C0544521C082AD0
:100FD8002C77F8D330BD0360C1600261704738B523
:100FE800044615460022626023685A68904700202C
:100FF8006061A061A5604FF4003032BD81604FF49C
:10100800003070472DE9F84304462079D4F80C8065
:10101800450748BF244845D466691D46A8F1010024
:1010280000EAD60306EBC506B6EBC50F666102D229
:10103800A669761CA6611746A66906EB5576A661D1
:101048000E46E918884225D2A8EB03094A463146DC
:10105800F81812F02DFC2268136839460FE0424652
:10106800384612F025FC23681A683946204690470E
:1010780007E0311811F00300F1D122681368204607
:101088009847484600EB0809A9F10101A942F0D3A5
:10109800002300E000202A1A3118F81812F008FC82
:1010A8004FF40030BDE8F283040002002DE9FC4F44
:1010B800024685B0D0681369DFF86CC1DFF86C812F
:1010C800A0EB030A506840F004005060002703A812
:1010D80002900DF10C0ED8E9003403A8544DC0E974
:1010E80000342878534D00280CBF00230423994668
:1010F8005CF803305EF80940234401261D601C6833
:101108009E60DCF80430039DDCF80090DEF8046093
:101118005D406540484C654089EA0606474C664094
:101128007519474C6540D8E9006B03AC0028C4E941
:10113800006B0EBF002404200424029E5CF800000B
:10114800345920183F4C04600126046886600398CF
:10115800029E43406340384C7068634089EA00004F
:10116800364C6040034438484340280018BF0120EB
:101178005B1E9B41042F2CBFC0B2D80F02F1140391
:1011880053F8200007F00303C3F10303DB00D84042
:101198000DF807007F1C082F9DD315460C466A6979
:1011A800AB69E868D20842EA4372401E00EA0207C7
:1011B800002302409B420AD8524508D28020E055BD
:1011C8007F1C574516D2AAEB0701E01910E08020D2
:1011D800E05500E0E355E8687F1C8742FAD32A68A7
:1011E800136828469847BAF1000F03D051462046A5
:1011F80012F060FB2A68069E059F93686946284698
:1012080098472A68D2F8009021462846C8472B6894
:10121800DA683946284690470EB1A86830604FF41E
:10122800003007B0BDE8F08F803A0108541200087A
:10123800D80800205FC5109304850012FC68017A65
:10124800C0F524FF24AF33D426AF698B04B0010165
:1012580000170145F8B501240094002300240DE08F
:10126800009D065D0F5D7E40F643761CF60F86F006
:10127800010635400095641C009DEB189442EFD39D
:101288001846F2BDF8B5002301240094002A11E0A5
:10129800009C85188F1815F8016C17F8015C6E40D2
:1012A800F643761CF60F86F0010634400094009C45
:1012B800E318521EECD11846F2BD00005D1200087A
:1012C8008D120008010000002DE9F84F1D46DDF8D9
:1012D80028900B9F0D9C4FF0FF3300930E469246CB
:1012E800D9F800B0804632465146D847834664B3A1
:1012F800D9F8043032465146404698476FEA0B0207
:10130800521C42EA0B0200996FEAD2735B1C194027
:10131800C2430091521C024300996FEAD2735B1CCE
:101328001940009186F05531484087EA000181F064
:101338005531216080F05531C943491C0843009A52
:101348006FEAD070401C82430092D9F80800012847
:1013580009D17540E943491C0D4300986FEAD572DD
:10136800521C90430AE0F11C85EA9102D243521CB8
:10137800154300986FEAD5735B1C984386F0AA362C
:10138800009086EA0B0686F0AA33F243DB430C98FA
:10139800C2F3C0725B1C42EAD3720099D243521C5A
:1013A80091430091774000998843009987F0AA37C4
:1013B8000F403843BDE8F28F034613F8012B002A8B
:1013C800FBD1181A0138704781F0004102E000BFD4
:1013D80083F0004330B54FEA41044FEA430594EAED
:1013E800050F08BF90EA020F1FBF54EA000C55EA28
:1013F800020C7FEA645C7FEA655C00F0E2804FEAF9
:101408005454D4EB5555B8BF6D420CDD2C4480EADA
:10141800020281EA030382EA000083EA010180EA0A
:10142800020281EA0303362D88BF30BD11F0004F58
:101438004FEA01314FF4801C4CEA113102D040428E
:1014480061EB410113F0004F4FEA03334CEA1333C9
:1014580002D0524263EB430394EA050F00F0A780E1
:10146800A4F10104D5F1200E0DDB02FA0EFC22FADC
:1014780005F2801841F1000103FA0EF2801843FAD0
:1014880005F359410EE0A5F120050EF1200E012AC1
:1014980003FA0EFC28BF4CF0020C43FA05F3C018FF
:1014A80051EBE37101F0004507D54FF0000EDCF178
:1014B800000C7EEB00006EEB0101B1F5801F1BD321
:1014C800B1F5001F0CD349085FEA30004FEA3C0C25
:1014D80004F101044FEA445212F5800F80F09A801B
:1014E800BCF1004F08BF5FEA500C50F1000041EB1F
:1014F800045141EA050130BD5FEA4C0C404141EB23
:101508000101013C28BFB1F5801FE9D291F0000F1D
:1015180004BF01460020B1FA81F308BF2033A3F1CC
:101528000B03B3F120020CDA0C3208DD02F1140CC3
:10153800C2F10C0201FA0CF021FA02F10CE002F1FE
:101548001402D8BFC2F1200C01FA02F120FA0CFCF7
:10155800DCBF41EA0C019040E41AA2BF01EB045140
:10156800294330BD6FEA04041F3C1CDA0C340EDC3E
:1015780004F11404C4F1200220FA04F001FA02F381
:1015880040EA030021FA04F345EA030130BDC4F13F
:101598000C04C4F1200220FA02F001FA04F340EA34
:1015A8000300294630BD21FA04F0294630BD94F0E5
:1015B800000F83F4801306BF81F480110134013DCC
:1015C8004EE77FEA645C18BF7FEA655C29D094EA3D
:1015D800050F08BF90EA020F05D054EA000C04BFBB
:1015E8001946104630BD91EA030F1EBF00210020A6
:1015F80030BD5FEA545C05D14000494128BF41F045
:10160800004130BD14F580043CBF01F5801130BDA8
:1016180001F0004545F0FE4141F470014FF0000033
:1016280030BD7FEA645C1ABF194610467FEA655CE4
:101638001CBF0B46024650EA013406BF52EA033586
:1016480091EA030F41F4002130BD00BF90F0000F74
:1016580004BF0021704730B54FF4806404F13204B0
:101668004FF000054FF0000150E700BF90F0000F69
:1016780004BF0021704730B54FF4806404F1320490
:1016880010F0004548BF40424FF000013EE700BF60
:1016980042004FEAE2014FEA31014FEA02701FBFF0
:1016A80012F07F4393F07F4F81F06051704732F022
:1016B8007F4208BF704793F07F4F04BF41F4002179
:1016C800704730B54FF4607401F0004521F00041D7
:1016D8001CE700BF50EA010208BF704730B54FF061
:1016E80000050AE050EA010208BF704730B511F062
:1016F800004502D5404261EB41014FF4806404F19A
:1017080032045FEA915C3FF4D8AE4FF003025FEA1F
:10171800DC0C18BF03325FEADC0C18BF033202EBA3
:10172800DC02C2F1200300FA03FC20FA02F001FAFD
:1017380003FE40EA0E0021FA02F11444BDE600BFA0
:101748004FF0FF3C06E000BF4FF0010C02E000BF85
:101758004FF0010C4DF804CD4FEA410C7FEA6C5C68
:101768004FEA430C18BF7FEA6C5C1BD001B050EA0B
:10177800410C0CBF52EA430C91EA030F02BF90EAF6
:10178800020F0020704710F1000F91EA030F58BFB5
:10179800994208BF90422CBFD8176FEAE37040F017
:1017A800010070474FEA410C7FEA6C5C02D150EAB5
:1017B800013C07D14FEA430C7FEA6C5CD6D152EA70
:1017C800033CD3D05DF8040B704700BF8446104635
:1017D80062468C461946634600E000BF01B5FFF734
:1017E800B7FF002848BF10F1000F01BD4DF808ED04
:1017F800FFF7F4FF0CBF012000205DF808FB00BFD5
:101808004DF808EDFFF7EAFF34BF012000205DF82E
:1018180008FB00BF4DF808EDFFF7E0FF94BF01207B
:1018280000205DF808FB00BF4DF808EDFFF7CEFF7C
:1018380094BF012000205DF808FB00BF4DF808EDBB
:10184800FFF7C4FF34BF012000205DF808FB00BF8C
:101858004FEA410212F5001215D211D56FF47873D0
:10186800B3EB625212D94FEAC12343F0004343EA73
:10187800505311F0004F23FA02F018BF404270474E
:101888004FF00000704750EA013005D111F00040D8
:1018980008BF6FF0004070474FF00000704700BF6E
:1018A80080F0004002E000BF81F0004142001FBF0D
:1018B8005FEA410392EA030F7FEA226C7FEA236C16
:1018C8006AD04FEA1262D2EB1363C1BFD21841400B
:1018D80048404140B8BF5B42192B88BF704710F0A1
:1018E800004F40F4000020F07F4018BF404211F044
:1018F800004F41F4000121F07F4118BF494292EAAC
:10190800030F3FD0A2F1010241FA03FC10EB0C00D7
:10191800C3F1200301FA03F100F0004302D5494264
:1019280060EB4000B0F5000F13D3B0F1807F06D311
:1019380040084FEA310102F10102FE2A51D2B1F109
:10194800004F40EBC25008BF20F0010040EA0300FE
:101958007047490040EB0000013A28BFB0F5000F7E
:10196800EDD2B0FA80FCACF1080CB2EB0C0200FA34
:101978000CF0AABF00EBC25052421843BCBFD04083
:101988001843704792F0000F81F4000106BF80F4FD
:1019980000000132013BB5E74FEA41037FEA226CC0
:1019A80018BF7FEA236C21D092EA030F04D092F08B
:1019B800000F08BF0846704790EA010F1CBF0020BF
:1019C800704712F07F4F04D1400028BF40F000401C
:1019D800704712F100723CBF00F50000704700F03C
:1019E800004343F0FE4040F4000070477FEA226263
:1019F80016BF08467FEA23630146420206BF5FEA34
:101A0800412390EA010F40F4800070474FF0000333
:101A180004E000BF10F0004348BF40425FEA000CFA
:101A280008BF704743F0964301464FF000001CE0A2
:101A380050EA010208BF70474FF000030AE000BFF8
:101A480050EA010208BF704711F0004302D5404236
:101A580061EB41015FEA010C02BF844601460020A8
:101A680043F0B64308BFA3F18053A3F50003BCFAC3
:101A78008CF2083AA3EBC25310DB01FA02FC634470
:101A880000FA02FCC2F12002BCF1004F20FA02F277
:101A980043EB020008BF20F00100704702F120026A
:101AA80001FA02FCC2F1200250EA4C0021FA02F2CB
:101AB80043EB020008BF20EADC7070474FEA40029F
:101AC800B2F1FE4F0FD34FF09E03B3EB12620DD964
:101AD8004FEA002343F0004310F0004F23FA02F0CE
:101AE80018BF404270474FF00000704712F1610F75
:101AF80001D1420205D110F0004008BF6FF000404C
:101B080070474FF00000704753B94AB9002908BF21
:101B180000281CBF4FF0FF314FF0FF3000F06AB9CA
:101B2800ADF1080C6DE904CE00F006F8DDF804E02C
:101B3800DDE9022304B070472DE9F047089D0C4603
:101B4800002B4ED194468C458646B2FA82F262D971
:101B58004AB1C2F12003914020FA03F30CFA02FCC7
:101B6800194300FA02FE4FEA1C471FFA8CF6B1FB34
:101B7800F7F44FEA1E4307FB141143EA014304FB41
:101B880006F199420AD91CEB030304F1FF3080F0F7
:101B98001281994240F20F81023C6344591A1FFA9C
:101BA8008EF3B1FBF7F007FB101143EA014300FB8A
:101BB80006F69E420AD91CEB030300F1FF3180F0C0
:101BC800FC809E4240F2F980634402389B1B40EA45
:101BD800044000211DB1D3400022C5E90032BDE810
:101BE800F0878B4205D90DB1C5E9000100210846EF
:101BF800F5E7B3FA83F1002946D1A34202D3904214
:101C0800C0F0F080861A64EB03030120002DE6D0B3
:101C1800C5E90063E3E7002A40F09080A1EB0C04DB
:101C28004FEA1C481FFA8CF70121B4FBF8F64FEA7B
:101C38001E4308FB164443EA044307FB06F0984298
:101C480008D91CEB030306F1FF3402D2984200F2D4
:101C5800CD8026461C1A1FFA8EF3B4FBF8F008FB59
:101C6800104443EA044300FB07F79F4208D91CEBE2
:101C7800030300F1FF3402D29F4200F2B0802046F5
:101C8800DB1B40EA0640A5E7C1F120068B4022FA9B
:101C980006F71F4320FA06FC04FA01F343EA0C0393
:101CA800F44000FA01F8380C4FEA1349B4FBF0FE8F
:101CB8001FFA87FC00FB1E4449EA04440EFB0CF99A
:101CC800A14502FA01F20AD93C190EF1FF3A80F057
:101CD8008480A14540F28180AEF1020E3C44A4EB21
:101CE80009041FFA83F9B4FBF0F300FB134449EA33
:101CF800044403FB0CFCA44507D93C1903F1FF304D
:101D080067D2A44565D9023B3C4443EA0E40A0FB98
:101D18000293A4EB0C049C42CE469C4651D34ED071
:101D280055B1B8EB0E0364EB0C0404FA06F6CB408D
:101D38001E43CC40C5E90064002150E7C2F12003EE
:101D480020FA03F10CFA02FC24FA03F394400C4342
:101D58004FEA1C4800FA02FE1FFA8CF7B3FBF8F0B2
:101D680008FB1031230C43EA014300FB07F19942B9
:101D780008D91CEB030300F1FF362CD299422AD96B
:101D8800023863445B1AA4B2B3FBF8F108FB1133C1
:101D980044EA034401FB07F3A34208D91CEB0404FB
:101DA80001F1FF3613D2A34211D902396444E41A6F
:101DB80041EA004139E70446F0E6084606E7C84527
:101DC800AED2B9EB020E63EB070C0138A8E7314637
:101DD800EDE7034699E73046D4E7D6467FE7634404
:101DE80002384DE70646234608460FE7023E63449D
:101DF80030E700BF704700BF1348144A08B54FF0DA
:101E08000043C0E900230422426101220023C26189
:101E18004FF480510722C0E90233C0E90933C0E911
:101E28000C1203610383837680F8203080F82C300D
:101E3800826380F83C30C36404F0D0FE18B1BDE87A
:101E4800084000F037BC08BDDC0800200024014031
:101E580010B5044688B01422002103A811F0F4FC40
:101E68002268114B9A421DD14FF0B04303A91A6E54
:101E780042F400721A661A6E02F400720292029A12
:101E8800DA6C42F00102DA64DB6C03F001030193BF
:101E9800019B4FF4004203234FF09040CDE9032308
:101EA80005F0BAFD08B010BD002401400268084BD7
:101EB8009A420BD14FF0B0424FF40041136E23F415
:101EC800007313664FF0904005F052BE704700BF94
:101ED8000024014030B585B000240546CDE9014411
:101EE8000394FFF789FF144805F00CFA08B100F0D5
:101EF800E1FB1148039401A9CDE9015404F0CCFF9A
:101F080008B100F0D7FB0C4805F026F908B100F03D
:101F1800D1FB4FF0FF31084804F060FF064805F098
:101F2800D3F9054804F0B4FF0446034805F076F9F0
:101F3800204605B030BD00BFDC080020014B024A36
:101F48001A607047DC0800200024014008B50948E1
:101F5800FFF7C0FF68B1084BB3F8AA304FF6FF721D
:101F6800934216BF40F6E442044B5343B3FBF0F3ED
:101F780098B208BD002000B40075FF1FD8084C00B7
:101F880013B50023ADF80630FFF7E0FF0446194803
:101F9800FFF7A0FF184BB3F8C820B3F8A8108A427F
:101FA80004FB00F018D040F6E443B0FBF3F36420E0
:101FB8005B1A4343521A93FBF2F31E331BB2ADF87C
:101FC8000630BDF806305BB21B02ADF80630BDF82E
:101FD800060000B202B010BD4FF47A7240F6FF73EB
:101FE800B0FBF3F35343A3F53923A3F50C6340F691
:101FF800C412E0E7001000B00075FF1F08B50C48D8
:10200800FFF768FF88B10B4BB3F8AA304FF6FF72A1
:1020180093421FBF40F6E4425343B3FBF0F398B238
:1020280004BF40F6D803B3FBF0F0400080B208BD0F
:102038000008002C0075FF1F4FF0B04382B09A6A69
:1020480022F480529A629A6C42F480529A649B6C91
:1020580003F480530193019B002002B070474FF0B6
:10206800B04307B59A6C42F004029A649A6C02F085
:1020780004020192019A9A6C42F001029A649B6CE4
:10208800002203F00103114600930E20009B05F087
:10209800D7F90E2005F006FA002211460F2005F0A8
:1020A800CFF90F2005F0FEF900220221112005F0DA
:1020B800C7F9112003B05DF804EB05F0F3B900008F
:1020C80008B505F0C9FB10B16FF0040008BD064B58
:1020D8009A6942F040429A614CF2FA321A6105F06C
:1020E800CDFB0028F2D0EFE700400058F0B585B0EE
:1020F80000230D4600930646A8B3FFF7E1FF044608
:1021080070BB05F0A9FB88BB1A481B4A0223019340
:10211800D0F8E01506F1784302EA8121B3FBF1F724
:1021280001FB1733DB0A0293D0F8E00505F178418B
:102138000139314402EA8022B1FBF2F002FB1011AE
:10214800C3EBD1230133694601A8039305F016FCBC
:1021580020B1022814BF6FF00104012405F08EFBA2
:10216800204605B0F0BD6FF00504F9E76FF00404F0
:10217800F6E700BF0070FF1F00FCFF03014B18606B
:1021880000207047400900202DE9F04FB0F1006FA2
:1021980089B006460F469046C0F0C080DFF890919F
:1021A800644DD9F8E03505EA832303F10063013B68
:1021B800984200F2B380002900F0B38040EA02039D
:1021C8005B0740F0AE80FFF77BFF044690BB05F04D
:1021D80043FB002840F0A880D9F8E015009705EAED
:1021E800812106F17842B2FBF1F301FB132208F1D9
:1021F8007843013B3344B3FBF1F001FB1033DB0AB6
:1022080001334FEAD22AA3EBD222012A039388BFD3
:10221800C6F30A050AF58037C6F108038CBFC5F571
:1022280000654546FF02B3460693039B9A4505D3CE
:1022380005F024FB204609B0BDE8F08FA6F108039D
:10224800069A1A4495421CD8009B04950193CDF830
:1022580014B04FF00009059B09EB0301049B994555
:102268003DD3009BAB442B44A8EB0505B5F5006FA7
:10227800009328BF4FF400650AF1010A07F50067CB
:10228800D3E753F8081F5A68B2F1FF3F08BFB1F10E
:10229800FF3FD5D0284B186810B96FF00504C7E781
:1022A80027B14FF40062394610F092FEDFF88890AB
:1022B8000099D9F80030CBF30A001844AAB210F0FC
:1022C80087FE4FF400613846FFF710FF00BBD9F8CE
:1022D800003001934FF4006305970493B9E7019B1D
:1022E80007914B4402930120D3E9002305F000FB3A
:1022F80088B90799019BD1E9000259F80310029B9C
:102308005B689A4208BF884205D109F10809A2E72B
:102318006FF001048CE76FF0030489E74FF0FF3496
:1023280088E76FF0050485E76FF0040482E700BFD3
:102338000070FF1F00FCFF0340090020B1F1006F8F
:1023480070B510D30B4BD3F8E0650B4B03EA86232B
:1023580003F10063013B994205D838B192B210F0FD
:1023680037FE002070BD4FF0FF30FBE76FF005002F
:10237800F8E700BF0070FF1F00FCFF03B0F1006F1B
:1023880010B40DD3084BD3F8E045084B03EA842377
:1023980003F10063013B984202D810BCFFF7A6BEC8
:1023A8004FF0FF3010BC70470070FF1F00FCFF03A8
:1023B8004FF0B04382B0DA6C0243DA64DB6C03405E
:1023C8000193019B02B070472DE9F04387B00024C8
:1023D8000120294E0594FFF7EBFF0220FFF7E8FFE5
:1023E800FFF7E6FF0120FFF7E3FF022708224FF47B
:1023F800041301A93046CDE9012301254FF0200936
:102408000394049705F008FB01A930464FF40078BF
:10241800CDE90195CDE9037405F0FEFA01A94FF065
:102428009040CDE90185CDE9037405F0F5FA142350
:1024380001A93046CDE90135CDE9037405F0ECFA80
:102448002A464946304605F00DFC2A4641464FF0DB
:10245800904005F007FC2A463046102105F002FCA2
:1024680022462146092004F0EBFF092005F01AF85E
:1024780007B0BDE8F08300BF000400481248134AC3
:1024880008B540F61463C0E9002300230122C0E91F
:102498000232C0E90433C0E90633036205F05EFD89
:1024A80008B100F007F90848002105F0D7FE08B187
:1024B80000F000F90448002105F0F6FE18B1BDE867
:1024C800084000F0F7B808BD040A00200058004092
:1024D80070B596B005461422002103A811F0B4F98E
:1024E8003822002108A811F0AFF92A68304B9A4227
:1024F8005BD18023089308A84FF440230E9306F07D
:102508002FFC08B100F0D6F84FF0B0444FF4C0509B
:10251800E36C43F00103E364E36C03F0010302930B
:10252800029B12230026CDE903030323CDE90563AB
:102538004FF09040042303A9079305F06DFAA36DAB
:10254800DFF870C043F48003A365A36D1A4C03F44D
:1025580080030193019B26620D23C4E900C3204632
:102568008023C4E90266C4E90436C4E9066604F0B7
:10257800F9FF08B100F09EF8104AEC63A562104C10
:102588000E23C4E900231021002380222046C4E939
:102598000213C4E90423C4E90633236204F0E2FF0A
:1025A80008B100F087F8AC63A56216B070BD00BF33
:1025B8000058004044000240A4090020580002408E
:1025C8004409002000B59BB04822002108A811F05A
:1025D8003BF91822002102A811F036F905F08AFE0D
:1025E8004FF0B0420120D2F8903023F01803C2F81F
:1025F8009030D2F8003423F4C06343F40073C2F877
:102608000034D2F8003403F4C0630193019B2423FF
:10261800089381230B930023CDE91003B02208A867
:10262800CDE9122305F0DEFF08B172B6FEE74F23AD
:10263800CDE90230CDE90400CDE90600022102A867
:1026480006F06AFA08B172B6FEE71BB05DF804FB43
:1026580008B5154C04F088FAFFF7B4FFFFF7B4FE8D
:10266800124807F077F9FFF7FAFCFFF707FFD4F8ED
:102678008830DB0504D400F016FD00F01BFDFCE7F4
:10268800012204210A4805F0EDFA0123C4F8883034
:102698000723A3614FF4FA6000F042FA04480022CD
:1026A800042105F0DFFAE8E700040058340B0020A5
:1026B8000004004872B6FEE700B58DB02C22002158
:1026C80001A811F0C1F81748174B03601F23836056
:1026D8004FF080420023C0E90433C0E90723836137
:1026E8004FF48073436206F0BDFC08B1FFF7E2FFC8
:1026F8000C4806F0E3FD08B1FFF7DCFF4FF000538C
:1027080000220793074808924FF4807301A90292A8
:1027180006920B9306F006FD08B1FFF7CBFF0DB04C
:102728005DF804FB580A00200028004010B5044654
:1027380090B03822002102A811F086F82268194BBF
:102748009A422CD14FF48033029302A84FF480733D
:102758000F9306F005FB08B1FFF7ACFF4FF0B0434D
:102768000220D3F8902042F40042C3F890209A6DDA
:1027780042F480629A659B6D002203F480631146DF
:102788000193019B04F05CFE022004F08BFE002202
:102798002A20114604F054FE2A2004F083FE10B0CB
:1027A80010BD00BF002800407047000008B50F4862
:1027B80007F0D0F800F0D2FB4FF6FF714FF09040D1
:1027C80005F0D6F90A484FF6FF7105F0D1F9094826
:1027D8004FF6FF7105F0CCF904F0DCF9064B012047
:1027E800C3F88800BDE8084005F0DCBD340B0020C4
:1027F80000040048000800480004005804F0D1B95B
:1028080008B504F0CEF9BDE80840FFF7DDBD08B50E
:1028180004F0C0F9BDE808400121002005F072BDB0
:1028280070477047FEE7FEE7FEE7FEE7FEE7704702
:102838007047704770470000014806F065BD00BF4B
:10284800580A0020014804F099BF00BFA4090020DD
:10285800014804F093BF00BF44090020082005F098
:102868000FBA0000014806F083BB00BF580A0020D9
:10287800014806F072BF00BFBC0A00202DE9F043F2
:1028880089B080460020109E0790894615461F464D
:10289800FDF7C6FCF0B9104CCDE90090CDE9020473
:1028A80007AB0E480593142304933A46434629463A
:1028B8000068FDF77FFD2346324604F1140153F802
:1028C800044B42F8044B8B42F9D1079B337509B08E
:1028D800BDE8F0830120FAE7A60A00207C3A010847
:1028E8001FB50E4C00233C2202A8CDE902336275C5
:1028F800237500F0B7F8042303AA009412210848AE
:10290800FFF7BCFF07491422204610F08DFFB0FAEC
:1029180080F35B09637504B010BD00BF900A002006
:10292800A43A0108E50D0020054808B5082303600E
:1029380006F030FD18B1BDE80840FFF7BBBE08BD82
:10294800BC0A00204FF0B04307B55A6E42F00102AE
:102958005A665B6E002203F0010301931146322090
:10296800019B04F06DFD322003B05DF804EB04F028
:1029780099BD00000CB407B5054A05AB10210193B9
:1029880010F030FE03B05DF804EB02B0704700BFF2
:10299800B63A010830B585B0044602A80D4610F0D5
:1029A8004DFCBDF90C30064A00931021029B2046CD
:1029B800FFF7E0FF2046FEF7FFFC288005B030BD9A
:1029C800B63A01084FF0B04210B5936823F40043BB
:1029D800936010F0BBFC0D4B01241C7010F088F9BB
:1029E8000B4810F09FF90B4B4FF400421A6100207E
:1029F80010F09EF9FFF7A2FA00F0B4F810F092FA7E
:102A080021462046BDE8104010F0ACBAC80A0020A4
:102A18009D2900080040005810F0BABA08B5FFF721
:102A280095FA40F6B83398420CD8B0F5E16F0BD35D
:102A3800FE23A0F5E16058434FF49663B0FBF3F032
:102A4800C0B208BDFE20FCE70020FAE77FB5684663
:102A580000F06CF80198FFF731F800B207B05DF8A4
:102A680004FB0000194A38B5D2F88035591C0446D1
:102A780019D104F09DF8054604F0A6F8054404F0C1
:102A88009DF82B0EE3712B0CA3712B0A6371030EB7
:102A9800E370C0F30742C0F307232571C0B2A270E8
:102AA8006370207038BD190AC3718171190C1B0E2F
:102AB80041710371D2F88435C370D2F88405C0F32C
:102AC8000722C0F30743000EE9E700BF0070FF1FAD
:102AD80038B5094BD3F8803503600133054609D171
:102AE80004F066F8044604F069F8444004F06CF811
:102AF80044402C6038BD00BF0070FF1F0121022038
:102B080010F01ABA0021022010F016BA00207047FF
:102B1800024B187808B100F05DB87047C80A002069
:102B280082B00190019802B000F0F0B810B50446E8
:102B3800FFF726FA074BA36040F30F20FEF76AFF62
:102B4800054B064A2360064B6060C4E90323002056
:102B580010BD00BF0000484200007A440D093E0045
:102B6800AB03050000207047014B1868704700BF91
:102B7800CC0A00200320704708B501464FF47A724A
:102B880000238002890DFEF7BFFF08BD4FF47A735A
:102B9800A0FB0303800A40EA83507047034B986800
:102BA8009A689042FBD1C043704700BF002800409C
:102BB80008B5FFF7F3FF014B186008BDCC0A0020E9
:102BC80008B5FFF7EBFF024B1B68C01A08BD00BF32
:102BD800CC0A0020024B187808B1FFF7DFBF704716
:102BE800D00A002010B5074B074C0122DA654FF4D4
:102BF8008071204606F082F94FF0FF3323630020EE
:102C080010BD00BF00280040580A002002460021DD
:102C1800014806F08ABB00BF580A0020024601217D
:102C2800014806F082BB00BF580A002010B58CB0DE
:102C38002C220021044601A810F006FEFFF7D2FF5F
:102C48000C4B0D481B681C440023089306934FF057
:102C58000053E443079301224FF4807301A90294BF
:102C68000B9306F05FFA08B1FFF724FD00200CB0C3
:102C780010BD00BFCC0A0020580A002038B5054610
:102C8800FFF78CFF02210446074806F055FBC4F302
:102C980009024FF47A71A2FB0121920AA30A2A8041
:102CA80043EA805038BD00BF580A0020014800217F
:102CB80006F042BB580A00200148012106F03CBB3F
:102CC800580A0020F8B50F4D2E78CEB90E4C4FF0AB
:102CD800FF372763FFF7F0FCFFF784FF4FF480719D
:102CE800204606F00BF92046276306F0C9FA32465B
:102CF8002046022106F019FBFFF75AFF01232B702B
:102D08000020F8BDD00A0020580A0020014610B55E
:102D18004FF47A7200238002890DFEF7F5FE014612
:102D2800FFF73CFF0446FFF739FF031B8B4200D334
:102D380010BD00BFF7E710F011BC000010B5064C3D
:102D48000221204606F0F8FA0221421C2046BDE87E
:102D5800104006F0EABA00BF580A00201348144A87
:102D680008B54FF4E133C0E9002300230C22C0E981
:102D78000233C0E90523C0E90733C0E90933036119
:102D880007F003FB08B1FFF795FC0848002107F09E
:102D980071FC08B1FFF78EFC044807F04BFC18B132
:102DA800BDE80840FFF786BC08BD00BF340B002013
:102DB8000044004070B596B006461422002103A8CE
:102DC80010F042FD3822002108A810F03DFD3268BD
:102DD8002C4B9A4254D10223089308A82A4B0A93F1
:102DE80005F0BEFF08B1FFF765FC4FF0B0430025C2
:102DF8009A6D42F400329A659A6D02F4003202929A
:102E0800029ADA6C42F00102DA64DB6C03F0010327
:102E180001930422019B0223CDE903230324072302
:102E280003A94FF09040CDE90554079304F0F4FD51
:102E3800082303A94FF09040CDE90334CDE90555A7
:102E4800124C04F0E9FD124925621423C4E9001369
:102E58001023C4E9023520468023C4E90435C4E9B7
:102E6800065504F07FFB08B1FFF724FC2520F46722
:102E780000220221A66204F0E3FA252004F012FBE6
:102E880016B070BD0044004004000C00D40A0020B5
:102E98008000024002680C4B9A4210B5044612D1D9
:102EA8004FF0B0420C21936D23F4003393654FF03B
:102EB800904004F05DFEE06F04F0C6FBBDE81040F2
:102EC800252004F0FDBA10BD0044004008B50A46AC
:102ED8000146024806F05EFD002008BD340B0020C4
:102EE80013B5114B114C18604FF40013009302AB4B
:102EF80013E90600204607F041FB2368DA69D1038D
:102F0800FCD4DA695202FCD59A68084842F4800277
:102F18009A6007F079FB06490448012207F0EAFAAB
:102F2800002002B010BD00BFC80B0020340B0020E9
:102F3800D00B002008B5074B1860FFF790F8FFF793
:102F48000DFF054AD2F8803043F00063C2F88030A4
:102F5800002008BDCC0B00200008005808B54FF031
:102F6800B04308489A6B42F400329A639A6B22F491
:102F780000329A63FFF78EFF112004F0A1FA0020B7
:102F880008BD00BF340B00200268044B9A4203D1ED
:102F9800034B00201B681847704700BF00440040DF
:102FA800CC0B002002680B4B9A4210B504460FD197
:102FB800094B1B682BB1D0F8902012B907480121A2
:102FC800984720460549BDE81040012207F092BA0B
:102FD80010BD00BF00440040C80B0020D00B0020EB
:102FE80010B50A4C23780BB9E37C6BB1FFF778FC7A
:102FF8000038074B18BF0120400018701B78022BBF
:1030080002BF00232370E37410BD00BFE50D00204C
:10301800D80B002038B5114C2378F3B9E37CE3B919
:103028000F4D2B68012B07D92B68042B04D80D4AA8
:103038000421012000F00EFA2B68042B0DD9FFF7AC
:103048004FFC0038084B18BF0120400018701B784F
:10305800022B02BF00232370E37438BDE50D002066
:10306800D40B0020103B0108D80B002001F0F8B861
:1030780002480122102104F0F5BD00BF00040048F9
:1030880002480022102104F0EDBD00BF00040048F2
:10309800022803D80248102104F0E9BD704700BF98
:1030A80000040048704708B5FFF78CFCBDE80840ED
:1030B80000F070BB4FF0FF300FF0CEBF7047704785
:1030C80070470000014BD870704700BF0C0000200B
:1030D800014B1874704700BF0C00002008B502208F
:1030E80000210FF081FFBDE80840014810F0E4B965
:1030F800480D0020002101200FF076BF10B544F6DE
:103108002063084C002818BF03460748236010F0C6
:1031180085F92168044810F009FABDE81040024812
:1031280010F0CAB908000020480D002010B5094C5D
:10313800206023680BB9084B2360084810F06EF92B
:103148002168064810F0F2F9BDE81040034810F075
:10315800B3B900BFB4000020400D0300DC0B002011
:103168000A460149FFF7EAB800F0030838B50C48E9
:1031780010F054F907F0DEFE60B90A4C0A48012540
:10318800257007F06BFD2078294607F0BFFA044840
:1031980010F092F9BDE83840044810F08DB900BF2E
:1031A800480D0020700000200C000020300D002089
:1031B80007F05EBF7FB5FFF731FC0446FEF71EFF40
:1031C800054607F09DFB0646B0B10024484810F0BC
:1031D80025F9484B46481B689C42214638BF19468A
:1031E80010F0A4F9424810F067F94348002204217E
:1031F80004F038FD04B070BD3F480122102104F0EE
:1032080031FD012204213C4804F02CFD01F026F890
:1032180001F026F8684601F025F8374832461021B3
:1032280004F020FD23B203EB4303FE2203EB431318
:10323800B3FBF2F38DF80C30304B39221A70304A58
:10324800596812780A7059684E7059682720887032
:1032580059680120C87058686421B5FBF1F1C9B2FA
:103268000171284804781CB35968067062F07F021F
:103278000A703A221A7005222349244C0978012938
:1032880088BF00225A70637A33B107F025FB012802
:1032980002D1204610F0C2F81D4B1848D9780022F8
:1032A80007F044FB063090D107F010FB04468DE789
:1032B800184A194C107810B920780028DBD0002063
:1032C800207010705A6804205071BDF800205868AA
:1032D800140A84715868C271BDF808005A68000A57
:1032E8001072BDF80800507291720B22C4E700BF3B
:1032F800480D0020080000200004004800000020BD
:103308003C0C0020E10D0020D80B0020F40B00201D
:103318000C000020600D0020E30D002010B50446CD
:1033280080B190F906306BB9084810F077F8084B6F
:10333800E2791A70074B1868FFF7F8FE064B186811
:10334800FFF7DCFEBDE81040FFF734BFF40B0020A8
:10335800E20D0020B40000200800002020B103780E
:1033680013B1024810F0A8B8704700BF240C002021
:1033780008B5104B0122002102201A700FF034FE0C
:103388000D4810F099F80D4B1B788BB10C4B1A783F
:1033980072B9DB7C63B90B4B1A68042A9EBF1A68A2
:1033A80001321A600021BDE8084010200FF01CBE51
:1033B80008BD00BFE10D0020DC0B0020E20D00205D
:1033C800E50D0020D40B0020044B1B78022B03D101
:1033D800002108200FF008BE704700BF70000020D1
:1033E80008B507F0B0FD80B907F076FA01280CD1CE
:1033F800BFF34F8F0549064BCA6802F4E0621343D6
:10340800CB60BFF34F8F00BFFDE708BD00ED00E0C4
:103418000400FA0538B504460D4607484FF4006124
:10342800FEF7ACFF30B92A4621460348BDE83840CC
:10343800FEF7AABE38BD00BF00F00308704770470A
:1034480070477047082802BF014B01221A70704765
:10345800600E002070B505460C46164607F050FA77
:103468000346002835D000241B480FF0D7FF1B4B1C
:1034780019481B689C42214638BF194610F056F877
:10348800BDE87040144810F017B84A68F05CD05492
:103498000133DAB29442F8D8114B0D701B78012B26
:1034A80088BF00244C700F4C637A33B107F014FACC
:1034B800012802D120460FF0B1FF0B4B0B48D978F9
:1034C800002207F033FA0630CDD107F0FFF90446A1
:1034D800CAE70649DDE700BF480D002008000020C4
:1034E800D80B0020F40B00200C0000200000002066
:1034F800044B1B7823B9044A05210120FFF7AABF12
:10350800704700BFD80B0020153B010810B50024F8
:1035180090B03C22214601A8009410F095F92F4B59
:103528002022DA7219788DF8001059788DF8011078
:1035380099788DF80210D9788DF8031019798DF8DB
:10354800041059798DF8051099798DF80610D979F4
:103558008DF80710197A8DF80810597A8DF8091026
:10356800997A8DF80A108DF80B2021460DF10B027F
:1035780058180131007B02F8010F1C29F8D193F883
:1035880028208DF8282093F829208DF8292093F8F1
:103598002A208DF82A2093F82B208DF82B2093F8D9
:1035A8002C206AB193F83F2052B10DF12B01002273
:1035B8009818013290F82C0001F8010F142AF7D15D
:1035C80007484FF40061FEF7D9FE20B904484022AD
:1035D8006946FEF7D9FD10B010BD00BF710000208C
:1035E80000F80308014940220FF0F2BC00F8030874
:1035F80070B52A4D28796B794D2BC0B233D1C0EB09
:10360800001080000A2838BF0A204FF47A73584304
:10361800234BAC791860EB794D2BE4B22BD1C4EB7A
:103628000414A40095F82C301E4E63BB95F83F3067
:103638004BBB44F62060FFF761FD3068FFF776FD6D
:103648002B7A194A1949DBB213706B7A184ADBB224
:1036580013700023EA1892F82C20D2B2CA5401330E
:10366800142BF7D170BD6B79482B0ABF4FF46163F7
:103678006B795843C6E7EB79482B0ABF4FF461636F
:10368800EB795C43CEE7FFF739FD012C38BF012405
:103698004FF47A735C433460CFE700BF71000020B9
:1036A80008000020B4000020E40D0020E50D0020F3
:1036B800D80B002010B590B000213C2201A8009141
:1036C80010F0C2F84022314968460FF081FC9DF89D
:1036D80000203AB99DF80100272803D19DF802106F
:1036E800012909D0FFF712FF4FF47A70FFF718FA93
:1036F800FFF77EFF10B010BD254B1A7058709970F7
:103708009DF80310D9709DF8041019719DF80510E3
:1037180059719DF8061099719DF80710D9719DF897
:10372800081019729DF8091059729DF80A109972BB
:103738009DF80B1001F03F01D972D87AD1B28842B6
:103748001BD89DF8282083F828209DF8292083F885
:1037580029209DF82A2083F82A209DF82B2083F819
:103768002B200DF12B0100229818013211F8014F7E
:1037780080F82C40142AF7D1BAE701F140006844D8
:10378800194410F8340C08730132D6E700F803081E
:10379800710000201FB5002403A92046039407F0F8
:1037A800B7FB03A9012007F0B3FB384B3848009456
:1037B80022464FF4FA710FF0D3FD364B3648009489
:1037C80022464FF4FA710FF0CBFD344B3448009485
:1037D80001224FF4FA710FF0C3FD2046FEF7CEFC2C
:1037E80008B1FEF767FF2F4B009400224FF4FA61EF
:1037F8002D480FF0B5FD2D4A002101200FF0B0FC37
:103808002B4A002102200FF0ABFC2A4A0021042099
:103818000FF0A6FC284A002108200FF0A1FC00F0B8
:10382800A3FB2649264807F029FB264807F016FA85
:103838001B480FF041FE244B0021187806F066FF64
:1038480022490094224B0968224800220FF088FD83
:1038580020480FF031FEFFF72DFF1F4A00211020EE
:103868000FF07EFC1D4A00214FF480700FF078FCA9
:103878001B4B1C4819681C4B009400220FF070FD6C
:1038880018480FF019FE04B010BD00BF49340008F5
:10389800240C00204B3400080C0C00204534000890
:1038A800F40B0020D1330008300D002069AA00086D
:1038B800BD310008B9310008753100080000030166
:1038C800240000200C0000207000002008000020C8
:1038D800E5300008480D00201D300008753000084C
:1038E800B4000020DC0B00207933000810B5002458
:1038F800A2B07C22214603A802940FF0A5FF53230F
:103908008DF8083040F22713ADF80A3001238DF8FE
:103918000C30ADF80440FFF781F800B200EB40002E
:1039280000EB4010FE23B0FBF3F08DF80D0001A86A
:1039380000F0A8FCA0B958238DF80E300724802287
:10394800002112480FF080FF224602A90F480FF00D
:10395800B4FF0E4A21460120FFF77CFD22B010BDBE
:103968008DF80E0000F094FD094B1A6812128DF8BC
:103978000F201A688DF810205A685B688DF812308D
:1039880012128DF811200B24D9E700BF610D002019
:10399800640E002030B50378592B91B0044640F0EE
:1039A800FC81052959D84378443B162B55D8DFE8C4
:1039B80013F03D0154002D0154003501540054000A
:1039C800540054009200540018015400540054004C
:1039D800A30154005400AE005400540054001700D2
:1039E8008578482D11D1BB4A14210120FFF732FDFB
:1039F80041F28830FFF794F840F6B830FFF790F8B6
:103A080011B0BDE83040FFF7EBBC532D0ED180223A
:103A18000021B1480FF018FFFFF768FF41F2883026
:103A2800FFF77EF8AC4A1521012085E0432D16D119
:103A3800002468468DF8004007F088F8A64A4C2311
:103A48001370272393709DF8003054700120413380
:103A5800D07013710521FFF7FDFC11B030BD442D66
:103A6800FBD19D4C592323705A236370A57000F035
:103A7800F7FB7F220021601C0FF0E6FE272325704C
:103A88000125A370E5702571FEF7C8FF9349FE2351
:103A9800B0FBF3F00B6864229BB2B3FBF2F3A371A3
:103AA8000B6800EB400000EB40109BB26071B3FB69
:103AB800F2F002FB1033E3714B689BB2B3FBF2F3F5
:103AC80023724B689BB2B3FBF2F102FB11336372B2
:103AD80022460A21A8E78378303BDBB2092BBCD801
:103AE8007F49804A0B700B78DBB253727A4A5923AC
:103AF80013704D2353700B780120303303219370DA
:103B0800FFF7A8FC11B0BDE83040FFF7FFBC85788F
:103B1800482D16D1704A562313700023537027235B
:103B28009370032313711823537105230120937194
:103B38001D23D070D371082111B0BDE83040FFF7C4
:103B480089BC432D89D1002421463C2201A8009438
:103B58000FF07AFE6846FFF745FD634B2146732256
:103B680018460FF071FE9DF8002000F80C2C9DF807
:103B7800012000F80B2C9DF8022000F80A2C9DF873
:103B8800032000F8092C9DF8042000F8082C9DF863
:103B9800052000F8072C9DF8062000F8062C9DF853
:103BA800072000F8052C9DF8082000F80D5C00F8A7
:103BB800042C9DF80B509DF8092000F8032C9DF863
:103BC8000A2000F8022C03A92A46A0F10D0400F8E7
:103BD800015C0FF072FE05F10D012246C9B2012009
:103BE80039E7807839280CD83038C0B2FFF740FA66
:103BF800394A2378137063785370A378937003213C
:103C080012E711B0BDE83040FFF772BC8078392860
:103C1800F7D83038C0B2FFF733FAE9E780783928A7
:103C2800EFD83038C0B2FFF733FAE1E78378303B9A
:103C3800DAB2092AE5D8C0783038C2B2092AE0D801
:103C48002179A1F14802D2B20B2ADAD8274D45FAD8
:103C580002F2D507D5D40A224D2902FB030034D13C
:103C68003C2358434FF47A735843214B1860FFF7AD
:103C780045FA194A2378137063785370A3789370C0
:103C8800E378D3700521237913710120FFF7E2FB54
:103C9800144B00221A7027225A7001229A70DA7087
:103CA800A278303A02EB8201E278303A02EB410224
:103CB800D2B21A7122795A710E4A1278D2B21A7295
:103CC800074A1278D2B25A721CE74829CAD14FF46F
:103CD8006163C6E71B3B0108610D0020640E0020EC
:103CE800D80B0020710000206E0D0020DEF7FFFFCA
:103CF80008000020E40D00208278303AD3B2092B66
:103D08003FF67FAFC378303BD9B209293FF679AF88
:103D18000079A0F14801C9B20B293FF672AF624D94
:103D280045FA01F1C9073FF56CAF0A214D2801FB9F
:103D380002332DD13C2253434FF47A7253435B4AEA
:103D480013601068FFF7F2F9594A23781370637803
:103D58005370A3789370E378D37005212379137196
:103D68000120FFF777FB534B00221A7027225A7065
:103D780001229A70DA70A278303A02EB8201E27876
:103D8800303A02EB4102D2B29A712279DA7193E7A2
:103D98004828D1D14FF46162CDE7502B48D1022990
:103DA8007FF65BAE4378303B012B3FF656AE837807
:103DB800312B7FF452AE0B2904D8FFF799FB002171
:103DC8003B4A31E63B4D0234002214F8013FA91862
:103DD800303B0132DBB20C2A0B73F6D1FFF762F9E4
:103DE800334B502227211A709970002201215A70F2
:103DF800D97003F8041FA9180132097B0C2A01F1B4
:103E0800300103F8011FF6D100232B7027236B70B4
:103E18000123AB70EB70284B1B78DBB22B72274B5E
:103E28001B78DBB26B72EA72FFF770FB1121C7E7F0
:103E3800412B7FF412AE4378432B7FF40EAE162944
:103E48007FF40BAE1E4D421C002312F8011FE954EB
:103E58000133142BF9D1FFF7C3F81A4B5B7D012B03
:103E68001DD114490023EA5CC8180133D2B2142BBF
:103E780080F82C20F7D1114B00221A701B78DBB286
:103E88004B72FFF743FB0A4A631E153413F8011FF0
:103E980002F8011BA342F9D1054A1621C4E5074BD4
:103EA80002221A70EFE700BFDEF7FFFFB400002020
:103EB800610D002071000020E40D0020D80B0020C7
:103EC800E50D0020900A002037B504460D4600296C
:103ED80039D022480FF0F0FA2B78A3B39CB360686E
:103EE800237880B3032B0DD0392B2ED0022B2AD167
:103EF8006178012927D00B0625D403B0BDE83040EE
:103F0800FFF748BD6378012B07D10078012802D05C
:103F1800022800D008B906F0D3FD00240DF10700EF
:103F28008DF8074006F012FE0D4A4C231370272324
:103F380093709DF807305470012041330521D070EB
:103F48001371FFF787FA03B030BD6378012BFAD1FC
:103F58000378044A03F001031370F4E70C0C002003
:103F6800610D00203C0C0020034B0022C3E9022213
:103F78000122C3E900227047FC0D00200048704769
:103F8800FC0D00204FF0B04382B0DA6C0243DA64D3
:103F9800DB6C03400193019B02B070472DE9F041AF
:103FA80086B000240220154D0594FFF7EBFF04208E
:103FB800FFF7E8FF124F03944FF4807601230DEBCF
:103FC8000001CDE901632846032304934FF4005808
:103FD80003F022FD01A93846CDF8048003F01CFD4A
:103FE80022464146384603F03DFE284622463146E1
:103FF80003F038FE204606B0BDE8F0810004004812
:1040080000080048032810B50ED8012810D868B950
:1040180002460B484FF4807103F024FE0022094841
:104028004FF4005103F01EFE002010BD0122F0E7FE
:10403800002203484FF4807103F014FE0122EEE7DA
:10404800000400480008004802207047002070471C
:1040580001207047002814BF16200F207047000069
:104068000D48854602F07EFD0C480D490D4A002397
:1040780002E0D458C4500433C4188C42F9D30A4A15
:104088000A4C002301E013600432A242FBD30FF074
:10409800E3FBFEF7DDFAFEE7000001200000002048
:1040A800BC08002024460108BC080020602C002021
:1040B800FEE74FF0B04382B0DA6C42F00102DA64F6
:1040C800DB6C03F001030193019B02B07047000011
:1040D80070B5012286B05248102103F0C3FDFFF7E6
:1040E800E8FF4FF4805101224FF0904003F0BAFDF1
:1040F80001224FF400614FF0904003F0B3FD4FF4FC
:10410800C0501123CDE9010301A901234FF09040CC
:10411800039303F081FC08240A2500224FF4805100
:104128004FF0904003F09EFD0120FEF7F9FC0122BC
:104138004FF480514FF0904003F094FD0120FEF7BA
:10414800EFFC013DE9D14FF400614FF0904003F0DE
:1041580083FD08B9013CDFD14FF400614FF0904076
:1041680003F07AFD044660BB0425FFF7A2FF012691
:1041780003900DEB05012A48CDE9015603F04CFCEC
:1041880032462946264803F06DFD2120FEF7C8FC7B
:1041980022462946224803F065FD2120FEF7C0FC8F
:1041A800324629461E4803F05DFD2120FEF7B8FC83
:1041B8001B482246294603F055FD4FF42570FEF7AB
:1041C800AFFCFFF776FF4FF0B04300249A6D42F43E
:1041D80080029A659B6D03F4800300934FF4C052EC
:1041E800009B1223CDE901230323CDE903430423D4
:1041F8000DEB03014FF09040059303F00DFC0948C7
:104208000949846040F61463C0E900130123C0E93A
:104218000334C0E90744446103F0A0FE06B070BD52
:10422800000400480C0E002000580040FFF750BF63
:1042380010B1012809D0704701394A424A414FF06C
:1042480090404FF4007103F00DBD4B1E5A420248D6
:104258005A412021F7E700BF00040048FFF7E6BFF6
:1042680000F016B9054B1A6802805A689B684381AA
:10427800034B028101221A70704700BF640E0020B0
:10428800E30D002010B5044600F008F810F0FF0018
:104298001CBFEE232370AA23637010BD2DE9F743DA
:1042A80000242D4E2D4D346021462046FFF7C0FFD7
:1042B80021460120FFF7BCFF21460220FFF7B8FF87
:1042C8005227A046012195F8640185F86071C5F868
:1042D8006881FFF7ADFF0320FEF722FC0DF106020F
:1042E800C021284602F0FCFB80BBBDF806204EF634
:1042F800AA639A422AD14FEA440909F154095FFA9C
:1043080089F94946284600F025F9F8B985F86091F9
:104318000DF10602C021284602F0E2FB284600F013
:10432800D5FA98B9326801231A4432600C4AC5F8A4
:1043380068311168A3400B4313600134032C05F561
:10434800C875BFD1306803B0BDE8F0830021E0B282
:10435800FFF76EFFF1E700BF780E0020B8000020DD
:10436800740E00202DE9F74F344C054604F5966B82
:104378004FF00A0A4FF00E0948F2E8084FF4901778
:104388004FF48046D4F86831002B50D0204600F016
:104398008DFD0DF102020DF10101204600F04EFBEA
:1043A8000DF1030201A9204600F082FE00212046FB
:1043B80000F0D4F801220021204600F094F90122EF
:1043C8001146204600F08FF9022D0ED81C4B33F809
:1043D80015601C4B53F825701B4B53F825801B4B5D
:1043E80013F805901A4B13F805A032460121204610
:1043F80000F0C2F93A460021204600F0BDF94146D6
:10440800204600F0C5F84A460021204600F0C2F8D0
:1044180052460121204600F0BDF80DF102020DF1CF
:104428000101204600F00AFB0123C4F87C3104F5A1
:10443800C874A345A6D103B0BDE8F08FB80000202A
:10444800503B0108443B0108383B0108333B010855
:10445800303B010810B50B7E9BB9D0F87C21098947
:1044680012B1C0E95E1310BD084BD0F878411A6844
:10447800C2F580734B4304FB02331B12C0F878313A
:10448800F1E70123C0F87C31EDE700BF68050020A3
:104498002DE9F047DFF8A480294FFFF7C7FED8F8C9
:1044A80000300BB13B6813B9FFF7F8FE38603B6882
:1044B800002B3BDDDFF88C90234D02200024FFF712
:1044C80051FF89F80040D5F86861012E1ED1DFF848
:1044D8007CA02846514600F049FCB8B95146284608
:1044E800FFF7B8FF9AF8183083B9194BD5F8782137
:1044F80043F82420D8F80030A6401E4399F800302D
:10450800C8F8006043F0010389F800301E20013428
:10451800FEF706FB032C05F5C875D4D199F80030D1
:104528000023C8F800303B60BDE8F087084B4FF423
:104538007A721A605A609A60F2E700BF740E00201F
:10454800700E0020E30D0020B80000207C0E002033
:10455800640E00204A088A2102F072BA152906D88A
:10456800044BCB40DB0702D50174002070476FF085
:10457800070070470B00300010B50A460C460921A9
:1045880002F080FA18B9237803F00103237010BDF4
:1045980001F051BE01F02EBD01F033BEF7B5002386
:1045A8000F46144601210DF1070206468DF8073023
:1045B80002F068FA0546D0B9012C9DF8073025D1DC
:1045C800042F39D8DFE807F00316191C1F0043F041
:1045D80010049C420BD022460121304602F030FAEA
:1045E80068BB716986F830413046FFF7D1FF28462D
:1045F80003B0F0BD43F02804EBE743F00404E8E718
:1046080043F04004E5E743F08004E2E7042F13D8C1
:10461800DFE807F00306090C0F0003F0EF04D8E702
:1046280003F0D704D5E703F0FB04D2E703F0BF0497
:10463800CFE703F07F04CCE76FF00305D7E7054623
:10464800D5E713B500230C460DF1070201218DF8BB
:10465800073002F017FA78B99DF80730C3F3001253
:104668002270C3F3C002A270C3F380026270C3F366
:104678008012DB09E270237102B010BD37B50D4618
:104688000DF10202F821044602F02AFA70B901AAD3
:104698000421204602F042FA40B9BDF802201AB1BE
:1046A800019BB3FBF2F32B602B68A36103B030BD11
:1046B800037F0B700020704737B50D460DF10602D9
:1046C8002021044602F00CFA28B9BDF8063023B9B7
:1046D800236A2B60207703B030BDDB002B60236298
:1046E80001232377F7E70529F8B504460E46154652
:1046F80033D862B100EB810301215A6B0023701E8D
:10470800042807D8DFE800F010191C1F26001146FE
:104718000123F4E784F82810003D344418BF01252C
:1047280084F82850002007E0C2F34F224421204695
:1047380002F096F90028EFD0F8BD84F82A10EBE7CC
:1047480084F82B10E8E75B00FE226021204602F087
:10475800B0F9EFE71B01EF22F7E76FF00300EBE793
:10476800052996BF4018002390F82830137094BF8D
:1047780000206FF00300704770B54318044693F8A3
:1047880028300E4615463BB105291BD8DFE801F055
:10479800030912141616426304EB860400206563AD
:1047A80007E0C2F34F224421204602F059F90028BD
:1047B800F2D070BDC263EFE70264EDE7C2F34F22A7
:1047C8006421F1E76FF00300F3E737B504461546B7
:1047D80005292AD8DFE801F0030614161818436BD8
:1047E8002B601FE00DF10602442102F079F9D0B9DF
:1047F800BDF8062053028AB12B60A36301230FE0A2
:10480800C36BEDE7036CEBE70DF10602642102F0E0
:1048180067F940B9BDF806305B02E1E7A26B2A6090
:1048280084F82930002003B030BD6FF00300FAE7A8
:1048380037B50D460DF107020121044602F022F9B1
:1048480038B99DF8073084F83031DB092B7084F8CB
:104858004C3003B030BD2DE9F843037C0C4601F819
:10486800083B0546FFF70AFF40BB207304F110011F
:104878002846FFF721FF08BB04F11401284600F081
:1048880019FCD8B904F1240705F1270904F1170820
:1048980006463A46B1B22846FFF797FF70B9013687
:1048A80019F8013F08F8013F062E07F10407F0D177
:1048B80004F13C012846FFF7BBFF08B1BDE8F883C7
:1048C800211D2846BDE8F84301F01DBDF0B50022C2
:1048D800054693B0882102F0B3F84FF47A72A5F830
:1048E80052214FF4C872A5F85421514AC5F85821ED
:1048F8000023504A85F8F030C5F8D4202B6202A96D
:104908002846FFF7A8FF044670B9ADF8080002AEC4
:104918000FCE05F110070FC70FCE0FC70FCE0FC769
:1049280096E80F0087E80F00434BC5F834314FF481
:10493800FA730126A5F838314FF42063A5F83C3105
:104948003246802185F85061284602F079F83246CF
:104958000746FF21284602F073F800221146074354
:10496800284602F06DF83C4364B204430DF1070297
:104978009121284602F086F864B29DF8073085F840
:104988003A31044332460021284602F059F864B20D
:1049980004430022FF21284602F052F864B204437F
:1049A80000228021284602F04BF864B2204340B22E
:1049B80000283BD013B0F0BD0028FBD1A1B20122E2
:1049C80028460134FFF78FFE062CF5D10028F1D1D7
:1049D80004466885024604212846FFF784FE00281D
:1049E800E8D1024605212846FFF77DFE0028E1D1DF
:1049F8004FF490136B634FF4804201212846FFF770
:104A0800BBFE0028D6D14FF40C13FF22C5E90F30A6
:104A180085F830210121284602F012F8012385F893
:104A280032310028C6D185F81541C3E70446C5E7E9
:104A3800856B0100A470090064008403012300F061
:104A480069BD2DE9F0428EB00C460C2304AA14214E
:104A5800054601F0DDFF8446002860D1BDF8162028
:104A6800BDF81830A075BDF81210206052BA5BBAB4
:104A78006060BDF81A60B5F8520192B29BB249BAAB
:104A88005B0252022361A18276BAE260B0F57A7FB6
:104A98008BB295F831719DF81010B6B20AD07043F8
:104AA80000F5FA704FF47A76B0FBF6F02E7F002E00
:104AB80039D186B2002F40D0B001C0B2B608E07537
:104AC8000DF10F002681CDE90040284601F072FE65
:104AD800844620BB9DF80FE084F818E005F15006E5
:104AE8000FCE07AF0FC796E80700E37D87E80700FA
:104AF800D4E90301A28AADF83020D4E90149CDE90F
:104B08000A01CDE9084907AC8DF833308DF834E057
:104B18000FCC50350FC597E8070086E807006046B8
:104B28000EB0BDE8F0822E8C5E43B2EB262F4FEA22
:104B3800262C04D157B948F6E0260020BFE780B2FA
:104B48005043A2EB0C06B0FBF6F0B2E742F2B826EF
:104B5800B2E70000F7B517460E210DF106021D4613
:104B68000B4C064601F0BCFFBDF8063004EA43438F
:104B78003B6050B90DF106020C21304601F0B0FF40
:104B8800BDF8063004EA43442C6003B0F0BD00BF12
:104B98000000FE1F73B590F8DA30013B022B064681
:104BA8000C4634D801AB6A460121FFF7D3FF009BBE
:104BB800B3F57F0F054603D8019BB3F57F0F23D9C3
:104BC80015BB34B11349304602B0BDE8704001F05E
:104BD800FFBB0422FF21304601F032FF2A4604467B
:104BE8007021304601F02CFF2A460443FF2130464D
:104BF80001F026FF64B204432A468021304601F0C2
:104C08001FFF64B2044365B2284602B070BD002598
:104C1800FAE700BF6C05002037B504460122802161
:104C2800057C01F00DFF0122FF21204601F008FF5D
:104C380000221146204601F003FF94F83A21912101
:104C4800204601F0FDFE01220021204601F0F8FE79
:104C58000022FF21204601F0F3FE00228021204699
:104C680001F0EEFE012D24D0032D32D0C5BB012268
:104C78002946204601F0E4FE01238DF80730B0B93B
:104C880005469DF80730DB0705F101050AD548B947
:104C9800B5F5FA6F27D001460DF10702204601F05D
:104CA800F1FEEEE7B5F5FA6F08BF6FF0060003B046
:104CB80030BD18B929462046FFF76CFF02220021B3
:104CC800204601F0BDFE0028F1D1042384F83231DA
:104CD800EDE718B901212046FFF75CFF0422EEE753
:104CE8006FF00700E3E76FF00600E0E738B5057CF2
:104CF800044625B1204600F03BFD28B138BDFFF73A
:104D08008BFF0028F6D0F9E7002DF7D1032384F8AC
:104D18003231F3E773B50646002501220B213046F0
:104D280001F08EFE002204460B21304601F088FE79
:104D38000DF1070204431321304601F0A3FE9DF84C
:104D4800073064B2044301355B0760B2EDB205D0A9
:104D5800032D08D00028E0D002B070BD032D08BF95
:104D68006FF00B00F8E76FF00B00F5E738B500239C
:104D7800037404460D46FFF7B9FF50B9294620468B
:104D8800FFF75FFE28B901462046BDE83840FFF727
:104D9800C1BF38BD152970B5054616461C4667D1F2
:104DA8000122FF2101F04CFE00221146044628464C
:104DB80001F046FE00220443FF21284601F040FE90
:104DC80064B2044301228021284601F039FE64B20E
:104DD800044302228521284601F032FE64B20443CE
:104DE8000422FF21284601F02BFE64B2044300226E
:104DF800CD21284601F024FE64B204431122CC21BF
:104E0800284601F01DFE64B204430722FF2128460C
:104E180001F016FE64B204430022BE21284601F0C8
:104E28000FFE64B204430622FF21284601F008FE63
:104E380064B204430922CC21284601F001FE64B281
:104E480004430022FF21284601F0FAFD64B204431E
:104E58000122FF21284601F0F3FD64B20022044339
:104E68001146284601F0ECFD64B2204340B270BD03
:104E7800042A17D80A2101F0E3FD0028F7D1231EE0
:104E880018BF01231B01EF228421284601F011FEDF
:104E98000028ECD185F8DA6001462846BDE8704064
:104EA800FFF738BF6FF00A00E1E7000070B594B073
:104EB80005464022002104A80EF0C6FC002301216B
:104EC8002846ADF806308DF803308DF8043002938B
:104ED80000F0A0FC95F8142195F81311012A04D8C4
:104EE80040F0AD80202940F2AC8001AA02A92846F2
:104EF80000F02BFB0446002840F09E8095F85031C6
:104F0800002B40F0A280D5F84C11284601F060FA39
:104F18000446002840F090800346014604222846B3
:104F2800FFF738FF0446002840F086800122FF2161
:104F3800284601F085FD0DF1060206468421284623
:104F480001F0CEFD22460643FF21284601F078FDF8
:104F580076B2064374B2002C6ED1BDF806301B0140
:104F6800C5F8D43004A92846FFF775FC0446002884
:104F780062D10DF103012846FFF7FEFA0446002826
:104F88005AD19DF8033085F8313104AC0FCC05F1C6
:104F980010060FC60FCC0FC60FCC0FC694E80F0033
:104FA80086E80F000DF103020121284601F06AFD91
:104FB8000446002840D19DF8033085F83031024678
:104FC80001462846FFF7EAFA0446A8BB0246022132
:104FD8002846FFF7E3FA044670BB0323014685F829
:104FE80032310DF10502284601F00BF9044618BBD1
:104FF8009DF8053085F8E8300DF1050201212846B5
:1050080001F0FFF80446B8B99DF8053085F8E0309E
:1050180003AA0321284600F0E7FE044660B9039B73
:10502800C5F8E43003AA0421284600F0DDFE044652
:1050380010B9039BC5F8DC30204614B070BD0C29AC
:1050480051E7284600F013F954E701495DE700BF2E
:105058002207002013B50C460DF10702132101F0B9
:1050680011FD9DF8073013F0180F03F0070218BF61
:105078006FF00500226002B010BD13B590F8DA3069
:10508800042B0C4609D101A9FFF7E4FF019B1A1F65
:1050980053425341237002B010BD01AA142101F0FC
:1050A800F1FC0028F7D19DF8043003F00103F1E783
:1050B80000F04BBA13B50C460DF10602282101F099
:1050C8000FFD78B9BDF80620C2F30B0312F4006F88
:1050D80018BFA3F580534FF0FA0214BF13FB02F375
:1050E8005343236002B010BDF0B54FEAD20C4FF025
:1050F800FF341C6002F00702664600278E4200D289
:1051080007B1F0BD845D664503BF1441E4B215469E
:105118003D4614F0010705D005EBC6051D600127C3
:105128000136EBE70135082D4FEA5404F8D014F0A6
:10513800010FF0E7034B800953F82000003818BF2F
:10514800012070471808002010B5B1EBD20F4FEAC4
:10515800D20402F0070381BF01229A40035D134382
:105168008ABF03556FF03100002010BD0A460623A0
:10517800B02101F02FBC0A460623B02101F048BC3B
:105188002DE9F04F85B00546109F0E9E01978A467F
:1051980093461C464FF00009119B994508D10023FE
:1051A800129A176013B36FF0310005B0BDE8F08FA5
:1051B80001AB3A4631465846FFF796FFDDF80480C2
:1051C800B8F1FF3F0FD00F9B08EB0300FFF7B2FFCA
:1051D800504508D142462046FFF7B6FF08F10107BF
:1051E80009F10109D8E76FF03103D9E721462846CC
:1051F800FFF7BCFF0028D8D102A92846FFF7BBFF5C
:1052080002ABA2199442D0D014F8015B13F8011B29
:105218008D42F7D0C7E770B5C02288B00E4601218D
:1052280090F83051044601F00BFCF0B901A9204672
:10523800FFF79CFDC8B90122FF21204601F000FCC0
:1052480098B93246B621204601F04AFC68B90246B0
:10525800FF21204601F0F4FB38B92A4601212046F7
:1052680001F0EEFB08B984F8305108B070BDF0B514
:105278000F4689B01646FF210122044601F0E0FBE3
:105288000246A8B94F21204601F0DAFB80B92C224A
:105298004E21204601F0D4FB024648B9FF212046A2
:1052A80001F0CEFB20B9B422B621204601F0C8FB9C
:1052B8000025C4F82451A4F82851DEB9354607ABB7
:1052C800B422CDE903730623CDE90032029504F533
:1052D800927304F5957231462046FFF751FF30B9B5
:1052E800012384F8153184F8137184F8146109B026
:1052F800F0BD013505F1B400FFF71CFF0028DED131
:105308002C2DF6D1DBE710B541F00102002104464F
:1053180001F096FB78B9204600F02AFA58B9014600
:105328002046FFF7F7FC30B9024601462046BDE8A3
:10533800104001F085BB10BD2DE9F74F4FF0000B71
:1053480088461746FF21012205461E469DF838A0CB
:105358009DF83C908DF807B001F072FB5A46044660
:105368005946284601F06CFB5A460443FF2128465B
:1053780001F066FB64B2044364B2B8F1000F32D0A6
:10538800BAF1000F06D00C9ACB21284601F07AFB1F
:10539800204344B2B9F1000F07D00DF10702EE2106
:1053A800284601F06FFB204344B20122FF21284622
:1053B80001F046FB012204430021284601F040FB8E
:1053C80064B204430022FF21284601F039FB64B28D
:1053D8009DF807300D9A204323F0100340B2137054
:1053E80003B0BDE8F08FBAF1000F06D03A46CB21E2
:1053F800284601F025FB204344B2B9F1000FD4D070
:1054080033468022EE21284601F053FBCBE72DE9F5
:10541800F04387B09146002205460E468DF81720C6
:105428001F4653B390F8308101221146284601F0F7
:1054380007FB044648BB40212846FFF764FFF0B944
:10544800B9F1010F24D10DF11703CDE90294CDE98B
:1054580000632246234649462846FFF76DFF044667
:1054680078B947B142460121284601F0E9FA0446D5
:1054780038B985F83081002403E09846D4E73470C1
:105488000446204607B0BDE8F08300233370F8E7F0
:105498003070E6E72DE9F043054687B00E469146A1
:1054A8001F4653B390F8308102220121284601F0AB
:1054B800C7FA044648BB01462846FFF724FFF0B95F
:1054C800B9F1010F24D10DF11703CDE90249009379
:1054D80022462346019649462846FFF72DFF0446F3
:1054E80078B947B142460121284601F0A9FA044695
:1054F80038B985F83081002403E09846D4E7347041
:105508000446204607B0BDE8F08300233370F8E76F
:105518003070E6E7F8B51D46164600232A4690F88F
:1055280030710446FFF773FF70B903462A463146C7
:105538002046FFF7AFFF38B93A460121204601F06F
:105548007FFA08B984F83071F8BD2DE9F04F0023CF
:1055580093B0CDE90A12C0F82431A0F8283101220D
:10556800FF21CDE90E33B0F83C818DF83430044684
:105578008DF8353001F064FA002840F0F0800246DA
:105588004F21204601F05CFA002840F0E8802C22E8
:105598004E21204601F054FA002840F0E0800246EF
:1055A800FF21204601F04CFA002840F0D880B422B0
:1055B800B621204601F044FA002840F0D080024687
:1055C8008021204601F03CFA002840F0C8800346BC
:1055D8000DF135020DA92046FFF79CFF002840F089
:1055E800BE8004F5957307930323CDE90203B42124
:1055F800062304F592790EAECDE9003104960146F2
:105608004B4604F595722046FFF7BAFD002840F096
:10561800A6800DF1360120460E9DFFF7FCFD0028FF
:1056280040F09D80BDF83630434541D9C4F8240187
:10563800A4F8280105F1B400FFF77CFD08B92B2D6B
:105648001FD90623B42204960326CDE90032CDE9FA
:105658000256079A4B4601212046FFF791FD002884
:105668007DD10DF1360120460E9DFFF7D4FD0028AF
:1056780075D1BDF83630434574D901274FF0010A7A
:1056880019E00135D6E7089E099324E0089E0A9B95
:105698001E600B9B1F70012384F815310A9B1B6841
:1056A80084F813310B9B1B7884F81431002056E0E2
:1056B80000273E46BA46BDF836304345E7D2A3EB4D
:1056C800080383EAE372A2EBE3725FFA8AF70992AE
:1056D800032604F5927BDBF80000BBF80430109039
:1056E800ADF844302A460FAB07980621FFF7FCFCBB
:1056F8000F9D6B1C39D005F1B400FFF71BFD504519
:10570800C5D1731C2A4648460893FFF71DFD30BBD8
:10571800494620460135FFF729FD00BB0DF136014A
:105728002046FFF778FDD0B9BDF83620A2EB080374
:10573800002BB8BF5B424245A5D9099A9342A5D927
:1057480010A92046FFF712FDBDF844200346109823
:10575800C4F82401ABF804201846002B97D013B0E6
:10576800BDE8F08F0746064688E76FF03100F6E798
:1057780037B5002304468DF807304FF4FA650DF16C
:1057880007012046FFF779FC58B99DF80730012B2F
:1057980007D0013D03D0204601F0DEF9EFE76FF0B6
:1057A800060003B030BD02464FF08043934202D852
:1057B800002013B970479B08F8E7C11891424FEAD7
:1057C80050009CBFC018521A9B08F2E773B500221C
:1057D8008321054601F034F9044690B906460DF1D7
:1057E80007028321284601F04DF99DF8073003434D
:1057F800DBB204462BB90136B6F5FA6FEFD16FF07C
:10580800060401228321284601F01AF9204340B2F8
:1058180002B070BD2DE9F04F90F8F06091B04FF0F4
:105828000009072ECDE9079904460F4600F0A28229
:105838000122802101F004F901228046FF2120463F
:1058480001F0FEF84A4648EA00084946204601F0B9
:10585800F7F84FFA88F848EA00080622FF212046A0
:1058680001F0EEF84FFA88F848EA00080DF1150241
:105878008321204601F006F99DF815204FFA88F893
:1058880048EA000842F004028321204601F0D8F8D3
:105898004FFA88F848EA00080722FF21204601F05D
:1058A800CFF84FFA88F80122812148EA00082046FB
:1058B80001F0C6F84FFA88F848EA0008204601F0D7
:1058C8004BF94FFA88F848EA00080122802120465F
:1058D80001F0B6F84FFA88F848EA000517F0010B0E
:1058E8006DB200F01E82F20700F11E826B22942135
:1058F800204601F0A5F880462046FFF767FF06AA74
:1059080048EA00089021204601F008F945EA080510
:10591800069B6DB22422942105432046C3F3062A30
:10592800C3F3C03901F08CF86DB205432046FFF788
:105938004DFF6DB2054306AA9021204601F0EEF80E
:10594800069B6DB21BBA2522942105432046099374
:1059580001F076F86DB205432046FFF737FF6DB2C8
:10596800054306AA9021204601F0D8F8069B6DB29F
:105978001A0E05431B0C6DB28DF828208DF82930BE
:1059880017F00203029300F0DB8016F0020840F0E3
:10599800D78002229421204601F052F80190204637
:1059A800FFF714FF019B0DF11602034390212046D7
:1059B8001D4301F067F86DB27B2294210543204610
:1059C80001F03EF86DB205432046FFF7FFFE6DB2C9
:1059D80005430DF117029021204601F053F86DB2EE
:1059E800772294210543204601F02AF86DB2054339
:1059F8002046FFF7EBFE6DB2054306AA902120462C
:105A080001F08CF8069B5A0E8DF82C20C3F38642C1
:105A18008DF82D20C3F3C6228DF82E206DB2C3F366
:105A28000612DB0003F07803942105438DF82F203C
:105A3800204678228DF8153001F002F86DB2054342
:105A48002046FFF7C3FE6DB2054306AA9021204603
:105A580001F064F8069B9DF8152002EB53728DF84F
:105A68003020C3F386528DF83120C3F3C6328DF847
:105A78003220C3F306228DF833206DB2C3F34602F9
:105A88009B0103F04003942105438DF83420204600
:105A980079228DF8153000F0D3FF6DB2054320460A
:105AA800FFF794FE6DB2054306AA9021204601F047
:105AB80035F8069B9DF8152002EB93628DF835208A
:105AC800C3F3C6428DF83620C3F306328DF837206B
:105AD8006DB2C3F346129B0003F07C039421054387
:105AE8008DF8382020467A228DF8153000F0A8FF6E
:105AF8006DB205432046FFF769FE6DB2054306AA5D
:105B08009021204601F00AF8069B9DF815208DF893
:105B18003E8002EB93728DF83920C3F3C6526DB202
:105B28008DF83A20C3F3064205438DF83B20C3F3B2
:105B38004622C3F386036DB28DF83C208DF83D30C4
:105B480017F00403019300F0F180730700F1EE8071
:105B58007B229421204600F073FF80462046FFF701
:105B680035FE07AA48EA00089021204600F0D6FF33
:105B780045EA08084FFA88F848EA00057C2294218B
:105B8800204600F05DFF6DB205432046FFF71EFE7C
:105B98006DB2054308AA9021204600F0BFFF6DB200
:105BA800732294210543204600F04AFF6DB2054355
:105BB8002046FFF70BFE6DB2054306AA902120464A
:105BC80000F0ACFF069B6DB21B02742294210543C2
:105BD80020461FFA83F800F033FF6DB205432046D4
:105BE800FFF7F4FD6DB2054306AA9021204600F0A8
:105BF80095FF6DB29DF81B30752294210543204610
:105C080043EA080800F01CFF6DB205432046FFF781
:105C1800DDFD6DB2054306AA9021204600F07EFF07
:105C2800069B6DB21B029BB2762294210543204647
:105C3800039300F005FF6DB205432046FFF7C6FD4C
:105C48006DB2054306AA9021204600F067FF6DB2A9
:105C58009DF81B20039B05436DB21343002281214D
:105C68002046039300F0ECFE06220543FF21204660
:105C780000F0E6FE6DB205430DF1150283212046C2
:105C880000F000FF9DF815206DB2054302F0FB02FD
:105C98008321204600F0D4FE6DB205430122FF2186
:105CA800204600F0CDFE6DB20543012200212046BA
:105CB80000F0C6FE6DB205430022FF21204600F029
:105CC800BFFE6DB2054300228021204600F0B8FED9
:105CD8006DB205436DB2039BFDB9BBF1000F29D12D
:105CE800029AAABB019AAAB1720713D4079AC4F8F8
:105CF8001821089AC4F81C214FEA4822C4F8202128
:105D08003BB1A3F5C8534FF47A7253431B095B4266
:105D18001BB2E3603E4384F8F060284611B0BDE84A
:105D2800F08FD946DA462BE6CA4629E64FF0000836
:105D3800434693E7F007D3D40998BDF8282084F8A0
:105D480013A184F81491C4F82A01A4F82E21C7E7F6
:105D5800B107C7D49DF8162084F8F1209DF81720C4
:105D680084F8F2200BA904F1F30002930DF098FDDA
:105D7800029BB7E74D46D0E740B101380023FF2822
:105D880003F1010203D800EB032080B270474008FA
:105D98001346F4E7C3B2000A03FA00F00130704773
:105DA800084B5A434FF47A7302F5FA724FF4FA60CB
:105DB800B2FBF0F0B2FBF3F203FB0100B0FBF2F030
:105DC800704700BF002F3A00064B5A434FF47A70D1
:105DD80002F5FA72B2FBF0F24A4302F5FA72B2FB2C
:105DE800F0F07047002F3A002DE9FF4102294FF0EB
:105DF8000005074616468DF80350ADF804501CD828
:105E08000DF102022946FEF7C7FB044630B90DF131
:105E180003024621384600F035FE04469DF803008B
:105E2800FFF7B8FF81B29DF802203846FFF7CCFF94
:105E38003060204604B0BDE8F081032918D10DF187
:105E480002022946FEF7A8FB0446002846D101466F
:105E58000DF102023846FEF79FFB044628B901AA55
:105E68005121384600F03CFE0446BDF80400D7E74F
:105E7800042935D102A9FEF7E4FB9DF80B304BB39A
:105E88000DF1020229463846FEF786FB044618BB88
:105E980001AA5121384600F023FE0446BDF804004B
:105EA800FFF778FF85B2BCB90DF10202012138462F
:105EB800FEF772FB044678B90DF1060271213846E7
:105EC80000F00EFE0446BDF80600FFF763FF80B23F
:105ED800401BA7E71D46E7E70020F9E72846A7E7A4
:105EE80028462C46A4E7F0B5022985B00546164693
:105EF8001ED80DF105020021FEF74EFB0446A0B99D
:105F08009DF8052031462846FFF74AFF83B2B3F5CE
:105F1800807F9ABF00F1FF32D2B2FF22A5F8D820C5
:105F28004621284600F08CFD0446204605B0F0BD09
:105F3800032920D10DF105020021FEF72DFB9DF864
:105F48000520044631462846FFF72AFF80B2FFF7AE
:105F580013FF0246ADF80600A5F8D800002CE4D1DE
:105F68005121284600F07CFD04460028DDD1C5F803
:105F7800E4600024D9E7042939D102A9FEF761FBBE
:105F88009DF80B70B7B10DF1050200212846FEF708
:105F980003FB04460028C8D10DF10602512128460A
:105FA80000F09EFD04460028BFD1BDF80600FFF7AB
:105FB800F1FE87B20DF1050201212846FEF7ECFA41
:105FC80004460028B1D19DF8052031462846FFF740
:105FD800E7FE3844FFF7D0FE71210246284600F05C
:105FE8003FFD04460028A0D1C5F8DC60C1E76FF08A
:105FF80003049AE7F0B585B000238DF80330D30782
:1060080005460F46164605D441B9A2F10C03DAB28B
:10601800062A12D96FF0030005B0F0BD012920D17E
:10602800A2F10803DAB2062AF4D8062B19D8DFE859
:1060380003F03718651886189900062B11D8DFE881
:1060480003F0041029102B102D0018225721284680
:1060580000F0F6FC08225621284600F0F1FC002842
:10606800DAD17408013CE4B2002F00F08E80012FD1
:10607800D0D101AA04212846FFF7B6FE38B9224636
:106088007021284600F0DCFC002800F0B28085F87A
:10609800E060C1E73022D9E74022D7E75022D5E7B0
:1060A8001022482100F0CCFC08224721284600F0A5
:1060B800C7FC022204463221284600F0C1FC0C220B
:1060C80004433021284600F0BBFC64B2044301229B
:1060D800FF21284600F0B4FC64B2044364B23022C5
:1060E8003021284600F0ACFC00220443FF2128465A
:1060F80000F0A6FC64B2204340B2B0E72822482151
:1061080000F09EFC08224721284600F099FC032253
:1061180004463221284600F093FC044364B2092265
:106128003021284600F08CFC01220443FF21284638
:1061380000F086FC64B2044364B22022D0E738221F
:10614800482100F07DFC08224721284600F078FC11
:10615800032204463221284600F072FC044364B24C
:106168000822DDE74822114600F06AFC0822472190
:10617800284600F065FC032204463221284600F038
:106188005FFC044364B20722CAE702AA0321284637
:10619800FFF72AFE88B903AA02212846FFF724FE42
:1061A80058B922465021284600F04AFC28B9029ADC
:1061B80003212846FFF797FE10B185F8E8602BE722
:1061C800039A02212846FFF78EFE85F8E86000282A
:1061D8007FF422AF69692846FEF7DAF900287FF4D0
:1061E8001BAF024601230DF103012846FFF752F9C0
:1061F80012E7019A04212846FFF775FE85F8E0604A
:10620800E5E713B5144629B1012910D06FF0030052
:1062180002B010BD0DF10702502100F033FC002838
:10622800F6D19DF8073001335B002370F0E70DF1DC
:1062380007027021F1E7F0B5002385B04FF4FA6248
:10624800CDE9002344F61F63994206460F4604D859
:106258006FF00305284605B0F0BD02A9FEF7F1F975
:1062680005460028F6D19DF809209DF8083013430B
:106278009DF80A201343A7F636341BD06A4602213C
:106288003046FFF7B1FD00283BD19DF808302BB10F
:10629800009B03F24E239C42DAD9E41A9DF80A3097
:1062A80023B3009B03F2B223B4EB430F4FEA43023C
:1062B800CED9A41A9DF80B305BB101AA0321304650
:1062C800FFF792FD019B03F525739C42C0D9C0B925
:1062D800E41A9DF80C30002BBCD0A4F2262204212D
:1062E8003046FFF700FE77610546B3E79DF80930B1
:1062F800002BDFD0009B03F525739C42A8D9E41A34
:10630800D8E70546A6E770B54FF4FA6286B00023D1
:10631800CDE9022340F636330B600C4604A9064645
:10632800FEF78FF90546002836D19DF811209DF813
:10633800103013439DF81220134319D002AA0221EA
:106348003046FFF751FD002840D19DF810302BB1A1
:10635800029B03F24E222368134423609DF81230F7
:10636800EBB1029B03F2B222236803EB42032360E2
:106378009DF81330EBB99DF814305BB101AA0421E4
:106388003046FFF731FD019B03F2262223681344B0
:106398002360D8B923687361284606B070BD9DF89C
:1063A8001130002BE4D0029B03F5257223681344B7
:1063B800DDE703AA03213046FFF716FD039B03F52B
:1063C80025722368134423600028D4D00546E3E7E8
:1063D8002DE9F743002406460D46204615F80480AB
:1063E800B8F1000F00D010B103B0BDE8F083671C0E
:1063F800B8F1FF0F15F8079029D1A71CEB5DB9F18B
:10640800030F36D8DFE809F0020B131B271D2C44B5
:10641800E27802EB0323A6F834313C46DEE7271D79
:106428002C44E27802EB0323A6F83631F5E7271D62
:106438002C44E27802EB0323A6F83831EDE7271D58
:106448002C44E27802EB0323A6F83C31E5E7B8F1E7
:10645800040F0ED802344246291901A80DF02DFA6E
:10646800434601AA4946304604EB080700F0B2FA51
:10647800D3E76FF00300D0E773B500230E4613602F
:106488000DF1070105461446FEF712F940B99DF8CB
:1064980007302BB1B38A2A6A534380331B0A23601F
:1064A80002B070BD13B5CB681360144601AAFFF79C
:1064B800E3FF18B92368019A1344236002B010BDA2
:1064C800F8B5B0F85451D0F8580168438030000A44
:1064D8000E464543DDE90717144652B1B60206EBEE
:1064E8005202B2FBF4F202EB4202524302F50042BE
:1064F800140C069A534301F50042120C062003328D
:10650800B2FBF0F2C2EBC202B2F5803F38BF0331F2
:1065180003F500433EBFB1FBF0F1C1EBC10101F54A
:1065280000414FEA134334BF090C1B4903FB03F333
:1065380038BF494303EB57030B44B3FBF7F39B0303
:10654800FE2205F120007F33B3FBF2F35C434FF4E6
:106558007A7704F5FA748009B4FBF7F42401FFF79D
:1065680022F904F5FA74BC4228BF4FF4FA630646D0
:1065780029BFB4FBF3F300205B19B4FBF7F428BF81
:10658800B3FBF4F0FFF70FF9099B864294BF1E6036
:1065980018600020F8BD00BF0000F0FF2DE9F04FA3
:1065A80091B0054607930B6908930F46CB680B9388
:1065B80093460FAAFFF776FF0EAA39462846FFF73B
:1065C8005BFF48BB0F9C95F8E0A0D5F8DC3005933D
:1065D8004FF47A7606FB04F101F50041049180340A
:1065E8000E99099124F0FF010A910F910499D5F8A9
:1065F800E4300693BAF1080F0CBF02230323090CF9
:1066080095F8E820DFF898810C9108D1079BCBF822
:106618000080C5F84081186011B0BDE8F08F069978
:106628000D932846FFF7BCFB52460599814628463C
:10663800FFF7B6FB0D9B5B490C9A814403FB09F9F4
:106648004FEAC92940F2776309F5FA79240AB9FBB8
:10665800F6F903FB09F909F5FA79B9FBF6F909FB2B
:1066680004F404F18003089C74430C40B4FBF2F476
:106678004D4A1B0A944228BF1446012B38BF0123F8
:106688000C204FF4167258435443FFF78CF83B7EA6
:106698003A894FEA400A002B7FD14249049B0B40BC
:1066A80003F5FA71414B5A4341F25C23B2FBF3F212
:1066B800099B7343B3F5481F28BF4FF44813A1EB58
:1066C8004303B1FBF6F1B3FBF6F31B02B3FBF1F6A0
:1066D8003602C6F58036564306F50046360C06F5F2
:1066E800803676087643B60B4FF44873734303F548
:1066F800004304F500401B0C5B43000C00FB00301A
:10670800FFF751F803046422323341F28837B3FBB0
:10671800F2F340F6B532B3FBFAF302FB0377244BEE
:106728009F429CBF42F21073B7FBF3F7DDE90532D5
:10673800134403F5FA734FF47A7A4FF4FA62B3FB11
:10674800FAF0B3FBF2F202F5C812B2FBF0F088BF20
:106758004FF47047FFF727F8000200F5FA70B0FB16
:10676800FAF0404307FB0700FFF71DF80AFB00F0AB
:10677800079B404528BF4046CBF80000C5F84001BC
:10678800CDE902934FF448730093DDE90A120194AE
:1067980033462846FFF794FE3EE74FF48036A3E7DA
:1067A800AE878F020000FFFF666666009A990600B2
:1067B8000F279F242DE9F04F11F0780F8BB018BFE9
:1067C8004FF2A009C1F3C30B18BF29FA0BF9904681
:1067D8009A460DF10E024FF000034FF00001159F8D
:1067E8008DF80E3004468DF80F308DF810308DF886
:1067F8001130ADF81230099314BF09F001094FF0B8
:106808000109FDF7ADFF9DF80E500646D5B10028E9
:1068180040F09A80149909AB05AA2046FFF7BEFEFE
:10682800002840F09380149A099B5381014606AAD8
:106838002046FDF7CAFF069D25B1059B9D422CBF4A
:106848000025012520B904AA02212046FDF788FF6A
:106858009DF8106026B300287AD107AA02212046A5
:10686800FDF7B3FF88B90122FF21204600F0E8F8C0
:1068780058B90DF11202B621204600F031F920B9BD
:106888000246FF21204600F0DBF8BDF81230079ED3
:106898005B02C4F848311EB19E422CBF0026012677
:1068A80028B90DF1110203212046FDF759FF9DF883
:1068B800113093B100286CD1BAF1000F03D04FEA20
:1068C8000828B8FBFAFA08AA03212046FDF77DFF3D
:1068D800089B534594BF0023012320B9B9F1000F49
:1068E80038D0FF223A703A780AB914994A810DF1E2
:1068F8000F02012120460193FDF732FF08BB9DF8E6
:106908000E20019B002A08BF0125BBF1040F18BF08
:106918009DF80F2084F82E501ABFB2FA82F252095D
:10692800012284F82F209DF81020002A9DF81120BC
:1069380008BF0126002A08BF012384F8306084F8C4
:1069480031300BB0BDE8F08F002581E735467FE791
:106958000026ACE70BF1FF32092A0AD8DFE802F07B
:10696800050505090907090B070B0522BAE70422E3
:10697800B8E7012E01D10322B4E7BBF1040F01D01F
:10698800012B01D10222ADE7012D16BF00233D7076
:106998003B700023A7E707B502F10A03009393B2FF
:1069A8000A4690F86011D0F85C0101F029FB03B0A9
:1069B8005DF804FB13B502F10A0390F860410093F7
:1069C800D0F85C0193B20A4644F0010101F0AEFB35
:1069D80002B010BD3F2BF8B50E46054611461C46C1
:1069E80011D80A4F38461A4600F8016B0CF065FFBB
:1069F800621C39462846FFF7CEFF002814BF6FF007
:106A080013000020F8BD6FF00300FBE7980E00208C
:106A180073B515468DF8071001220DF107010446DC
:106A28001E46FFF7B8FF18B16FF0130002B070BD33
:106A3800324629462046FFF7BDFF0028F6D0F3E787
:106A480008B5064B19705A7019460222FFF7A3FFC2
:106A5800002814BF6FF01300002008BD980E002016
:106A680008B5074B1970110A59709A701946032214
:106A7800FFF791FF002814BF6FF01300002008BD36
:106A8800980E002037B515468DF8071001220DF134
:106A980007010446FFF77FFF18B16FF0130003B03A
:106AA80030BD012229462046FFF784FF0028F6D092
:106AB800F3E7F7B515460DF1070206460F461C46E3
:106AC800FFF7E0FF50B99DF807301D4044EA050282
:106AD800394630468DF80720FFF7B2FF03B0F0BD06
:106AE80073B514468DF8071001220DF1070105460C
:106AF800FFF751FF18B16FF0130002B070BD064EDA
:106B0800022231462846FFF755FF0028F3D1338883
:106B18005BBA2380F1E700BF980E002073B51446D6
:106B28008DF8071001220DF107010546FFF733FF25
:106B380018B16FF0130002B070BD064E0422314642
:106B48002846FFF737FF0028F3D133681BBA2360C4
:106B5800F1E700BF980E002008B50220FBF7E0FF20
:106B6800002008BD7047000010B5032000F056FC57
:106B780001F028FD064B18600F20FBF7C7FF0446FD
:106B880018B9FBF74EFE204610BD0124FBE700BFF5
:106B9800280800204FF0E022136923F00203136154
:106BA80070474FF0E022136943F002031361704706
:106BB800014BD3F8900570470070FF1F014BD3F8C5
:106BC800940570470070FF1F014BD3F89805704774
:106BD8000070FF1F8068C0F380007047F7B500237E
:106BE80001930446002800F0E980856D25B9FBF77C
:106BF8002FF9E56584F8545023689A68D00040F16D
:106C0800A1809A68D10000F1B480A26D42F0100210
:106C1800A265E26D42F00102E26501251846FFF720
:106C2800D9FFA26D02F01002024340F0C980A26DA4
:106C3800206922F4817242F00202A2659A68D207A2
:106C48005DD4226BA67E94F82CC0003A18BF0122AE
:106C58001703D4E902120A43217E42EA8132617E97
:106C680042EAC13242EA4632002842EA4C02B4BF44
:106C780020F000414FF400113A430A4394F82010E1
:106C8800012903D1002E76D142F48032616A21B104
:106C9800A66A01F4E07131430A43D968E66C21F42D
:106CA800FE3121F4FF711143D96094F83C206168EA
:106CB800012A01F0404C4CEA060609D1D4E9102714
:106CC8003A433243A66C324342EA0C0242F00106D0
:106CD8001F693E4A3A4032431A6121F00042B2F13C
:106CE800804F0CD0B1F1004F09D0394ED6F80827A3
:106CF80001F4701122F470120A43C6F808275A6981
:106D0800666BA16B22F0070232435A615A6922F07E
:106D1800700242EA01125A61002835D19A6A62F07B
:106D28000F029A625B6903F007039E423CD100237D
:106D3800E365A36D23F0030343F00103A36528462D
:106D480003B0F0BD9A68234922F0104222F01702DE
:106D580042F080529A60204A1268B2FBF1F2013286
:106D680052000192019A002A3FF44BAF019A013A6E
:106D7800F7E7002552E7A16D41F02001A165E16D1B
:106D880041F00101E16581E7B0F5001FCAD19A6AB7
:106D9800E269013A92006FF00F0102F01C0201FA59
:106DA80002F2216E0A43BCE7A36D23F0120343F0FD
:106DB8001003A365E36D43F00103E3650125BEE716
:106DC800A36D43F01003A365F8E700BF02FCFF1FA3
:106DD80000200140400D030028080020F8B545694F
:106DE800082D04460E460AD00368DB68D80705D587
:106DF800A36D43F02003A3650120F8BD0425FBF72C
:106E080087FE074623681A682A4220D0A26D42F4FA
:106E18000072A265DA6812F4406F14D1A27E92B9AA
:106E28001A6812070FD51846FFF7D4FE20BB5A6818
:106E380022F00C025A60A26D22F4807222F0010244
:106E480042F00102A265227EFAB10020D5E7711C4A
:106E5800D9D0FBF75DFEC01BB04201D8002ED1D1BE
:106E680023681B682B40CDD1A26D84F8543042F0C2
:106E78000402A2650320C0E7A26D42F02002A265C9
:106E8800E26D42F00102E265DDE70C221A60DCE700
:106E98000368186C70470000F7B50023019390F859
:106EA8005430012B044600F0C080056802690123B4
:106EB80080F854302846FFF78DFE002840F0AF8058
:106EC800D1E90030022822F004027ED0B2F1004F4E
:106ED800C3F3110E35D1AA6A42EA0E02AA628A6881
:106EE800686902EA032222F07C4222F0FF0220EACB
:106EF80003210A43002B6A611DDA4D4A4D4DD2F831
:106F08000817AB4201F0E07043D10D0213D4D2F858
:106F1800083723F0E073034343F40003C2F808374B
:106F2800454B1A68454BB2FBF3F20C2302FB0333C3
:106F38000193019B53BB0020002384F8543003B015
:106F4800F0BD226E00F01F074FF00F0C0CFA07FC83
:106F58006FEA0C0622EA0C0CBEF1000F11D1C3F344
:106F68008462BA4042EA0C0222668008E269013073
:106F78009042B4D8A86AC3F38362BA400640324349
:106F8800ACE793FAA3F2B2FA82F2EAE7019B013B7B
:106F9800CEE72B4DAB420BD1C901CCD4D2F8083780
:106FA80023F0E073034343F08073C2F80837C2E765
:106FB800244DAB42BFD14B02BDD4D2F8083723F0E1
:106FC800E073034343F48003EFE7B2F1004F01BFDE
:106FD800AA6AC3F311018A43AA62002BABDA1548E7
:106FE80013498342D1F8082709D1D1F8083702F0AC
:106FF800A07223F0E0731A43C1F808279BE71048F2
:10700800834204D1D1F8083702F44002F1E70D4871
:10701800834290D1D1F8083702F0C072E9E7A26D37
:1070280042F02002A265184686E7022087E700BFE3
:1070380000200140001000B028080020400D030087
:10704800004000B8002000B4026838B50446104675
:10705800FFF7C0FD08B9002038BD9368990707D429
:10706800936823F0004323F0170343F01003936061
:10707800FBF74EFD054623689B685B07EBD5FBF7DE
:1070880047FD401B0228F6D923689B685A07F2D5AA
:10709800A36D43F01003A365E36D43F00103E365BB
:1070A8000120D9E773B50023026801939368DD07CF
:1070B800044602D5002002B070BD9168214B1942E8
:1070C80009D0A36D43F01003A365E36D43F00103FA
:1070D800E3650120EFE7936823F0004323F01703EB
:1070E80043F001039360184BD3F8083718021CD4F7
:1070F800637E012BDED0FBF70BFD144E054622689C
:107108001368DB07D6D49368D9075FBF9368334009
:1071180043F001039360FBF7FBFC401B0228EED908
:1071280023681B68DA07EAD4CBE7094B094A1B68CE
:10713800B3FBF2F301330193019B002BD8D0019BE1
:10714800013BF8E71700008000200140E8FFFF7FBF
:1071580028080020400D030038B504460068FFF7F2
:1071680039FD054620BB94F85430012B20D001236B
:1071780084F854302046FFF795FFB0B9A36D226814
:1071880023F4706323F0010343F48073A3651C2385
:10719800E065136084F85400936823F0004323F0FB
:1071A800170343F00403936038BD84F85450FBE799
:1071B8000220F9E7026838B5936891680446C80761
:1071C80001D4002038BD9907FBD4936803F0050368
:1071D800012B19D1936823F0004323F0170343F0E0
:1071E8000203936003231360FBF792FC05462368B0
:1071F8009B68DB07E5D5FBF78BFC401B0228F6D91B
:1072080023689B68DA07F2D5A36D43F01003A365E2
:10721800E36D43F00103E3650120D3E770B504464D
:1072280000284BD0836D43F002038365FFF70CFF02
:10723800054668B92046FFF7BDFF054608B9012392
:10724800A3652268936823F0104323F01703936023
:1072580023685A6822F4677222F003025A6040F2E7
:107268009F321A60D968164A0A40DA601A6922F011
:1072780040421A615A6922F007025A611A6A02F0FA
:10728800F0221A625A6A02F0F0225A62DA6A02F0AE
:10729800F022DA629A6A0B4A00269E62D2F8083710
:1072A80023F0FE73C2F808372046FAF7FFFDE665BB
:1072B8002666A66584F85460284670BD0125FBE75C
:1072C80000023E830020014010B590F85430012B95
:1072D800044615D0012380F85430FFF7B5FE58B99D
:1072E8002046FFF767FF38B9A36D23F4807323F0B6
:1072F800010343F00103A365002384F8543010BD53
:107308000220FCE7F7B50023019390F85430012BD5
:1073180004467FD0012380F85430FFF74BFF2368E1
:107328009A6812F00102054607D0A36D43F01003D6
:10733800A365002384F854302DE0A16D364F21F465
:10734800817141F00201A165DE68D96826F4FF4623
:1073580026F07C0621F40041360421F00301360CA6
:10736800D96008209968394041F0004199609968CE
:10737800002913DA0199013101910199B1F52E3FE4
:10738800F5D3A36D23F0120343F01003A365002384
:1073980084F854300125284603B0F0BDD3F8B41062
:1073A800013801F07F010A44DCD199681A4801408C
:1073B80041F001019960D3F8B41021F07F0141EA4E
:1073C800D202C3F8B4209A68024042F002029A60DE
:1073D800FBF79EFB074623689A68D20708D4DA6849
:1073E8003243DA60A36D23F0030343F001039FE700
:1073F800FBF78EFBC01B0228EDD923689B68D907D1
:10740800E9D5A36D43F01003A365E36D43F00103D1
:10741800E365BFE70225BEE7E8FFFF7F0749CA68C3
:1074280022F4E0620302120403F4E063120C134333
:1074380043F0BF6343F40033CB60704700ED00E0D6
:10744800164B30B5DC68C4F30224C4F10703251DCC
:10745800042B28BF0423062D4FF0FF358CBF033CB7
:10746800002405FA03F321EA0303A54022EA0502F2
:10747800A340002843EA0203ACBF00F16040084A79
:107488004FEA0313B8BF00F00F00DBB2AABF00F544
:107498006140135480F8003330BD00BF00ED00E0B8
:1074A80014ED00E0002807DB044A4109012300F03D
:1074B8001F00834042F82130704700BF00E100E020
:1074C80000280CDB4309064900F01F002033012285
:1074D800824041F82320BFF34F8FBFF36F8F70476F
:1074E80000E100E070B5D0E913456560446D14B162
:1074F800D0E916456560D0E9105404F01C06012453
:10750800B4406C60046863608368102B0BBFA26092
:10751800A160E160E26070BD0268416CD3B210B551
:10752800083B1424B3FBF4F30B4CA24288BF0B4A6C
:1075380021F0030199BF01F1804202F5023252188D
:1075480007338264064AC26403F01F03012202FA69
:1075580003F3036510BD00BF070402401C08024086
:107568008008024038B500285CD002682E4B9A4249
:107578004FF014014AD82D4B1344B3FBF1F32C49B7
:107588009B00C0E91013022380F8253013680569B1
:1075980023F4FF4323F070031360D0E9024323432D
:1075A8002B43456911682B4385692B43C5692B43D8
:1075B800056A2B430B431360FFF7AEFFB4F5804F0A
:1075C80004BF002343604368816C03F07F020A60B4
:1075D800D0E91314013B032B4C601ED8154B1649F8
:1075E800816513449B000121013A01FA02F200214E
:1075F8004365C2651960114B5A6400230122C363B5
:1076080080F8243080F82520184638BD0C4B1344E8
:10761800B3FBF1F30B499B00B3E70023C0E9153333
:10762800C365EAE70120F0E707040240F8FFFDBF61
:10763800000002403F820010400902400009024059
:10764800F8FBFDBF0004024038B5002841D00268AD
:10765800136823F0010313601F4B9A424FF0140183
:1076680030D81E4B1344B3FBF1F31D499B00C0E90E
:107678001013012403F01C0304FA03F3002515601A
:107688004B60FFF749FF836C41681D60D0E91332F6
:107698005A604A1E032A06D8124B0B449B0094409A
:1076A8001D60114B5C640023C363C0E91533C0E956
:1076B8000B33C0E90D33C36580F8253080F82430DA
:1076C800184638BD094B1344B3FBF1F308499B0036
:1076D800CDE70120F5E700BF07040240F8FFFDBF32
:1076E800000002403F82001000090240F8FBFDBF85
:1076F8000004024070B590F82450012D04463BD098
:1077080090F825600125AE4280F824504FF000061D
:107718002CD1022580F825500568C6632E6826F00E
:1077280001062E60FFF7DEFE036BBBB12B6843F04A
:107738000E032B60A36C1A68D20342BF1A6842F486
:1077480080721A60636D1BB11A6842F480721A6005
:107758002B6843F001032B60002070BD2B6823F0D9
:1077680004032B602B6843F00A03E2E78023C3631A
:1077780080F824602846F0E70220EEE770B4426CF7
:10778800046C036826681D6802F01C0204219140FD
:1077980031420FD015F0040F0CD01A6892065EBF64
:1077A8001A6822F004021A60036B6160002B33D060
:1077B80070BC184702219140314217D015F0020FD2
:1077C80014D01A68940606D41A6822F00A021A60BD
:1077D800012280F82520114A93428CBF104B114B8F
:1077E8005960002380F82430C36ADFE708219140FC
:1077F800314211D029070FD5196821F00E011960FF
:10780800012303FA02F26260C36380F82530002383
:1078180080F82430436BC9E770BC70478000024091
:1078280000040240000002400A4A536943F48023DE
:1078380030B55361EFF3108472B60023CD58C550AC
:107848000433B3F5807FF9D11369DB03FCD484F3E7
:10785800108830BD00400058064B5A69002ABFBF47
:10786800054A9A6002F188329A60BABF5869C00F17
:10787800002070470040005823016745044B5A69AF
:1078880042F000425A615869C043C00F704700BFB8
:107898000040005870B50546FBF73AF9124E044609
:1078A8003369D90313D43369DA0744BF012232613B
:1078B8004CF2FA32134011D10B4E306910F480208B
:1078C8000BD0FBF725F9001BA842F6D304E0FBF721
:1078D8001FF9001BA842E3D3032070BD024A1361BD
:1078E800024A01205360F8E700400058D80E0020F3
:1078F8002DE9F041184D98462B78012B06460C4689
:10790800174626D001232B704FF47A7000236B6042
:10791800FFF7C0FFA0B9012E16D1104A536943F0F2
:10792800010353612760BFF36F8FC4F804804FF4DD
:107938007A70FFF7AFFF094A536923EA06035361D8
:1079480000232B70BDE8F08139462046FFF76CFF15
:10795800EDE70220F6E700BFD80E002000400058EF
:10796800054A536923F47E7343EAC00040F480302B
:1079780040F0020050617047004000582DE9F04186
:10798800234F3B78012B054688463FD001233B70A7
:107998004FF47A7000237B60FFF77CFF044688B9B8
:1079A8002B68042B13D11B4A536943F4803343F0EB
:1079B800040353614FF47A70FFF76CFF0446154BCC
:1079C8001A681B6800233B702046BDE8F0814FF021
:1079D800FF33C8F800306E68D5E901321344B3426A
:1079E8000AD93046FFF7BCFF4FF47A70FFF752FF11
:1079F80050B1C8F800600446064A536923F47E7300
:107A080023F002035361DAE70136E5E70224DBE7F6
:107A1800D80E0020004000582DE9F04F524C0023AA
:107A28004FF00F090A6832FA03F501D1BDE8F08F6B
:107A3800012505FA03F818EA020200F08E804E6864
:107A4800032706F003054FEA430E07FA0EFC6F1EE4
:107A5800012F6FEA0C0C32D8876807EA0C0ACF6846
:107A680007FA0EF747EA0A078760476827EA08080F
:107A7800C6F300179F4047EA08074760C76807EA48
:107A88000C088F6807FA0EF747EA0807022DC76047
:107A980017D14FEAD30800EB880803F0070AD8F893
:107AA80020704FEA8A0A09FA0AFB27EA0B0B0F69CA
:107AB80007FA0AF747EA0B07C8F8207001E0032D18
:107AC800DCD1076805FA0EF507EA0C073D4316F402
:107AD800403F056041D023F0030707F1804707F5D1
:107AE800803703F0030CBD684FEA8C0C4FF0070E8B
:107AF8000EFA0CFEB0F1904F25EA0E0E2FD01B4D5A
:107B0800A8422ED005F58065A84214BF0725022596
:107B180005FA0CF545EA0E05BD602568D74316F44D
:107B2800801F0CBF3D4015432560656816F4001F93
:107B38000CBF3D4015436560D4F8805016F4803F73
:107B48000CBF3D401543C4F88050D4F88450B603A8
:107B580054BF3D401543C4F88450013362E7002503
:107B6800D6E70125D4E700BF000800580004004804
:107B7800374A2DE9F04F00234FF0010A4FF0070B69
:107B88004FF00F0931FA03F401D1BDE8F08F0AFA7A
:107B980003FC1CEA010654D023F0030404F18044DA
:107BA80004F5803403F00307A568BF000BFA07F853
:107BB800B0F1904F08EA050E45D0264DA84244D0B2
:107BC80005F58065A8420CBF02250725BD4075450F
:107BD80017D1D2F8805025EA0605C2F88050D2F8AD
:107BE800845025EA0605C2F88450156825EA06057A
:107BF8001560556825EA06055560A56825EA080553
:107C0800A560056803265C0006FA04F423FA06F664
:107C1800254300EB8606056003F00705376AAD00CB
:107C280009FA05F527EA05073762856825EA040594
:107C38008560456825EA0C054560C56825EA0404A1
:107C4800C46001339EE70025C0E70125BEE700BFF9
:107C580000080058000400480369194214BF0120B5
:107C6800002070470AB1816170478162704743699B
:107C780001EA030221EA030141EA024181617047F6
:107C8800044AD168014208B502D0D060FBF7DAFB9C
:107C980008BD00BF0008005803689A69910744BFEF
:107CA80000229A629A69D2075EBF9A6942F001027D
:107CB8009A61704730B5039D04682B4343EA024339
:107CC800064A6068C1F309010B4342EA555223F0A2
:107CD800004320EA02000343636030BDFF63FF03F3
:107CE80003682DE9F0419C6914F0100405460F461D
:107CF80016466FD010220024DA61A0462B689A69D4
:107D0800900661D4B8F1000F35D044F00404012086
:107D18002E68B369D90541BF4FF48072F26144F00F
:107D2800010401205A0541BF4FF4806244F0080461
:107D3800F26101209B054FD54FF4007344F0020413
:107D4800F3612846FFF7A8FF736823F0FF7323F455
:107D58008B3323F4FF7323F0010373606B6C2343AD
:107D68006B64202385F84130002385F8423085F87C
:107D78004030012032E07A1CC1D0FAF7C9FE801BDE
:107D8800B84201D8002FB9D12B68596895F842201C
:107D980098690004D2B20AD5490408D4202A06D02A
:107DA8005A6842F480425A60FAF7B2FE06462B68D7
:107DB8009B699B06A2D4FAF7ABFE801B1928F6D95B
:107DC80020244FF0010899E7B8F1000F9DD1202237
:107DD800DA619AE720469BE70028B2D1BDE8F08136
:107DE80070B504460D46164623689B699B0701D566
:107DF80000201BE0324629462046FFF771FFA0B954
:107E08006A1CF1D0FAF784FE801BA84201D8002D25
:107E1800EAD1636C43F020036364202384F8413083
:107E2800002384F8423084F84030012070BD70B5DA
:107E380004460D46164623689B699B0601D500201B
:107E480019E0324629462046FFF74AFF90B9FAF76B
:107E58005FFE801BA84201D8002DECD1636C43F073
:107E680020036364202384F84130002384F84230DF
:107E780084F84030012070BD70B504460D461646A2
:107E880023689B695B070ED4324629462046FFF7D4
:107E980027FF38BB23689A69910625D59A69520746
:107EA80003D5228D0AB1002070BD9A6912F0100224
:107EB8001CBF1022DA614FF0200118BF042262644F
:107EC800D9615A6822F0FF7222F48B3222F4FF72D1
:107ED80022F001025A60002384F8411084F84230ED
:107EE80084F840300120DFE7FAF712FE801BA84231
:107EF80001D8002DC4D1636C43F0200363642023B0
:107F080084F841300023EBE72DE9F041069F044651
:107F1800884616461D462268936938EA03030CBF53
:107F280001230023B34201D0002015E06B1CF3D0DD
:107F3800FAF7EEFDC01BA84201D8002DEBD1636C07
:107F480043F020036364202384F84130002384F83D
:107F5800423084F840300120BDE8F08110B5044675
:107F680000284AD090F8413003F0FF021BB980F88E
:107F78004020FAF7ADFA242384F8413023681A68C0
:107F880022F001021A60626822F070621A619A682F
:107F980022F400429A60D4E90221012924D142F452
:107FA80000429A605A6842F0007242F400425A60F5
:107FB800DA6822F40042DA60D4E904210A43A169AC
:107FC80042EA0122DA60D4E907210A431A601A68F2
:107FD80042F001021A6000202023606484F84130D6
:107FE800206384F8420010BD42F4044202299A60DA
:107FF80004BF4FF400625A60D4E70120F3E70000A1
:108008002DE9F347984690F841300A9F202B044603
:108018000E46914640F0868090F84030012B00F0E3
:1080280081804FF0010A80F840A0FAF771FD19230A
:108038000546009052464FF400412046FFF764FF82
:1080480018B1012002B0BDE8F087212384F841303F
:10805800102384F842306064A4F82A80638DC4F841
:1080680024909BB2FF2B60632F4B26D9FF222285D9
:1080780000934FF0807331462046FFF71BFE638D57
:108088009BB22A4639462046FBB9FFF7D0FE0028A6
:10809800D7D123682021D9615A6822F0FF7222F4CF
:1080A8008B3222F4FF7222F001025A6084F84110E8
:1080B80084F8400084F84200C4E7628D92B22285B9
:1080C80000934FF00073D2B2D5E7FFF789FE00287E
:1080D800B7D1636A226813F8011B91626362638DEA
:1080E800228D013B9BB26385638D013A92B29BB2AC
:1080F8002285002BC3D0002AC1D100953B468021A0
:108108002046FFF701FF00289BD1638D9BB2FF2B10
:1081180003D9FF2222850090ABE7628D92B22285B7
:108128000090CEE702208DE7002000802DE9F3477C
:10813800984690F841300A9F202B04460E469146F7
:1081480040F0878090F84030012B00F082804FF09B
:10815800010A80F840A0FAF7DBFC192305460090D5
:1081680052464FF400412046FFF7CEFE18B10120D9
:1081780002B0BDE8F087222384F84130102384F848
:1081880042306064A4F82A80638DC4F824909BB2BE
:10819800FF2B6063304B26D9FF22228500934FF0D6
:1081A800807331462046FFF785FD638D9BB22A46D2
:1081B80039462046FBB9FFF73AFE0028D7D1236895
:1081C8002021D9615A6822F0FF7222F48B3222F4FE
:1081D800FF7222F001025A6084F8411084F84000CE
:1081E80084F84200C4E7628D92B2228500934FF072
:1081F8000073D2B2D5E7FFF73FFE0028B7D1236856
:108208005A6A636A1A70636A228D01336362638DE6
:10821800013B9BB26385638D013A92B29BB2228582
:10822800002BC2D0002AC0D100953B4680212046B1
:10823800FFF76AFE00289AD1638D9BB2FF2B03D902
:10824800FF2222850090AAE7628D92B222850090D3
:10825800CDE702208CE700BF0024008010B590F81D
:108268004120202A0346D4B21CD190F84020012A8C
:1082780018D0242280F841200268106820F00100FC
:108288001060106820F4805010601068014311607D
:108298001168002041F00101116083F8414083F822
:1082A800400010BD0220FCE710B590F84120202ABC
:1082B8000346D4B21BD190F84020012A17D02422BB
:1082C80080F841200268106820F0010010601068F2
:1082D80020F4706040EA012111601168002041F02B
:1082E8000101116083F8414083F8400010BD02206D
:1082F800FCE70000024A136843F480731360704778
:10830800000400580D4B10B55B690C4628B99A0556
:1083180007D500F027F820B110BD9B0501D400F067
:1083280019F8074A1369012C23F00403136101D1DA
:1083380030BFF1E740BF20BF20BFEDE70004005881
:1083480000ED00E0024B186800F4C060704700BF01
:1083580000040058024A136843F4804313607047CE
:10836800000400580C4A136823F4804313600B4B35
:108378001B6832214B430A49B3FBF1F35169890564
:1083880000D533B9536913F4007F14BF03200020CC
:108398007047013BF2E700BF00040058280800209E
:1083A80040420F000B4A136823F0070343F002030F
:1083B8001360094B1A69012842F004021A6105D1B9
:1083C80030BF1A6922F004021A61704740BF20BF0B
:1083D80020BFF6E70004005800ED00E04FF0B0437E
:1083E8001868C0F3404070474FF0B0431868C0F3B6
:1083F800400070474FF0B042536823F47F4343EA8C
:108408000023536070474FF0B0431868C0F34060D2
:10841800704700007FB54FF0B0432C4AD3F80831BD
:10842800C0F3031003F00F0352F82040284A52F813
:108438002330B4FBF3F4FFF785FF264B054693E89A
:108448000700B5F5007F04AB03E9070010D0224B05
:108458009C4218D303F5B70303F67F539C4229D9EE
:1084680003F5741303F510639C4225D802230BE02F
:108478001A4B9C4207D91A4B9C421BD903F5370368
:1084880003F5D853F0E7002304AA02EB830353F85B
:108498000C4C144D2B6823F0070323432B60FAF789
:1084A80037FB06462B6803F007039C4206D10020E1
:1084B80004B070BD0123E7E70024EAE7FAF728FBD8
:1084C800801B0228EED90320F2E700BF583B0108C1
:1084D800B83B0108003A0108C0CF6A00BFEA210191
:1084E8003F933402004000584FF0B04310B59A68EB
:1084F800D96812F00C0205D00C2A4AD101F0030306
:10850800012B51D14FF0B0412B480B6813F00803F1
:1085180006D00B6813F0080337D1D1F8941007E0A0
:108528000C68240756BFD1F894300968C3F30323B5
:1085380050F82330002A0CBF184600204FF0B041F5
:108548008A6802F00C020C2A1ED1CA6802F00302E3
:10855800022A2ED0032A06D10B68184A13F4801F6A
:10856800174B18BF13464FF0B042D068D168D26895
:10857800C0F306205843C1F302130133B0FBF3F0F4
:10858800530F0133B0FBF3F010BD0B68C3F30313B3
:10859800CEE7042A05D0082A06D11B6813F48013F5
:1085A80005D006480023C9E700231846C6E7044853
:1085B800C4E7024BD7E700BF583B01080024F4008A
:1085C8000048E80108B5FFF78FFF4FF0B043044AB1
:1085D8009B68C3F3031352F82330B0FBF3F008BDD4
:1085E800B83B01082DE9F0410446002853D04FF06C
:1085F800B0439D68DE6803689B0605F00C0506F02D
:10860800030668D5026A1DB10C2D46D1012E44D14E
:10861800002A40D04FF0B043A16A1A68170756BF26
:10862800D3F894301B681B0903F0F00399421FD953
:108638000846FFF7EFFE00282DD14FF0B04213682F
:1086480043F0080313601368A16A23F0F0030B4397
:108658001360606AFFF7CEFEFFF7B4FFAB4B1860FC
:10866800AB4B1868FAF752FA002834D0BDE8F0810D
:108678004FF0B042136843F008031360136823F007
:10868800F0030B431360606AFFF7B4FE0846FFF778
:10869800C1FE0028E0D00120E8E74FF0B043002AEF
:1086A80054D01A6842F001021A60FAF731FA074604
:1086B800FFF79AFE002842D04FF0B042136843F00B
:1086C800080313601368A16A23F0F0030B431360D7
:1086D800606AFFF78FFE2368D80748D42368990794
:1086E80000F18C8023681E0740F1FA80A3694FF0DF
:1086F800B046002B00F0E180D6F89430E16903F031
:108708001002914200F0C48003F00302022AC2D092
:10871800D80740F1B380D6F8943023F00103C6F8A7
:108728009430FAF7F5F90746D6F89430990740F1EE
:10873800A580FAF7EDF9C31B112BF5D904E0FAF778
:10874800E7F9C01B0228B3D903208FE71A6822F083
:1087580001021A60FAF7DCF90746FFF745FE002820
:10876800B9D0FAF7D5F9C01B0228F6D9ECE7082DDD
:1087780003D00C2D05D1032E03D16368002BADD196
:1087880089E74FF0B043A1681A6822F480120A43BF
:108798001A606268B2F5803F10D11A6842F48032DC
:1087A8001A60FAF7B5F90746FFF718FE002895D1C1
:1087B800FAF7AEF9C01B6428F6D9C5E7B2F5041F6D
:1087C80004D11A6842F400121A60E6E7196821F425
:1087D80080311960196821F400111960002AE0D16C
:1087E800FAF796F90746FFF7F9FD00283FF476AF48
:1087F800FAF78EF9C01B6428F5D9A5E7042D23697B
:1088080003D00C2D0ED1022E0CD1002B3FF443AF18
:108818004FF0B0426169536823F0FE4343EA0163B5
:1088280053605FE74FF0B046BBB1336843F48073E1
:108838003360FAF76DF9074633685A0505D4FAF735
:1088480067F9C31B022BF7D97EE77368626923F0C7
:10885800FE4343EA0263736044E7336823F480739A
:108868003360FAF755F9074633685B057FF53AAF89
:10887800FAF74EF9C31B022BF6D965E74FF0B04261
:10888800E169D2F8943023F010030B43C2F8943016
:108898004FF0B047D7F8943043F00103C7F894304D
:1088A800FAF736F90646D7F894309A0718D4FAF743
:1088B8002FF9831B112BF6D946E7D6F8943023F00D
:1088C8000103C6F89430FAF723F90746D6F894302E
:1088D8009B0705D5FAF71CF9C31B112BF6D933E70B
:1088E8002368580754D50B4F3B68D90514D4FFF7B4
:1088F80001FDFAF70DF906463B68DA050CD4FAF7DC
:1089080007F9831B022BF7D91EE700BF28080020B0
:108918002C08002000040058E3684FF0B046002BF4
:1089280058D023F08003052B02BFD6F8903043F0CF
:108938000403C6F890304FF0B046FAF7E9F8D6F8D5
:10894800903043F001030746C6F8903041F288386A
:10895800D6F890309B0705D4FAF7DAF8C31B4345DD
:10896800F6D9F1E6E36823F00403812B1BD1FAF76B
:10897800CFF8D6F8903043F08003C6F89030074619
:108988004FF0B04641F28838D6F89030180504D533
:10899800E36A002B4AD1002068E6FAF7B9F8C01B51
:1089A8004045F1D9D0E6FAF7B3F8D6F8903023F07D
:1089B8008003C6F8903007464FF0B04641F2883839
:1089C800D6F890301905E3D5FAF7A2F8C01B404550
:1089D800F6D9B9E6FAF79CF8D6F8903023F0800378
:1089E8000746C6F8903041F28838D6F890301A0514
:1089F80016D4FAF78DF8D6F8903023F00103C6F8AC
:108A0800903007464FF0B04841F28836D8F8903099
:108A18009B07BDD5FAF77CF8C31BB342F6D993E69A
:108A2800FAF776F8C01B4045DFD98DE60C2D4ED0FD
:108A3800022B4FF0B0431A6822F080721A6033D1CB
:108A4800FAF766F80546FFF7DEFC38BBD4E90C31C7
:108A58004FF0B0420B43D0682D4901400B43E16B06
:108A68000B43216C0B43616C0B43A16B43EA01235D
:108A7800D360136843F080731360D36843F0805366
:108A8800D360FAF745F80446FFF7BDFC002882D109
:108A9800FAF73EF8001B0A28F6D955E6FAF738F82F
:108AA800401B0A28CFD94FE6FAF732F80446FFF7F9
:108AB800AAFC30B94FF0B042164BD1680B40D360D6
:108AC80069E7FAF725F8001B0A28F0D93CE6012BDC
:108AD8003FF4E1AD4FF0B043D868236B00F00302D8
:108AE8009A427FF4D8AD626B00F0700393427FF432
:108AF800D2ADA26B00F4FE43B3EB022F7FF4CBADF3
:108B0800636C00F06040C01A18BF0120AEE500BFDA
:108B18008C80C111FCFFFEEE2DE9F0410D460446A4
:108B280010B90120BDE8F081684E336803F00703EF
:108B38008B4216D323689A0727D54FF0B047A2680F
:108B4800BB6823F0F0031343BB60F9F7E1FF064667
:108B5800BB68DB0319D4F9F7DBFF831B022BF7D9BA
:108B680011E0336823F007030B433360F9F7D0FFB4
:108B78000746336803F00703AB42DBD0F9F7C8FFB9
:108B8800C01B0228F5D90320CCE72368580617D55F
:108B98004FF0B0476269D7F8083123F00F0343EA72
:108BA8001213C7F80831F9F7B3FF0646D7F80831AA
:108BB800D90305D4F9F7ACFF831B022BF6D9E2E7FA
:108BC80023685A0713D54FF0B047E268BB6823F40F
:108BD800E0631343BB60F9F79BFF0646BB689B0342
:108BE80005D4F9F795FF831B022BF7D9CBE7236848
:108BF800180714D54FF0B0472269BB6823F46053B7
:108C080043EAC203BB60F9F783FF0646BB68590312
:108C180005D4F9F77DFF831B022BF7D9B3E7236847
:108C2800DA070FD4294C236803F00703AB4239D87D
:108C3800FFF7C8FC264B1860264BBDE8F0411868C2
:108C4800F9F764BF6268022A1DD1FFF7C7FB002845
:108C58003FF467AF4FF0B04641F28838B36823F06D
:108C680003031343B360F9F753FF0746B368626819
:108C780003F00C03B3EB820FD4D0F9F749FFC01B04
:108C88004045F3D97FE7032A02D1FFF7BCFBDEE7B3
:108C980012B9FFF7A9FBDAE74FF0B0431B685B0591
:108CA800D8D43EE7236823F007032B432360F9F762
:108CB8002FFF0646236803F00703AB42B8D0F9F745
:108CC80027FF801B0228F5D95DE700BF0040005848
:108CD800280800202C08002008B5FFF773FC4FF087
:108CE800B043044A9B68C3F3022352F82330D840A8
:108CF80008BD00BF983B010808B5FFF763FC4FF0BB
:108D0800B043044A9B68C3F3C22352F82330D840C7
:108D180008BD00BF983B01084FF0B043D3F890005E
:108D2800C0F3400070474FF0B0410209D1F88830D5
:108D380002F47F22000123EA020300F47F200343A8
:108D4800C1F8883070474FF0B041020CD1F8883034
:108D5800120423EA020343EA0040C1F8880070477E
:108D68000368DA0370B5044639D5FFF7C3FAF9F793
:108D7800CFFE614E05463368DB0532D54FF0B04370
:108D8800616BD3F8902002F4407291421DD0D3F861
:108D98009010D3F8902042F48032C3F89020D3F892
:108DA800902021F4407022F480328D07C3F890207F
:108DB800C3F8900009D5F9F7ABFE41F288360546AD
:108DC800FFF7AAFF012840F090804FF0B042616B96
:108DD800D2F8903023F440730B43C2F89030002649
:108DE80005E0F9F795FE401B0228C4D9032625683B
:108DF800E8070AD54FF0B0416268D1F8883023EA15
:108E0800124392B21343C1F88830A9070AD54FF02C
:108E1800B041A268D1F8883023EA124392B21343D2
:108E2800C1F88830AA0609D54FF0B0422169D2F8B6
:108E3800883023F440630B43C2F88830AB0502D571
:108E4800206AFFF780FF680502D5606AFFF77BFF9D
:108E5800290502D5A06AFFF776FF6A0602D5606980
:108E6800FFF761FF2B0602D5A069FFF75CFFE80555
:108E780002D5E069FFF757FFE90610D54FF0B04279
:108E8800E168D2F8883023F440730B43C2F8883085
:108E9800B1F5807F02BFD36843F08073D3602A04A2
:108EA8000ED54FF0B042216BD2F8883023F0404302
:108EB8000B43C2F8883019B9D36843F08073D36084
:108EC8006B0410D54FF0B042E16AD2F8883023F035
:108ED80040530B43B1F1005FC2F8883003D1D36827
:108EE80043F48033D360304670BDF9F711FE401B60
:108EF800B0427FF665AF79E70004005830B590F8C6
:108F08002C30012B02464FF0020022D0174B82F87A
:108F18002D00CA24012582F82C505C6253245C621F
:108F2800B1F5807F146B996914D121F48851996146
:108F3800596C24F0010421F0004159641463DD6583
:108F48000A4BFF2159620020012382F82D3082F854
:108F58002C0030BD21F408519961D96C24F0020429
:108F680021F00041D9641463D865E9E7002800407E
:108F780070B50B4E036B756D1D40EA07044603D5AB
:108F88000123F365F9F7D7FEAB0704D50223F36590
:108F9800204600F0C9F9012384F82D3070BD00BFC8
:108FA8000028004038B50A4CE36823F02003E3604A
:108FB800F9F7AEFD0546E3689B0601D5002038BDEC
:108FC800F9F7A6FD401BB0F57A7FF4D90320F6E740
:108FD80000280040F8B5114DEC6814F0400406462E
:108FE8001AD1EB6843F08003EB60F9F791FD234653
:108FF8000746EC6814F0400401D1032B01D1184650
:10900800F8BDF9F785FDC01BB0F57A7F234684BF0C
:10901800032386F82D30ECE70023F0E70028004012
:1090280038B50F4CE36823F08003E360A3699B061F
:10903800054606D4FFF7B6FF10B1032085F82D00CA
:1090480038BDA36923F02003A361FFF7ABFF10B17C
:10905800032085F82D00A36943F02003A361EFE7FF
:109068000028004038B5044600284BD090F82D3031
:1090780003F0FF021BB980F82C20F9F757FB0223F5
:10908800214D84F82D30EB68DB0636D4CA236B6299
:1090980053236B622046FFF79DFF10B1FF236B62DD
:1090A80038BDAB6923F08E6323F04003AB612169BF
:1090B8006368AA690B431343A2691343AB61D4E9FC
:1090C800022343EA02432B61D4E90931EA680B43DE
:1090D80022F4F8521343EB602046FFF7A1FF002863
:1090E800DCD1D4E90713AA690B4322F06042134389
:1090F80062691343AB61FF236B62012384F82D304F
:109108000020CDE70120CBE70028004000230928F4
:1091180003D840EA0310C0B270470A380133C0B21E
:10912800F5E700002DE9F04790F82C30012B0546B3
:109138004FF0020069D0012385F82C304E4B85F89A
:109148002D00DE6806F44076B6F5807F78D04C694D
:10915800087891F8019091F802A091F82470002AFB
:1091680055D19B6913F0400308BFCB70FFF7CEFFC2
:1091780080464846FFF7CAFF02465046FFF7C6FF3B
:1091880081463846FFF7C2FF0B6ACF78234343EA8C
:10919800875343EA090343EA084343EA022343EABD
:1091A8000063354ACA205062532050628C6A88692D
:1091B800B4F5807F946945D124F4885494610124DE
:1091C800D465B6F5807F09BFCB6913640343536444
:1091D80018BF5064284B4A681A672A6B42F001028C
:1091E8002A639A6942F488529A61244AD2F88030F4
:1091F80043F40033C2F880301F4BFF225A6200202C
:10920800012385F82D3085F82C00BDE8F087B4F1EE
:10921800803F07D0B4F5000F04D09B6913F04003DA
:1092280008BFCB700B6ACA781C4344EA0A0444EAB4
:10923800004343EA092343EA825343EA0763B0E75A
:109248000023AEE724F4085494610224D465B6F5EB
:10925800807F09BFCB6993640343D36418BFD0648C
:10926800054B4A685A672A6B42F002022A639A69D8
:1092780042F40852B8E700BF002800400008005830
:1092880090F82C20012A03464FF0020012D00A4A17
:1092980083F82D00CA21516253215162916941F02E
:1092A80020019161FF2151620020012283F82D20C5
:1092B80083F82C00704700BF0028004090F82C204D
:1092C800012A03464FF0020019D00D4A83F82D00F9
:1092D800CA2151625321516291690A4841F08001C3
:1092E8009161D0F8801041F48021C0F88010FF21EE
:1092F80051620020012283F82D2083F82C0070474A
:109308000028004000080058064B5A6D520610B558
:10931800044603D54022DA65F9F710FD012384F8E5
:109328002D3010BD002800407047890001F18041B0
:1093380001F531410A607047890001F1804101F56A
:109348003141086870470000034AD2F8903043F46E
:109358000043C2F89030704700040058034AD2F81E
:10936800903023F40043C2F890307047000400584E
:10937800074B1A6822F040021A6040F441704FF41B
:10938800B85218605A601A6842F040021A60704772
:109398000000015837B5054600284ED0837903F000
:1093A800FF046BB1032C0BD0254B4FF400629A617C
:1093B8002868FFF7DDFF002401232B71AC602FE044
:1093C80000236B712846F9F7BDFA1E4AD2F890308F
:1093D80043F48053C2F89030002CE5D102234FF0BB
:1093E800B042AB71D2F8943023F40043C2F8943001
:1093F800154B1B681C214B43DB0C64214B43019329
:10940800019B93B90124AC60FFF79EFF0C4B9A684F
:1094180042F400629A604FF400629A61002CC7D04F
:109428000123AB71204603B030BD019B013B019382
:10943800D2F894305B04E3D4E6E70124F2E700BFF6
:1094480000040058000800582808002037B5174DB8
:109458002B6802461C204343DB0C6420434314481A
:109468000193019B93B901209060114C21732B68E3
:109478001C214B43DB0C64214B430193019B6BB9CB
:10948800012090600A4BDB6803B030BD019B013BB3
:10949800019383689C07E4D50020E6E7019B013B24
:1094A8000193A368DB07E9D5ECE700BF2808002093
:1094B8000000015837B5184D2B6802461C2043435D
:1094C800DB0C6420434315480193019BA3B9012099
:1094D8009060124CFF2323732B681C256B43DB0C15
:1094E80064256B430193019B73B9012090600B4B7A
:1094F800DB680B7003B030BD019B013B01938368AF
:109508009C07E2D50020E4E7019B013B0193A36897
:10951800DB07E8D5EBE700BF28080020000001586A
:109528000E4B0F491B681822534382B01B0D64224F
:10953800534301934B69019AC3F3800322B9022371
:109548008360012002B07047019A013A01924A698A
:10955800920701D5002BEDD10020F3E72808002061
:109568000004005807B50379012B0FD10A4B1B687B
:10957800182253431B0C0193FFF7F0FE019B013B9C
:109588000193019B002BF9D1FFF7DEFE03B05DF8D4
:1095980004EBFFF7C5BF00BF28080020F8B51E463A
:1095A8008379012B154604460F46DAB22DD143794B
:1095B800012B2AD0022342718371FFF7D3FF0D21BB
:1095C8002046FFF7CBFEFFF741FF390A2046FFF799
:1095D8003DFFF9B22046FFF739FF2E44B5420ED1C0
:1095E8002046FFF7B1FEFFF79BFFA0680123003874
:1095F800A3714FF0000318BF01206371F8BD15F87F
:10960800011B2046FFF722FFE8E70220F6E7F8B53E
:109618001E468379012B154604460F46DAB22FD130
:109628004379012B2CD04271FFF79CFF1D21204666
:10963800FFF794FEFFF70AFF390A2046FFF706FFF7
:10964800F9B22046FFF702FF00212046FFF7FEFE91
:109658002E44B5420ED12046FFF776FEFFF760FF95
:10966800A06801230038A3714FF0000318BF012040
:109678006371F8BD29462046FFF71CFF0135E8E76E
:109688000220F6E7F8B51F468379012B15460446F4
:109698000E46DAB22CD14379012B29D04271FFF75B
:1096A80061FF06F0EF03A3F1840253425341237193
:1096B80031462046FFF752FEFFF7C8FE2F44AF425F
:1096C80010D1FFF741FE842E02D02046FFF728FF75
:1096D800A06801230038A3714FF0000318BF0120D0
:1096E8006371F8BD15F8011B2046FFF7AFFEE6E7EA
:1096F8000220F6E7F8B51E468379012B1546044685
:109708000F46DAB227D14379012B24D04271FFF7F3
:1097180029FF39462046FFF721FEFFF797FE002173
:109728002046FFF793FE2E44B5420ED12046FFF7A0
:109738000BFEFFF7F5FEA06801230038A3714FF078
:10974800000318BF01206371F8BD29462046FFF7C2
:10975800B1FE0135E8E70220F6E737B50023ADF89A
:10976800043001AA022312210546FFF7C3FFBDF802
:109778000440022364BA01AAA4B219462846FFF796
:1097880081FFE20702D5284609F0B4F9A30702D5FC
:10979800284609F0B5F9600702D5284609F0DAF934
:1097A800210702D5284609F0DBF9E20602D528464A
:1097B80009F0DCF9A30602D5284609F0C5F96006C8
:1097C80002D5284609F0A2F9210606D514F48071BD
:1097D80018BF0121284609F09FF9A20502D528469D
:1097E80009F0AAF9630402D5284609F0C5F903B0BF
:1097F80030BDF8B51E468379012B154604460F4641
:10980800DAB227D14379012B24D04271FFF7AAFE9F
:109818000E212046FFF7A2FDFFF718FE3946204625
:10982800FFF714FE2E44B5420ED12046FFF78CFDFB
:10983800FFF776FEA06801230038A3714FF00003FC
:1098480018BF01206371F8BD15F8011B2046FFF70A
:10985800FDFDE8E70220F6E7F8B51E468379012BFF
:10986800154604460F46DAB22BD14379012B28D08E
:109878004271FFF777FE1E212046FFF76FFDFFF7C5
:10988800E5FD39462046FFF7E1FD00212046FFF7B8
:10989800DDFD2E44B5420ED12046FFF755FDFFF7FA
:1098A8003FFEA06801230038A3714FF0000318BFE2
:1098B80001206371F8BD29462046FFF7FBFD0135FD
:1098C800E8E70220F6E7026852E8003F23F0C00309
:1098D80042E8003102680029F5D102F1080353E893
:1098E800003F23F4000302F1080C4CE80031002982
:1098F800F3D12023C0F888307047000010B5026803
:1099080052E8003F23F4907342E8003102680029CE
:10991800F5D10F4C02F1080353E8003F234002F150
:10992800080C4CE800310029F4D1C36E012B07D193
:1099380052E8003F23F0100342E800310029F7D134
:109948002023C0F88C300023C366436710BD00BFD6
:10995800FEFFFFEF38B50546C8B12423C0F88830AC
:1099680003681A68002422F001021A601C605C6017
:109978009C60F9F78FFAC5F8904085F88440C5F8DF
:1099880088402046C5F88C40EC662C6738BD01201D
:10999800FCE70000F8B504461346D4F88850202D9B
:1099A80032D1F1B1EAB1E06FA4F85620A4F85420FE
:1099B80000262122C4F890602165C4F88820226816
:1099C80088B1124FC762124F0763124F2832C0E99D
:1099D8000D76FDF78FFE30B11023C4F89030C4F82F
:1099E80088500120F8BD236840221A62226802F1DB
:1099F800080353E8003F43F0800302F1080141E8FF
:109A080000300028F3D1EDE70220EBE7219A0008A7
:109A1800699A0008759A000808B50346806A1B68A9
:109A28001B6813F0200317D1A0F85630026802F122
:109A3800080353E8003F23F08003083242E800316E
:109A480002680029F2D152E8003F43F0400342E89F
:109A580000310029F7D108BDF9F796FAFBE77047FE
:109A680008B5806AFFF7FBFF08BD7047806A38B504
:109A78000468D0F88830D0F88C50A268120606D551
:109A8800212B04D10023A0F85630FFF71CFFA36850
:109A98005B0606D5222D04D10023A0F85E30FFF71F
:109AA8002DFFD0F8903043F01003C0F89030FFF746
:109AB800DCFF38BD70470000D0F88C20B0F860108B
:109AC800222A08B5036855D15B6A826D0B40137072
:109AD800836D01338365B0F85E30013B9BB2A0F81B
:109AE8005E30B0F85E309BB2002B42D1026852E87B
:109AF800003F23F4907342E8003103680029F5D150
:109B080003F1080252E8002F22F0010203F1080CC9
:109B18004CE800210029F3D12022C0F88C20184AF3
:109B280041679342016705D1C26E012A0ED0F9F749
:109B380039FA1EE05A681102F6D553E8002F22F0D0
:109B4800806243E800210029F7D1EDE70022C266D0
:109B580053E8002F22F0100243E800210029F7D132
:109B6800DA69B0F85C10D20644BF10221A62FFF717
:109B7800A1FF08BD9A6942F008029A61F9E700BF9F
:109B880000800040D0F88C20B0F86010222A08B578
:109B9800036852D15A6A1140826D22F8021B82650D
:109BA800B0F85E20013A92B2A0F85E20B0F85E20CC
:109BB80092B2002A40D153E8002F22F4907243E871
:109BC80000210029F7D103F1080252E8002F22F002
:109BD800010203F1080C4CE800210029F3D12022EE
:109BE800C0F88C20174A41679342016705D1C26EBD
:109BF800012A0ED0F9F7D6F91EE05A681102F6D5F7
:109C080053E8002F22F0806243E800210029F7D1B1
:109C1800EDE70022C26653E8002F22F0100243E865
:109C280000210029F7D1DA69B0F85C10D20644BFE8
:109C380010221A62FFF73EFF08BD9A6942F0080237
:109C48009A61F9E7008000402DE9F84F0368B0F801
:109C58006060D3F81CB01F689D68D0F88C20222A59
:109C6800044640F0B980B0F8683043B1DFF8749129
:109C7800DFF874A14FF000081BF0200F20D1B4F8D2
:109C88005E309BB2D3B1B4F868209A4216D92268E4
:109C980002F1080353E8003F23F08053083242E8FA
:109CA800003122680029F2D1504B636752E8003F27
:109CB80043F0200342E800310029F7D1BDE8F88FCE
:109CC8002368A26D5B6A33401370A36D0133A365EB
:109CD800B4F85E30013B9BB2A4F85E302368D3F839
:109CE8001CB01BF0070F2ED01BF0010F09D0F9058F
:109CF80007D501221A62D4F8902042F00102C4F874
:109D080090201BF0020F09D0EA0707D502221A6239
:109D1800D4F8902042F00402C4F890201BF0040FFD
:109D280009D0E80707D504221A62D4F8903043F026
:109D38000203C4F89030D4F8903023B12046FFF7DE
:109D480094FEC4F89080B4F85E309BB2002B93D197
:109D5800226852E8003F23F4807342E80031236808
:109D68000029F5D103F1080252E8002F02EA09029E
:109D780003F1080040E800210029F3D120225345CF
:109D8800C4F88C20616721670AD05A68110207D588
:109D980053E8002F22F0806243E800210029F7D120
:109DA800E26E012A14D10022E26653E8002F22F065
:109DB800100243E800210029F7D1DA69B4F85C10F1
:109DC800D20644BF10221A622046FFF773FE53E7FB
:109DD8002046F9F7E7F84FE79A6942F008029A61D6
:109DE8006CE700BFFEFFFFEF00800040C19A00084B
:109DF8002DE9F84F0368B0F86060D3F81CB01F680D
:109E08009D68D0F88C20222A044640F0B780B0F82C
:109E1800683043B1DFF87091DFF870A14FF00008A7
:109E28001BF0200F20D1B4F85E309BB2D3B1B4F848
:109E380068209A4216D9226802F1080353E8003FC5
:109E480023F08053083242E8003122680029F2D119
:109E58004F4B636752E8003F43F0200342E800316C
:109E68000029F7D1BDE8F88F2368A26D596A3140FF
:109E780022F8021BA265B4F85E20013A92B2A4F857
:109E88005E20D3F81CB01BF0070F2ED01BF0010F7B
:109E980009D0F90507D501221A62D4F8902042F0BA
:109EA8000102C4F890201BF0020F09D0EA0707D579
:109EB80002221A62D4F8902042F00402C4F89020DA
:109EC8001BF0040F09D0E80707D504221A62D4F85A
:109ED800903043F00203C4F89030D4F8903023B1A6
:109EE8002046FFF7C2FDC4F89080B4F85E309BB2FC
:109EF800002B95D1226852E8003F23F4807342E892
:109F0800003123680029F5D103F1080252E8002F37
:109F180002EA090203F1080040E800210029F3D110
:109F280020225345C4F88C20616721670AD05A68FB
:109F3800110207D553E8002F22F0806243E8002180
:109F48000029F7D1E26E012A14D10022E26653E813
:109F5800002F22F0100243E800210029F7D1DA6926
:109F6800B4F85C10D20644BF10221A622046FFF7EC
:109F7800A1FD55E72046F9F715F851E79A6942F02F
:109F880008029A616EE700BFFEFFFFEF0080004005
:109F98008D9B000838B5044603682169A2681D68CE
:109FA800C0690A4361690A437749024329400A4361
:109FB8001A605A68E16822F440520A435A60734AA8
:109FC800A16993421CBF226A11439A6822F06E422B
:109FD80022F430620A439A60DA6A616A22F00F0258
:109FE8000A43DA626A4A934219D14FF0B043694A88
:109FF800D3F8883003F0030343F44033934200F06E
:10A00800B480B3F1031F24D0013A934240F0B580E5
:10A01800B0F5004F40F08F80FEF766FA6EE05E4ABA
:10A0280093421CD14FF0B0435C49D3F8883003F019
:10A038000C0343F440228A4200F0978006D8002B94
:10A048007CD0574B9A42E3D0012026E0B2F10C1F96
:10A05800FAD1B0F5004F53D04FF4004075E04B4AA9
:10A068009342F1D14FF0B043D3F8883003F4406302
:10A07800B3F5006F18D006D85BB1B3F5806FE3D1A4
:10A08800FEF732FA07E0B3F5406FDDD14FF4004038
:10A098000BE0FEF721FE40B900204FF00113A36644
:10A0A8000023C4E91D3338BD3E4865683E4B626AEB
:10A0B80005EB450133F81220B0FBF2F39942C3D8FF
:10A0C800B3EB053FC0D800231946F7F71DFD090279
:10A0D80041EA10616B080002C0182A464FF00003DD
:10A0E80041F10001F7F710FD304BA0F540729A429C
:10A0F800AAD82368D860CFE7FEF7EEFD0028CBD0BA
:10A108006168294B626A33F81220B0FBF2F24B08FF
:10A1180003EB42034FF6EF72B3FBF1F3A3F1100127
:10A12800914291D823F00F02216892B2C3F34203FF
:10A138001343CB60B0E7FEF7D7F904E0B0F5004F62
:10A14800DAD0FEF7C9FD0028A6D06368616A164A0E
:10A1580032F81120B0FBF2F000EB5300B0FBF3F043
:10A168004FF6EF73A0F11002C1E7B0F5004F0D48AC
:10A17800EBD1C5E7FEF7C0FDC0E7B0F5004FF9D059
:10A18800FEF7BAFDDFE700BFF369FFCF00800040AC
:10A1980000380140020003000044004008000C00A1
:10A1A80004000C000024F400F83B0108FFFC0F0039
:10A1B800836ADA0710B506D50168C46A4A6822F4CA
:10A1C800003222434A609C0706D50168046B4A683E
:10A1D80022F4803222434A60590706D50168446B4D
:10A1E8004A6822F4802222434A601A0706D5016889
:10A1F800846B4A6822F4004222434A60DC0606D592
:10A208000168C46B8A6822F4805222438A609906E6
:10A2180006D50168046C8A6822F4005222438A60D9
:10A228005A060FD50168446C4A6822F4801222430A
:10A23800B4F5801F4A6005D14A68846C22F4C002D4
:10A2480022434A601B0606D50268C16C536823F492
:10A2580000230B43536010BD2DE9F843DDF820902F
:10A2680005460F46164698462A68D36937EA030317
:10A278000CBF01230023B34201D0002029E0B9F12B
:10A28800FF3FF2D0F8F744FCA0EB080048452C68E3
:10A2980002D8B9F1000F1ED154E8003F23F4D0735F
:10A2A80044E80032002AF7D104F1080353E8003FDC
:10A2B80023F0010304F1080141E80032002AF3D138
:10A2C8002023C5F88830C5F88C30002385F8843001
:10A2D8000320BDE8F88323685A07C5D5E3691B0541
:10A2E800C2D54FF40063236254E8003F23F4D073CF
:10A2F80044E80032002AF7D104F1080353E8003F8C
:10A3080023F0010304F1080141E80032002AF3D1E7
:10A318002023C5F88830C5F88C30C5F89030D4E7CC
:10A3280073B504460026C0F89060F8F7F1FB23687F
:10A338001B681A07054619D423681B685B070AD5EA
:10A348006FF07E43009300222B464FF48001204695
:10A35800FFF782FFB0B900202023C4F8883084F8C2
:10A368008400C4F88C30E06620670CE06FF07E4310
:10A378000093324603464FF400112046FFF76CFF66
:10A388000028D9D0032002B070BD10B5044650B3E0
:10A39800D0F888301BB980F88430F8F70BFD2268B4
:10A3A8002423C4F88830136823F00103136020467F
:10A3B800FFF7F0FD012816D0A36A13B12046FFF776
:10A3C800F7FE23685A6822F490425A609A6822F08D
:10A3D8002A029A601A6842F0010220461A60BDE813
:10A3E8001040FFF79DBF012010BD000030B581650A
:10A3F8008168A0F85C200023B1F5805FA0F85E209A
:10A40800436735D10369002B40F2FF1318BFFF23C0
:10A41800A0F860300023C0F890302223C0F88C30B8
:10A42800016801F1080353E8003F43F001030831D4
:10A4380041E800340368002CF2D1456E8468016954
:10A44800B5F1005F32D1B0F8685095422ED8B4F516
:10A45800805F244A03D1244C002908BF2246426762
:10A46800B1B153E8002F42F4807243E80021F7E7C6
:10A4780029B90369002B14BF7F23FF23C8E7B1F173
:10A48800805FC5D10369002B14BF3F237F23BFE73B
:10A4980003F1080252E8002F42F0805203F108004D
:10A4A80040E800210029F3D1002030BDB4F5805FD9
:10A4B8000E4A03D10E4C002908BF2246426741B11B
:10A4C80053E8002F42F4907243E800210029F7D1A5
:10A4D800EAE753E8002F42F0200243E80021002970
:10A4E800F7D1E1E7519C0008F99D0008C19A0008DE
:10A4F8008D9B0008D0F88C30202B30B415D1B9B121
:10A50800B2B100230468C3660A4B9C420AD0636850
:10A518001B0207D554E8003F43F0806344E8003548
:10A52800002DF7D130BCFFF761BF022030BC704767
:10A538000120FBE700800040436E30B52BB90123B2
:10A54800A0F86A30A0F8683030BD0368094D9A68F1
:10A558009968094C490FC2F342626B5C615CDB008D
:10A56800B3FBF1F3A0F86A30AB5CA25CDB00B3FB91
:10A57800F2F3E7E7183C0108103C01081FB504ABEB
:10A5880003E9060090F88430012B04463AD00123F1
:10A5980080F884302423C0F8883003681A6822F0D1
:10A5A80001021A609A6822F440120A439A6071B94B
:10A5B8005A68BDF80C009DF80E1022F010020243F4
:10A5C8005A605A6822F07F4242EA01625A601A6869
:10A5D80042F001021A60F8F79BFA6FF07E420346D8
:10A5E80000924FF4800100222046FFF735FE38B96B
:10A5F8002023C4F88830002384F8843004B010BDC8
:10A608000320F8E70220F9E790F88430012B0FD0F7
:10A61800012380F88430016851E8002F42F00202DB
:10A6280041E80023002BF6D180F8843018467047A3
:10A638000220704710B590F88430012B044617D0DB
:10A648002423C0F8883003681A68196821F00101CA
:10A65800196042F000524FF0005141661A60FFF74E
:10A668006BFF2023C0F88830002084F8840010BDD8
:10A678000220FCE770B590F88430012B044617D00F
:10A6880005682423C0F888302E682B6823F001035E
:10A698002B60AB6823F060431943A960FFF74CFFB8
:10A6A80020232E60C0F88830002084F8840070BD14
:10A6B8000220FCE738B5084D052455F8043B2BB9B2
:10A6C800013C14F0FF04F8D1204638BDDB689847F8
:10A6D8000028F5D0F9E700BF2C100020034BD870F4
:10A6E800034B1B681B6C03B11847704714100020FC
:10A6F80010100020034B1874034B1B685B6C03B1EC
:10A70800184770471410002010100020F0B5314D84
:10A71800314B95F90420314E91B00C46012795F93B
:10A7280005108DF8047002288DF809208DF80A109C
:10A7380010D18DF80800D8711C7202F063FD3378CF
:10A7480003B114B101A803F0C1F9254B059A1A60A9
:10A7580011B0F0BD59714FF480711A71D9801C7213
:10A7680033788DF8087053BB1F2306A88DF81C207A
:10A778008DF8183002F024FF20238DF8183006A831
:10A788002B798DF81C3002F01BFF22238DF818302E
:10A7980006A86B798DF81C3002F012FF21238DF882
:10A7A800183006A86B798DF81C3002F009FF2923B0
:10A7B8008DF8183006A80B4B079302F001FF02F042
:10A7C80021FD012306A88DF818308DF81C3002F001
:10A7D800F7FEB4E71410002060080020F00E0020F7
:10A7E800E40F0020000400017FB5092301A88DF8BB
:10A7F800043003F06BF90038044B059A1A6018BF4F
:10A808000120404207B05DF804FB00BFE40F0020C0
:10A8180070B504460B46144962784A700020A27845
:10A828000A7208701A884A729A788A72DB780B74EE
:10A838006368CB600D4B1B68DA6A2AB1237803F092
:10A84800FB030A2B00D09047094E002556F8043B1D
:10A858001BB15B6A0BB1204698470135EBB2052B5B
:10A868006DB2F3D170BD00BF300800201010002079
:10A878002C10002070B5044611480123037063783A
:10A888004370A3788372E368C360E378037623692F
:10A898004376237943720B4B1B689B6A03B1984735
:10A8A800094E002556F8043B1BB19B690BB12046A5
:10A8B80098470135EBB2052B6DB2F3D170BD00BFDF
:10A8C80044080020101000202C100020014B1868AC
:10A8D800704700BFE40F002000B58BB00123684625
:10A8E8008DF8003002F046FD38B99DF804000038B4
:10A8F80018BF01200BB05DF804FB0020FAE7000048
:10A9080008B501F037FE40B9FFF7E6FF012806D089
:10A91800054B197AD879FFF7F9FE012008BDBDE883
:10A928000840FFF7C7BE00BF600800202DE9F041CE
:10A9380086B005460E46174601F01CFE002873D166
:10A9480001F030FE044640B9FFF7C6FF01280AD0DF
:10A958003D4B197AD879FFF7D9FE6FF002042046EB
:10A9680006B0BDE8F081DFF8E48088F80860003EB2
:10A9780018BF01268DF80460354E687833798DF854
:10A988001230694602F094FC00283FD08DF804404C
:10A998000394ADF810406FF0060495E803002D4BC2
:10A9A80083E80300337988F80A30394601A803F0B0
:10A9B80091F9294B059A1A6011283FD801A353F839
:10A9C80020F000BF37AA000831AA000845AA0008ED
:10A9D80045AA000845AA000845AA000845AA000893
:10A9E80063A9000845AA000845AA000845AA000866
:10A9F8002BAA000845AA000845AA000831AA0008A1
:10AA080031AA000831AA00084BAA00082B788DF853
:10AA180008306B78ADF810306B6803934FF0FF3453
:10AA2800BBE76FF005049AE76FF0010497E70B4B5B
:10AA380000221A70E31D18BF144690E74FF0FF3448
:10AA48008DE76FF004048AE76008002044080020BE
:10AA58001410002054080020E40F0020E30F002009
:10AA680037B501F0A9FD134D052455F8043B4BB14A
:10AA78001A693AB19B682BB1984718B155F8043C4C
:10AA88001B699847013C14F0FF04EED1FFF712FE52
:10AA980068B9094D2B7853B1084BADF80040D97807
:10AAA800019422466846FFF741FF00B92C7003B0B5
:10AAB80030BD00BF2C100020E30F00201410002030
:10AAC80030B58BB0044601F055FD0546002835D158
:10AAD800FFF702FF012834D168468DF8005002F0D4
:10AAE80049FC40BB9DF80430A34204D0012C22D07D
:10AAF800022C12D014B100200BB030BD002BFAD0BC
:10AB080068468DF8044002F05BFDA0B90E4B1B6847
:10AB18001B6B002BEFD09847EDE763B968468DF8BB
:10AB2800044002F04DFD30B9074B1B681B6B002B2E
:10AB3800E1D02046EFE74FF0FF30DDE76FF001008E
:10AB4800DAE76FF00200D7E71010002010B50446CE
:10AB58008AB018B94FF0FF300AB010BD002368461C
:10AB68008DF8003002F006FC0028F3D19DF804307F
:10AB78002370F1E77FB500220B4620498DF80720A6
:10AB880001220A7042784A700446002A33D10279B9
:10AB98000A721A884A729A788A72DB780B74036987
:10ABA800CB60C378164D8DF80830037B8DF80930DB
:10ABB800836803932B68DB6A0BB102A898472B685C
:10ABC8009B6B13B1227E02B198470E4E052556F8AD
:10ABD800043B1BB1DB690BB120469847013D15F0DA
:10ABE800FF05F4D10DF10700FFF7B0FF637913B14A
:10ABF800054B01221A7004B070BD00BF3008002058
:10AC0800101000202C100020E30F002010B504467F
:10AC18008AB018B94FF0FF300AB010BD202368463B
:10AC28008DF8003002F0A6FB0028F3D1024A9DF906
:10AC3800043023701371EFE71410002000B58BB0B7
:10AC48002323019068468DF8003002F0B9FC0038E3
:10AC580018BF012040420BB05DF804FB70B5654C8D
:10AC680001468EB01822204606F0C0F8624B00223A
:10AC78001A70F9F783F923784068012202FA03F180
:10AC8800014004D15D4B084608F09CF8FEE75C499A
:10AC98005C481A4602F0F8F818B14FF0FF300EB0D1
:10ACA80070BD272304A88DF8103002F089FC564E99
:10ACB800564D002870D1012333702B68DB690BB126
:10ACC80000209847272304A88DF8103002F052FB83
:10ACD800059B93F84820227093F8182193F81A31AD
:10ACE8006270A370464BD3E9020105F06FFF054679
:10ACF8000028D2D1464E062304A88DF8103002F061
:10AD080039FB059B736104A802F05AFC022304A8CE
:10AD18008DF81030059602F02DFB0836032304A8A1
:10AD28008DF81030059602F025FB0F2606F014F872
:10AD3800012304A88DF814308DF8106002F040FC4F
:10AD480010230DEB03008DF810308DF8145002F02D
:10AD580037FC04238DF8103004A8A3788DF814303C
:10AD680002F02EFC3A238DF8103004A8636905938D
:10AD780002F026FC02A920788DF8086004F09CF8FF
:10AD8800003818BF0120E0711420FFF757FFE07961
:10AD980003F062F9284682E728238DF810302B68E3
:10ADA8001B6943B104A802F0E5FA2B6805981B69F2
:10ADB80040F2C4519847272304A88DF8103002F0B8
:10ADC800FFFB50B9012304A88DF8103002F0D2FA25
:10ADD8009DF81430002B7FF46EAF3378002B7FF48E
:10ADE8006CAF052204A88DF81020059302F0E8FB4B
:10ADF80078E700BF14100020E30F0020203C010872
:10AE0800E80F002000100020F00E00201010002095
:10AE18005010002037B500230D4601930446D0B9E1
:10AE280000F0A8FB0190019BD3B10F4A42F82430EF
:10AE38000E4A9A620E4A1268916B1963916C5963B3
:10AE480092690C49D9625A6128465B680A49F2221C
:10AE58009847002006E001A900F092FB0028E2D004
:10AE68004FF0FF3003B030BD2C10002015A70008AC
:10AE780010100020F1A70008F10E0020194B07B5AB
:10AE88001860194B194A1A60194A5A60194A9A6087
:10AE9800194ADA60194B02681A6042685A60826877
:10AEA8009A60C268DA60164A1A6182695A61154B5B
:10AEB800C26B5A60144A019119609A601946134A84
:10AEC800DA600020FFF7A6FF48B901A800F056FB9A
:10AED800003818BF0120404203B05DF804FB4FF072
:10AEE800FF30F9E710100020001000207DA80008AE
:10AEF8007DAB000891AF000819A80008E80F0020F2
:10AF080071EE000840100020E5A60008FDA6000824
:10AF180049B118B1012804D000207047034B0B60D9
:10AF2800FAE7034BFBE74FF0FF30704700040001DE
:10AF38000100010208B503F0ABF8002814BF6FF058
:10AF48000100002008BD08B502F084F9002814BFEC
:10AF58006FF00100002008BD10B504468AB018B98A
:10AF68004FF0FF300AB010BD212368468DF800303D
:10AF780002F000FA0028F3D1024A9DF90430237048
:10AF88005371EFE7141000202DE9F0412F4D304F99
:10AF980000232B7043786B703B689B6A8AB0044629
:10AFA8000BB128469847DFF8AC80002658F8043BD8
:10AFB8001BB11B6A0BB1204698470136F3B2052B2B
:10AFC80076B2F3D12378052B2FD00B2B35D0012B5C
:10AFD80025D1214C062368468DF8003002F0CAF9C5
:10AFE8000199E07905F038FE10B91C4B019A5A61B5
:10AFF8001B48FFF70BFE1B48FFF7AEFF6B788BB9BA
:10B00800A371194B5878FFF75BFD3B685B6A0BB17E
:10B01800114898476B7813B9E07905F0AFFE0AB08C
:10B02800BDE8F081FF23A371EFE7104B01225A74AA
:10B03800227A9A74627ADA74F1E76378002BEED098
:10B048000AB0BDE8F041FFF7CFBB00BF44080020BD
:10B05800101000202C100020600800205010002044
:10B068006408002065080020141000203008002023
:10B0780030B58BB0FFF767FF0446F0B903F0FCFE6C
:10B08800831C1DD0F8B9134D2B685B69DBB12723EE
:10B0980068468DF8003002F06DF92B6801985B69FD
:10B0A8004FF4B961984703F0F9FE78B92CB9094B08
:10B0B8001B68DB690BB10120984720460BB030BDF7
:10B0C8006FF00704EFE74FF0FF34ECE74FF0FF3481
:10B0D800F3E700BF10100020014B1878704700BF3D
:10B0E80084100020014B5878704700BF841000205E
:10B0F80070470000044B9A7A0AB101225A70034B38
:10B108005B6903B118477047841000206C08002061
:10B1180073B5224C6378002B33D008F03BF966688E
:10B128000546FFF7D3FB0644AE4214D2A37A93B187
:10B13800E0228DF800208DF80130217AE368019330
:10B1480001226846FFF7F2FB08B1073010D100234F
:10B158006370A372656094F83430EBB1002384F80F
:10B1680034300F4B5B6BBBB102B0BDE87040184781
:10B1780040F2DC510B4808F0D9F90A4808F09CF96C
:10B18800E8E794F83520002AE5D094F8360084F8EA
:10B198003530FFF795FCDEE702B070BD8410002063
:10B1A8006C0800206810002037B5104D104CC8B14D
:10B1B800C1B16272012300222860E16023700D484A
:10B1C8000D4B00924FF0FF3108F0CAF800250B48EC
:10B1D80025822022294605F01DFE6570A574A586E6
:10B1E80003B030BD00232B602370EFE780100020F0
:10B1F8008410002068100020FDB00008981000207E
:10B208002DE9F0478E4C23788CB0002B56D0C278AD
:10B218000AB9837B13B1238A01332382437B002B32
:10B228004CD0E02A4AD10023A372876897F800809F
:10B23800B8F1220F27D8B8F1220F30D8DFE818F07C
:10B248004100FB0052005A0061006E0075008E003C
:10B258009D00B400C7002F002F002F002F002F00E3
:10B268002F002F002F002F002F002F002F002F005E
:10B278002F002F002F002F002F002F002F002F004E
:10B28800C900D000D400B8F17E0F00F0CC80B8F12E
:10B298007F0F00F0DF80B8F17D0F00F0AB80A57A5A
:10B2A800002D00F05B81674C637A3BB94FF47A71EB
:10B2B800204608F03BF9204608F0FEF80CB0BDE83F
:10B2C800F087E36801220021A2721970A37AE1686D
:10B2D8009818A0720620C854A37AE1689818A0723A
:10B2E800CA54DCE7584B9B6A002BD8D001210220B6
:10B2F8009847D4E77B7884F83630012384F83530D2
:10B30800CDE704238DF804307B78003B18BF012378
:10B3180001A88DF8083002F053F9C0E778780038B2
:10B3280018BF012002F098FEB9E7484E0FCE01ADD4
:10B338000FC50FCE0FC596E8070085E807007B7894
:10B348000A2BACD8424A12685268002AA7D00CA926
:10B3580001EB830353F82C0C9047A0E77878431E41
:10B36800012B9CD83A4B01381B6818BF012020726A
:10B378009B68002B93D0984791E7E2680123082146
:10B38800A3721170627A057BA17AAA4228BF2A4665
:10B39800934284D285685A1CEB5CE56801334E1CE5
:10B3A800A6726B54D3B2EDE7E3680122A2720922B8
:10B3B8001A70A37AE268218A581CA072D154A27A22
:10B3C800238AE1681B0A501CA0728B5467E723820A
:10B3D80065E705238DF8043001A802F077FB5EE7E6
:10B3E800194BDB6A98475AE7194B78781B686075E0
:10B3F800DB68BEE7037B072B7FF451AF06238DF88C
:10B408000430B7F80130ADF808307B793A791B047D
:10B4180043EA0223FA781343642253430393BB7924
:10B428008DF81030D8E73B2201A88DF804208DF85C
:10B43800083002F0C5F8012384F834302FE700BF44
:10B4480084100020681000206C0800200C3A0108C5
:10B45800801000202A2301A88DF8043001F08AFF0B
:10B4680094F80A90E6689DF808009DF809509DF840
:10B478000A709DF80BC09DF80D309DF80E209DF8C0
:10B488000F109DF80CE009F1010A84F80AA006F8EB
:10B498000980354E94F80A903668D4F80C8009F182
:10B4A800010A84F80AA096F803A008F809A094F8FD
:10B4B8000A90D4F80C8009F1010A84F80AA096F8D9
:10B4C80002A008F809A094F80A90D4F80C8009F1B1
:10B4D800010A84F80AA096F801A008F809A094F8CF
:10B4E8000A9009F1010A84F80AA096F80080E66833
:10B4F80006F8098094F80A80E66808F1010984F8DA
:10B508000A9006F808C094F80AC0E6680CF1010829
:10B5180084F80A8006F80C70A77AE66807F1010C2F
:10B5280084F80AC0F555A57AE6686F1CA7727055AD
:10B53800A07AE568461CA6722954A17AE0684D1CD9
:10B54800A5724254A27AE168501CA0728B54A37A67
:10B55800E268591CA17202F803E0A0E6034807F06C
:10B568005DFF6570AAE600BF80100020681000200B
:10B5780070470000004870476C08002000207047A2
:10B588004FF0FF3070470000044B054A93F818311C
:10B59800022B18BF062382F8903470472817002022
:10B5A800EC1C0020034BD3F8483313B15B6903B19B
:10B5B80018477047EC1C0020034A137843F0040333
:10B5C8001370FFF7EFBF00BFD01000201FB50A4B64
:10B5D8008DF8090093F87C208DF80A2093F88C20C8
:10B5E80093F848000D3202A98DF8082003F064FC96
:10B5F800C0B205B05DF804FB2817002008B507485D
:10B6080007F00CFF064B93F81A2412B1012283F8B5
:10B618001924BDE80840FFF7C5BF00BFEC20002093
:10B62800EC1C002010B50C4CD4F8403343F08003D8
:10B63800C4F8403394F81A3413B10020FFF7DEFF42
:10B6480094F8913423F0120343F0120384F89134F0
:10B65800BDE81040FFF798BFEC1C00202DE9F04131
:10B66800DFF8AC8098F81831022B06460D4602D058
:10B67800284BDB6A984702F0A6FD044628B1022051
:10B6880002F097FD002002F099FD98F81831012B7F
:10B6980017D102F09AFD074630B1002002F08AFD6A
:10B6A800002002F08CFD3C4602F091FD48B10020DC
:10B6B80002F081FD002002F083FDBDE8F041FFF7B4
:10B6C80063BF002CF9D1144C94F8902494F81A34E0
:10B6D800BAB90BB184F84164304602F017FFD8F8C4
:10B6E8002C0007F061FED4F8B4339842E5D30B4838
:10B6F80007F094FE94F8913443F0100384F89134E1
:10B70800DBE70BB184F84154284602F0FFFEF1E76D
:10B71800281700209C430108EC1C002084200020EE
:10B72800074A10B5137843F002031370FFF73AFF86
:10B73800BDE81040034B01220021022007F042BB64
:10B74800D0100020693C0108074A10B5137843F06F
:10B7580008031370FFF726FFBDE81040034B0122D2
:10B768000021022007F02EBBD0100020793C0108F0
:10B778002DE9F0410F4616461D46804607F00AFEA1
:10B788000B4A0C4C1378278123F0110343F0110363
:10B79800C4E90008137066812573FFF703FFBDE84D
:10B7A800F041054B01220021022007F00BBB00BF2E
:10B7B800D0100020BC100020893C010813B507F008
:10B7C800E9FD0D4B6C461860204607F037FD94E8FC
:10B7D80003000A4A0A4B83E80300137843F0200366
:10B7E8001370FFF7DFFE074B01220021022002B091
:10B7F800BDE8104007F0E6BACC100020D0100020B9
:10B8080024200020963C01082DE9F04192B006461C
:10B8180002F0D9FC002840F05881AD4D95F8183158
:10B82800012B09D02B6BAB4C93B194F80431BBB10D
:10B83800042B6FD0032003E002F0C7FC18B10F20DF
:10B8480012B0BDE8F08102F0C2FC0028EAD0F6E7A9
:10B85800B5F82031D4F81C24013B53432B63E4E7AB
:10B868009D4803F060FA002840F0128194F80C31EA
:10B8780023802B6B0C930DF1180895F839308DF84F
:10B888003830404695F81C318DF83A3007F0FCFC0A
:10B89800D5F82831009302AF98E80600D5F824318E
:10B8A800384607F088FC97E803000FAB83E80300ED
:10B8B800EB6A0D9300238DF844302388ADF84630A9
:10B8C80095F8303101228DF839201BB98DF84420C4
:10B8D8008DF83930814B0093814B95F84800A3F1DE
:10B8E80079020CA903F05DFBC0B10B28A8D1D4F8EC
:10B8F800941499B1002EA3D0D4F84033794843F07A
:10B908002003C4F8403307F011FE764807F0D4FD51
:10B91800002095E7704803F03AFAA4E795F84870D4
:10B9280095F9693095F9392095F87D106E4E3846AD
:10B9380003F044FB009641B2EB6C95F85020384672
:10B94800183603F0DFFA0096EB6C95F8502095F95D
:10B95800701095F8480003F0D5FAD4F8C413AB6D0D
:10B96800D4F8DC230B44C4F8B033EB6D1344C4F8AB
:10B97800B43394F80431042B07D02B6E0B44C4F86D
:10B98800B0336B6E1344C4F8B4330023089395F8AE
:10B998003031002B40D100238DF8133095F8393021
:10B9A8008DF8213095F838308DF82230D5F8803070
:10B9B8000993D5F884300A932388ADF82C3095F88C
:10B9C800303194F81B648DF82E3095F84800474BB9
:10B9D8008DF820600DF1130208A903F0A7FA0123DE
:10B9E80084F8413495F8393084F842349DF813309E
:10B9F80084F84334D4F81C34C4F85064C4F8483488
:10BA0800C4F8583402F0E5FBC8B1D4F81C0402F0BD
:10BA1800F2FBA0B1102013E708A802F0A7FC60B958
:10BA280095F9390094F837629DF82070FFF7CEFD3C
:10BA38003E44B042AFD2082002E7132000E795F851
:10BA48001831012B01D102F0D8FB02F0C5FB00230D
:10BA5800059394F8043195F9395094F81B649BB117
:10BA6800042B7FF4E7AE05A802F0B4FE58BB94F8A7
:10BA7800183413B1059B013B0593174B05983246C3
:10BA8800E9B202F00DFF02E0134802F0DDFE08B152
:10BA98001120D5E6D4F8403394F80C11218043F0F6
:10BAA8000203C4F8403394F8183411480133DBB268
:10BAB80084F8183484F845340E4B00259B6AC4F882
:10BAC8009854984724E71220BAE60E20B8E600BF3B
:10BAD80028170020EC1C0020F41D00205817002017
:10BAE8008021002054200020A420002008210020CC
:10BAF800EE1C00209C43010873B5134D134E0096AD
:10BB0800EB6C95F8502095F9781095F8480003F0FB
:10BB1800F9F995F83031337595F8480040F201236A
:10BB280006F13C023146738203F0F8F950B196F8F9
:10BB38003C3086F88230064B00205B6B9847F37CDC
:10BB480086F8A83002B070BD28170020D420002045
:10BB58009C430108F8B5324C94F81831012B05467E
:10BB68000ED0022B4ED0002B57D138B9D4E91B0187
:10BB780004F1740383E803000020F8BD012806D10E
:10BB880002F02CFB0028F8D184F81851F5E70228B8
:10BB980043D1244E84F8180106F5747CBCE80F00E4
:10BBA80006F57A770FC79CE8030094F8E92094F823
:10BBB800003187E8030086F8FB53D2B1022B18D175
:10BBC800D4F804316367C6F8EC3394F87D3094F800
:10BBD800082186F8F83394F88C3084F8782086F8B1
:10BBE800F93396F81B2486F8E82340F20133A6F8C7
:10BBF800FA33002386F81A340B4BDB6A9847FFF7B1
:10BC08007BFFB9E748B9074B84F81801062283F887
:10BC18009024054BDB6A9847AEE70320ADE700BFE9
:10BC280028170020EC1C00209C430108F0B5504C5C
:10BC3800504EB4F8DC202287D4E92D0194F8B120C5
:10BC480084F8692004F16C0282E80300D4E92F012A
:10BC580004F1740282E80300B4F8C420A4F87C203C
:10BC680091B0D4F8CC20D4F8C810C4F884200025AA
:10BC7800D4F8D020C4F888200123A4F82031C4F8CF
:10BC8800801084F83051A56284F81B5184F83A502A
:10BC980084F81D5184F81E51C4F83451C6F89854DC
:10BCA800A6F8185486F81A54A4F838518DF81830A4
:10BCB80004F50973039304F50A7394F84800049390
:10BCC80003A92D4B84F84551C4E94F55A4F84651B2
:10BCD800059303F0FFF8E36EC6F8D43394F87D308B
:10BCE80086F8E03394F88C3086F8E1334FF48073AB
:10BCF800A6F8E23386F8D05394F8303186F8E43366
:10BD080006F574770FCF06F57A740FC497E8030029
:10BD180040F2012384E80300A6F8FA33D6F8483342
:10BD280086F81B54CDE901551BB15A685B6901922D
:10BD38000293124B0793A3F148020892A3F114024D
:10BD480009920F4A0B9229330A93A2F19C030C9390
:10BD5800A2F198030D93131D0E9301A902F14C0350
:10BD680007A802F599620F9302F022FA11B0F0BD0C
:10BD780028170020EC1C0020D4100020542100209B
:10BD88000C180020F8B50D4F0D4E0C4607F046FB79
:10BD98003B6B98470B4A96F84800214603F0BEF8DB
:10BDA80050B1094D706D95F8243485F86A347B6B71
:10BDB8009847E37C85F89034F8BD00BF9C430108A0
:10BDC8002817002010210020EC1C00200F4890F8B4
:10BDD8001B3480F8B8330E4B93F8692080F8BB23E6
:10BDE80093F87D2080F8C82393F88C2080F8C92325
:10BDF80093F8303180F8CC330022A0F8CA2300F53C
:10BE08006E7100F56070FFF7BDBF00BFEC1C00202D
:10BE180028170020114890F89034EBB190F81B34A3
:10BE280080F8D0330E4BDA6EC0F8D42393F87D2017
:10BE380080F8E02393F88C2080F8E12393F83031E0
:10BE480080F8E4334FF48072A0F8E22300F57471AF
:10BE580000F56670FFF796BF704700BFEC1C002026
:10BE68002817002070B5344C2421204604F0D4FF54
:10BE7800636A984218BF60624FF01C012F4814BFD4
:10BE88000125002504F0C8FF636C984218BF606460
:10BE98004FF480712A4818BF45F0020504F0BCFF32
:10BEA800D4F84831984218BFC4F848014FF0D4017B
:10BEB800244818BF45F0040504F0AEFFD4F820323A
:10BEC800984218BFC4F820024FF000011E4818BF5E
:10BED80045F0080504F0A0FFD4F82432984218BFB2
:10BEE800C4F824024FF46071184818BF45F01005D3
:10BEF80004F092FFD4F8A835984218BFC4F8A805F2
:10BF08004FF01401124818BF45F0200504F084FFD3
:10BF1800D4F8C03598420F4B18BFC4F8C005D3F801
:10BF2800483318BF45F040052BB11B691BB12846A3
:10BF3800BDE87040184770BD281700205017002032
:10BF480070170020741800204C1900205019002088
:10BF5800D41C0020EC1C00202DE9F04F8FB04FF0CE
:10BF68000009012B06460F4690468DF80D90ADF856
:10BF7800109002D84C46BC4202D30FB0BDE8F08FF7
:10BF8800305D02F033FA2044B842F6DC335D651CBC
:10BF9800023BEDB2112BF0D801A252F823F000BFFA
:10BFA800F1BF00081BC0000819C1000841C1000802
:10BFB800BFC10008E5C100084BC2000873C20008F1
:10BFC800F9C2000883BF000883BF00084DC30008FA
:10BFD80083BF000883BF0008F5C300081DC400081C
:10BFE80055C4000889C40008052002F0A7FA70B1FA
:10BFF8000521002002F068FA725DBA4BE51C023494
:10C00800E4B283F85C24325D83F85D24EDB22C46FB
:10C01800B1E700238DF80E308DF80F308DF814300D
:10C028008DF81830B9F1000F6DD1AF4C4FF00509FC
:10C0380094F87C208DF831206B1E94F839208DF807
:10C048003320334494F838200B938DF8342094F837
:10C058001A3194F868208DF83520D4F82C218DF801
:10C0680032300A9273B37B1C5B1BDBB28DF8303025
:10C0780006AB019305AB009394F848000DF10F034C
:10C088000DF10E020AA902F05DFF8DF80D0000F017
:10C098000700072813D194F939209DF90E3084F848
:10C0A80039309A429DF80F3084F83830B8BF0122F1
:10C0B8009DF81430B8BF84F81D2184F868304FF01B
:10C0C800000A09E00523D1E701220DF10D01032043
:10C0D80002F0A4F80AF1010A5FFA8AF29DF8183012
:10C0E800B3FBF9F19142EFD82B44DDB26B1EDBB202
:10C0F8009F420BD9F25C032A9AD0AF4288BF1D46F3
:10C108004FF0010983E70534E5B2F9E71D46F7E783
:10C11800735D754903F00F03012281F81B31023466
:10C1280002FA03F3A1F82031E4B2002204A90420A2
:10C1380002F074F825466AE707238DF80D30735D21
:10C14800C3F3021203F00F038DF82830E31CDBB2AF
:10C158008DF82920F25C231DDBB2651DF35C0234E7
:10C16800E4B21B0443EA0223325D5F4C13436422AA
:10C17800534394F848000B930AA902F0F2FE00F02A
:10C188000703072BEDB28DF80D000CD19DF8283070
:10C1980084F8703084F878300B9BE36663679DF809
:10C1A800293084F869308DF81000012204A905208F
:10C1B80002F034F82BE74B4BD3F8483363B11B68D4
:10C1C80053B1984708F03F038DF810008DF81130EF
:10C1D800022204A90620EBE7FF20F3E703238DF8EA
:10C1E8000D30735D8DF81C300AAB0693E31CDBB28F
:10C1F800A51DF25C231DDBB206A9F35C1B0443EA10
:10C208000223A21CD2B20534B25C13436422534306
:10C21800E4B20A9300230B93335D8DF83030324B30
:10C2280093F8480002F0A3FEC3B20028EDB28DF8DF
:10C238000D30FFF6ECAE8DF81030012204A907206E
:10C24800B6E7735D03F00F03012B4FF47A7238BF22
:10C2580001235343244A0234936503F57A73D36563
:10C26800E4B2002204A9082062E7735D1E4DC3F3FF
:10C2780040128DF8152095F84800C3F3001205A95F
:10C2880003F00F038DF814208DF8163002F075FEB8
:10C2980002340130E4B23FF44DAFBDF81430134A14
:10C2A800A5F87C309DF816309DF814A0D05CF5F701
:10C2B800ADFB0223C5F880000AA995F848008DF85F
:10C2C80028308DF82AA002F0F7FD95F9393006904C
:10C2D80040B29842B8BF184685F83900002204A930
:10C2E800092025E7EC1C002028170020A33C0108A2
:10C2F80003238DF80D30735D8DF82830E31CDBB215
:10C30800651DF25C231DDBB20234F35CE4B21B044E
:10C3180043EA0223325D1343642253430B93644B75
:10C328000AA993F8480002F02EFEC3B20028EDB225
:10C338008DF80D30FFF66BAE8DF81030012204A990
:10C348000A2035E7092002F0F9F8DFF868B100287B
:10C3580049D00921002002F0B7F80023ADF81E30BB
:10C36800A31CDBB2F25CE31CDBB216F803A0735D1E
:10C378004FEA0A4A4AEA022A4AEA030A231DDBB2BA
:10C38800A51D0534F35CE4B24AEA036A335D4FF451
:10C398007A7253430AAC1B122046ADF81C3006F0E3
:10C3A8004DFF454B53440693DBF83C3300930DF1A6
:10C3B800180A9AE80600DBF8383308A806F0FBFEEE
:10C3C800099B009394E80600089B504606F0D8FEA7
:10C3D8009AE8030006F00AFF01F00AFF0123EDB214
:10C3E8008BF8383413E68BF8380410E60C2002F08A
:10C3F800A5F800283FF40BAE0C21002002F064F8E9
:10C408002C4B93F89034043B012B7FF600AE01F0DF
:10C41800EBFEFCE5A31CDBB2725DF15CE31CDBB256
:10C42800651DF35C0434E4B21B04305D43EA012368
:10C4380013436421594300F00F0001F0D6FEEDB21A
:10C448008DF81000012204A91120B1E60D2002F098
:10C4580075F800283FF4DBAD0D21002002F034F818
:10C46800A31CDBB2154AF05C735D1268251D03340A
:10C47800E4B243EA0020315DEDB201F0B8FEC6E552
:10C48800725DA31C251D0334DBB2E4B2F15C335D9D
:10C498001B0443EA012313436420584301F0A9FE17
:10C4A800EDB28DF81000012204A9132080E600BF28
:10C4B80028170020EC1C0020803DD512BC1000205D
:10C4C8000E4B93F89124920703D593F88F24012AF1
:10C4D80008D90B4991F81A2122B18A6A501C18BF51
:10C4E80001328A620022A3F8182483F81A24D3F8A8
:10C4F800402322F00202C3F840237047EC1C0020BE
:10C508002817002070B5184C1848194D06F086FFFA
:10C51800D4F84033D4F89804D5F8906023F0200379
:10C52800C4F8403338B106F03FFF864203D20023F7
:10C5380085F83A3070BD0120FFF766F90028F9D078
:10C548000B28F7D095F8393084F84234092094F84C
:10C55800183484F8453484F8410401F0D7FFBDE865
:10C568007040FFF7ADBF00BFEC1C00205420002036
:10C5780028170020094BD3F84023012A0AD008497C
:10C588000978C90708D43AB993F89204013818BF52
:10C59800012070470020704701207047EC1C0020E4
:10C5A800D0100020034BD3F84003431E5842584193
:10C5B800704700BFEC1C00202DE9F04FA9B0EFF345
:10C5C800108272B6DFF8F0B20021DBF80030CBF849
:10C5D800001082F31088B94C002B00F0E180DAB229
:10C5E8009B06039264D5B64D95F81831022B02D0FC
:10C5F800B44BDB6A9847EFF3108872B6B24F06F077
:10C60800C9FE3E68D4F8B013361A3144AF4806F074
:10C618008DFFAE4806F050FFD4F8B413AC4831444F
:10C6280006F084FFAA4806F047FF88F3108894F8BC
:10C638001A34002B00F06B81152312A995F84800D5
:10C648008DF8483002F038FCD4F8B4130F90014448
:10C65800A04806F06BFF9F4806F02EFF3B6894F851
:10C668001B24EB620DAF38468DF870201D9306F041
:10C678000BFED5F82831009306AE97E80600D5F8EA
:10C688002431304606F097FD96E803001FAB83E897
:10C698000300D4F81C341E9395F8303195F84800FF
:10C6A800003B18BF01231CA98DF8713002F00DFC66
:10C6B800039BDF0648D5824DDFF81CA2D5F8E4209D
:10C6C80004929BF80020BAF90A809AF90C90A4F811
:10C6D8008C84002363F300020A9384F84434A4F89A
:10C6E800223484F82534C4F82834A4F82C3484F887
:10C6F8002E34C4F8303484F82034C4F8343484F840
:10C708003834C4F83C346F4B8BF8002094F89024EC
:10C71800DB6A84F88E9484F88F24DAF80470BAF807
:10C728000860984794F88F3413B9694806F076FE84
:10C738003146384601F045FD8346002800F0EA807E
:10C74800A4F87E8484F88094039B19071AD55C4B5F
:10C7580093F81831022B02D05A4BDB6A9847022013
:10C76800FEF712FF84F8410401F0D0FE94F81A3461
:10C7780013B1012384F8193494F8913443F0100369
:10C7880084F89134039B5A0703D506210520FEF748
:10C7980065FF039B9B0703D504210320FEF75EFF7B
:10C7A80001F02DFD94F89124D7065FD5002384F875
:10C7B8009234D4F840331E0644BF23F08203C4F8F1
:10C7C800403312F0050F00F0FB820B2001F0B6FE9B
:10C7D800002800F0F58294F89134DD0700F1F0822A
:10C7E800580740F10783D4F8403323F00203C4F814
:10C7F8004033D4F8402382BB94F8915415F00101DA
:10C808001EBF2B4662F3000384F8913494F89134E8
:10C818005E0744BF6FF3820384F89134012384F8E0
:10C82800923421B1D4F844332C481B6898476D07DB
:10C838000BD52B4801F08EFE01F0BCFE28B194F810
:10C84800913443F0040384F8913401F0C6FC94F861
:10C8580091346FF3041384F89134012384F89234EB
:10C8680094F8913443F0200384F8913494F8913487
:10C8780018070AD56FF3C3031A4984F89134D4F81A
:10C888004433A1F12400DB68984794F89134990760
:10C898000AD56FF34103134984F89134D4F844332B
:10C8A800A1F16C005B68984794F89034022B1BD177
:10C8B800FFF722F918E000BFD0100020EC1C002080
:10C8C800281700209C430108CC1000206C20002071
:10C8D80084200020EC200020BC1000202C21002007
:10C8E800402100207821002094F891349A0640F1E4
:10C8F800C4826FF3451384F89134D4F84033002B85
:10C9080040F0BB8229B0BDE8F04FFFF7ABBA84F81E
:10C918004134A3E695F81831012B0CD101F055FCF0
:10C92800804668B1584601F045FC584601F047FC7E
:10C93800042384F88F347EB9012384F821344FE12D
:10C9480001F045FC0028F6D0404601F034FC404692
:10C9580001F036FC0523ECE73B7805935B09013BC6
:10C96800062B00F21782DFE813F007001502950086
:10C978001502920015020602102EDDD995F8303105
:10C988001297F6B28DF84C60002BD5D11CA804F094
:10C9980055F912AA1CA9FF2002F09EF89DF85830FC
:10C9A800C3F3030307468DF82C3095F8480095F833
:10C9B8007D308DF82D3007220BA902F090FA002F58
:10C9C8005DD100285BD09DF853309DF85220159911
:10C9D800C5F8E4101B0443EA02239DF85120022005
:10C9E8001343C5F8E03004F037F99DF8583095F84E
:10C9F800480085F82E71C3F30212C3F3030385F8C8
:10CA0800703085F878309DF8593085F86920012B09
:10CA180038BF01234FF47A725343AB651344EB6577
:10CA28000DF15A034FF001081093113E94F81B348E
:10CA38008DF83C300FA985F868808DF8446002F0C5
:10CA480056FA0223404685F8303101F077FD18B1D7
:10CA58004146384601F038FD94F88F34012B00F236
:10CA6800A78194F81A34002B40F09A8194F89134F5
:10CA780043F0100384F89134FEF786FD64E6012044
:10CA880001F05CFD0028E7D001210720E2E701233F
:10CA980084F8203495F87D308DF82E3094F82434BD
:10CAA8008DF82D3095F88C3095F848000D330BA98A
:10CAB8008DF82C3002F000FAA6F10D031BB2099094
:10CAC80023EAE37300B283423FF736AF0B2E7FF6BB
:10CAD80033AFBA4B25931CA8FF231C978DF87460BD
:10CAE8008DF8983002F0C4F8074600287FF424AF88
:10CAF80095F81831012B13D101F067FB002872D08B
:10CB0800384601F057FB384601F059FB04239DF8DD
:10CB18007C101E9884F88F34C1F3001101F06EFB6D
:10CB28009DF87C301E99C4F8341413F00F0203D01A
:10CB38009DF89000002862D19DF89800002861D0E7
:10CB4800002A7FF4F9AE9DF89020002A14BF4FF018
:10CB580003084FF0020800220A92D5F8EC2095F855
:10CB6800E900914251D100284FD0D5F80C1195F821
:10CB7800EAB009680A9195F81811022902D103212F
:10CB880084F88F14B8F1030F7FF4D6AE13F0600F5A
:10CB98007FF4D2AE0492012795F82E31BBF1000F35
:10CBA80036D0BBF1010F13D1012B33D16FF0090639
:10CBB80046FA08F606F00106C6F10206F6B2BDF816
:10CBC8007E100AAA304601F011FE38B3072823D098
:10CBD800012384F821340A9BC4F83034C4F86C3437
:10CBE800FEF720FDB0E501F0F2FA002898D03846AB
:10CBF80001F0E1FA384601F0E3FA052387E74FF040
:10CC08000008A8E74FF00108A5E74FF0010BC3E7BC
:10CC18000426D4E70326D2E70823DAE71CAB0093FF
:10CC280004990A9B3246584601F0A2FE20B1022818
:10CC380014BF0B230A2380E60A9BC4F83034C4F8D7
:10CC48006C349DF87C3084F82104C3F3401384F8D5
:10CC58002E3484F8443494F88F3484F82274012BE9
:10CC68009EBF0122A86285F81E21012FC4F828045E
:10CC780084F82C0484F8410438D1022284F8202452
:10CC880095F83A20002A4AD19DF87C20D60646D449
:10CC9800012B94F840149DF87C2005D8012901D176
:10CCA800900601D501F04CFBB8F1020F94F88F34CF
:10CCB80043D0B8F1030F0AD09DF87C10B8F1010FEA
:10CCC8004A4601F00F0120A83BD0FFF745F99DF82F
:10CCD800903084F82334259BC4F828349DF8983084
:10CCE80084F82C34012384F82D3430E0059A02F0BE
:10CCF800E002A02A1BD195F82E11012285F83A20CE
:10CD080009B927996963012B84F8202407D9D5F834
:10CD18009020C4F83C24DAF80020C4F8982495F848
:10CD28001821002AB4D1012284F82524B0E7002272
:10CD380085F83A2084F82024A6E79DF898102598CD
:10CD48004A46FFF709F99DF8903084F823349DF896
:10CD58009020E02A08D195F81F312BB984F82324B4
:10CD6800C4F82834A4F82C3494F8913443F002031E
:10CD780084F8913470E6114D013EB2B2791C284610
:10CD880004F034F80323A4F82034C4F8285484F8B1
:10CD98002C64E9E7012384F82134FEF743FC5BE6C1
:10CDA80094F84434002B3FF461AE0020FEF726FCD3
:10CDB80094F88F34022B3FF45FAE57E6241F00200F
:10CDC80094F89134590715D5012001F0B7FB60B1EB
:10CDD800012001F08BFB08B984F81804D4F840331B
:10CDE80023F00203C4F8403304E0062001F0A6FB58
:10CDF8000028F3D194F89134DA077FF5FAAC94F867
:10CE080040240AB1032A18D11D4A94F8181492F83C
:10CE18006820914205D29B0723D594F88F34012BC3
:10CE28001FD8184806F0FAFAD4F8403323F0200344
:10CE3800C4F84033FFF744FBDBE4012A11D194F82E
:10CE48001924002A3FF4D5AC0D4A94F8181492F826
:10CE580068209142E5D29F0703D594F84434002B0B
:10CE6800DFD194F8913400206FF3041384F89134DF
:10CE780084F81904FFF746FBBBE429B0BDE8F08F3E
:10CE880028170020542000202DE9F04F89468DB046
:10CE980090460746002800F08F81002900F08C8119
:10CEA8000368002B00F088814368002B00F0848120
:10CEB8008368002B00F08081C368002B00F07C8120
:10CEC800104601F0F5FF002800F07881BD4CBE4DFA
:10CED800384601F0AFFA40F2C4520021204603F070
:10CEE80099FF40F21C520021284603F093FFB74BEC
:10CEF800C4F82C3104F50973089304F50A73002665
:10CF08004046099308A9B24B84F848800A9384F8EC
:10CF1800186184F88C608DF82C6001F0DBFF0F231A
:10CF280006A994F848008DF8183001F0C5FF801B59
:10CF380018BF01204FF00A0B84F81C0106A994F8C9
:10CF480048008DF818B001F0B7FF4FF0060A84F8D2
:10CF5800DC0006A994F848008DF818A001F0ACFF91
:10CF6800102384F8DD0006A994F848008DF81830DD
:10CF780001F0A2FF1123C4F89C0006A994F8480008
:10CF88008DF8183001F098FF1223C4F8A00006A904
:10CF980094F848008DF8183001F08EFF1323C4F878
:10CFA800A40006A994F848008DF8183001F084FF11
:10CFB8001423C4F8A80006A994F848008DF818307E
:10CFC80001F07AFF1623C4F8AC0006A994F84800CB
:10CFD8008DF8183001F070FF172384F8B10006A906
:10CFE80094F848008DF8183001F066FF18230DEB0F
:10CFF8000301C4F8B400C4F8BC0094F848008DF8E4
:10D00800183001F059FFC0B21D2384F8B80084F825
:10D01800C00006A994F848008DF8183001F04CFFBC
:10D028001E2384F8C40006A994F848008DF8183027
:10D0380001F042FF1F2384F8C50006A994F84800B0
:10D048008DF8183001F038FF2023C4F8C80006A96D
:10D0580094F848008DF8183001F02EFF0B23C4F81F
:10D06800CC0006A994F848008DF8183001F024FF88
:10D078000C2306A9A4F8D00094F848008DF81830BD
:10D0880001F01AFFD4F89C306365D4F8A030A3658A
:10D09800D4F8A430E365D4F8A83023664FF001082B
:10D0A800D4F8AC300590A4F8D200636684F8B08058
:10D0B800C4F894B084F898A0C4F84CB084F850A090
:10D0C80084F8688084F81F81C5F84893FEF7AEFDA0
:10D0D800C5F84473C4E90B663E4B84F8198185F89A
:10D0E8009164C5F8408332464FF0FF31009605F54C
:10D0F8005A7006F035F9384B009632464FF0FF313A
:10D1080005F5607006F02CF9344B009632464FF066
:10D11800FF3105F5667006F023F902AF304B009633
:10D1280032464FF0FF3105F5806006F019F93846B0
:10D1380006F0AAF897E8030004F5927383E8030061
:10D14800284B294F1E60294BC5F84C33284BC5F88E
:10D158005433284BC5F85C33274BC5F85033274B5D
:10D16800C5F8583305F553703B68984704F5A67021
:10D1780003F080FB20B1112630460DB0BDE8F08FDA
:10D18800204601F003FB0028F5D101F039F8B8B9C1
:10D198001B4801F04DFB06460028ECD17B699847F7
:10D1A80003F002FEBB6D94F819019847FB6A984793
:10D1B800012385F89234DFE70326DDE70926DBE75C
:10D1C8001326D9E728170020EC1C002000040001D2
:10D1D800D41000200DC50008D5BD00081DBE0008EC
:10D1E80005B60008D01000209C430108C5B7000808
:10D1F80079B70008C1B5000851B7000829B7000879
:10D208001018002008B5034B0020C3F84003FEF7B0
:10D21800BBF908BDEC1C002010B5FFF7ABF90A4CB0
:10D2280060B90A4B93F81831022B02D1084BDB6A1C
:10D2380098470123C4F84033002010BDD4F84003B8
:10D24800013818BF0120F8E7EC1C0020281700203F
:10D258009C43010838B5124C204606F0DFF804F16B
:10D26800180006F0DBF804F1300006F0D7F804F1F6
:10D27800980006F0D3F800F0AFFF0A4B0025DB6AF0
:10D28800984744F8285CFEF7EDFD0749074840F247
:10D29800C45203F0ABFD012344F8283C284638BDAE
:10D2A800542000209C430108281700206411002006
:10D2B80070B52E4B8AB0054693F8DD008DF809004D
:10D2C80093F8DC008DF80A0029489A6A90F8180447
:10D2D800039200268DF80B0004960C46002940D0D6
:10D2E8000692D3F8882007921A8F93F81A118DF8AE
:10D2F800151052BAADF8202093F87C2093F84830E6
:10D308008DF8243003AB8DF822008DF8232000938C
:10D318000DF10A020DF10B030DF1090105A88DF8B5
:10D32800146000F0D7FE9DF90900FEF74FF9607010
:10D3380004A801F01BF8B0B9049A0F2A0DD8637835
:10D348009A420AD81544AB42A3EB02012CBF002035
:10D3580001202170C0000AB070BD0023237008208E
:10D36800F9E70320F7E71320F5E700BF28170020A7
:10D37800EC1C00201FB50446002800F0108103783B
:10D38800412B00F20781DFE813F0420049004D000D
:10D398005100550059005E00050105010501050110
:10D3A8000501050105010501650069006D007800AA
:10D3B8007F00820085008A0088008C00900093001E
:10D3C800960099009C009F00AE00B200BA00B6001B
:10D3D800BE00C100C500CE00CA00CC000501D200C5
:10D3E8000501050105010501050105010501050105
:10D3F8000501050105010501050105010501DA0021
:10D40800DE00E200E700EB00EF00F300FC00664BF3
:10D4180093F818312371002004B010BD624B93F8C3
:10D428003031F7E7406803F0C3FBF4E7406803F0E6
:10D4380005FCF0E75C4B93F81A31EBE75A4BD3F84D
:10D44800E0306360E7E7584B011D93F8300103F0C3
:10D458000DFCE0E7544B93F81931DBE7524B93F896
:10D468008C30D7E71C238DF808304F4B02A993F86E
:10D47800480001F021FD6060CDE74C4B043493E88F
:10D48800030084E80300C6E7494B0434F7E7494B37
:10D498000434F4E7484B0434F1E71A23E3E719238B
:10D4A800E1E7414B93F86830B4E73F4B5B6DC8E761
:10D4B8003D4B9B6DC5E73C4BDB6DC2E73A4B1B6EA2
:10D4C800BFE7394B5B6EBCE702238DF80830364B5B
:10D4D80002A993F87C2093F848008DF80A2001F0FF
:10D4E800EBFC207197E7304B93F8DD3092E72E4B39
:10D4F80093F839308EE72C4B93F8DC308AE72A4BC7
:10D5080093F8383086E7284BDB6C9AE7264B93F87C
:10D5180050307FE7244BD3F8843063607BE7224B9D
:10D528008FE7264B8DE7204BD3F8CC30F5E71E4B21
:10D53800D3F82C31436001F04DFDA0606BE71A4B26
:10D54800D3F890307DE7184B93F81F3162E7164BFC
:10D55800B3F88830A3805EE7134BB3F88A30F9E755
:10D56800114BB3F8D030F5E70F4BB3F8D230F1E7F1
:10D578000D4B93F848200AB1062A12D1B3F8A0350A
:10D58800E8E7094B93F848200AB1062A09D1D3F8ED
:10D59800A43556E704B0BDE8104000F021BE0320D2
:10D5A8003AE7182038E700BF281700209417002012
:10D5B800DC1700209C170020E417002064110020CD
:10D5C8007FB5044610B9032004B070BDA34DD5F84B
:10D5D80040339A0700F16F820278412A00F268828C
:10D5E800DFE812F04200470055005B005F0064006E
:10D5F80069007600810087008D00930099009F00E4
:10D60800A500AB00B5006602BA00DC00EF00160109
:10D618003801290142014B014F01530157015B01B8
:10D6280066025F01710199018701AB01B101B8017F
:10D63800BD01C2016602280266026602660266022F
:10D648006602660266026602660266026602660292
:10D658006602660266026602340239023E0243022C
:10D6680048024D0252025C020079FEF773FA30B1AB
:10D67800AAE70379022BA6D0794A82F8303195F8C7
:10D68800913443F0200385F8913400209CE74068EA
:10D6980003F080FA0028F2D095E7406803F0BEFA5C
:10D6A800F8E76F4B027983F81A21E8E76C4B426878
:10D6B800C3F8E020E3E76A4E416896F8300103F0CA
:10D6C800CBFA00287FF47FAF6368C6F8E430D6E76A
:10D6D800416800293FF477AF002001F0DDF9002808
:10D6E800CDD0112070E7416800293FF46CAF0120CC
:10D6F800F3E7416800293FF466AF0820EDE7416889
:10D7080000293FF460AF0920E7E7416800293FF4AA
:10D718005AAF0C20E1E7416800293FF454AF0D20CF
:10D72800DBE7416800293FF44EAF0E20D5E741689A
:10D7380000293FF448AF0F20CFE74A4C484B007907
:10D7480083F81901A36D9847E36A984797E7444B14
:10D75800027983F88C2092E7414E037A8DF80430E1
:10D7680096F8480096F87D308DF80530072201A913
:10D7780001F0B5FB00283FF426AF636896F848002F
:10D788000193002201A901F0AAFB00283FF41BAF76
:10D798006C36D4E9010186E8030070E7304E037A5D
:10D7A8008DF8043096F8480096F87D308DF80530ED
:10D7B800072201A901F093FB00283FF404AFB43617
:10D7C800E7E7274E037A8DF8043096F8480096F874
:10D7D8007D308DF80530072201A901F080FB002873
:10D7E8003FF4F1AED4E9010106F1740383E80300C4
:10D7F80096F81831022B7FF442AF96F83031002B9F
:10D808003FF43DAF174BDB6A9847FEF775F936E7EB
:10D81800134E037A8DF8043096F8480096F87D3058
:10D828008DF80530072201A901F059FB00283FF4C3
:10D83800CAAEBC36ADE74368029301238DF80C30BD
:10D84800074B02A993F8480001F056FB00287FF423
:10D8580016AFB8E6436802930023EFE7EC1C0020FC
:10D86800281700209C43010803795A1E0E2A3FF608
:10D87800AAAE934A82F8683001E7914B42685A652C
:10D88800FDE68F4B42689A65F9E68D4B4268DA658A
:10D89800F5E68B4B42681A66F1E6894B42685A6690
:10D8A800EDE6874C037994F848008DF80430062299
:10D8B80001A901F014FB00283FF485AE9DF804305F
:10D8C80084F8DD30DBE67E4C03798DF8043094F87B
:10D8D800480094F87C308DF80630052201A901F043
:10D8E800FEFA00283FF46FAE9DF8043084F8393012
:10D8F800C5E6734C037994F848008DF804300A2281
:10D9080001A901F0ECFA00283FF45DAE9DF804305F
:10D9180084F8DC30B3E66A4C037994F848008DF853
:10D928000430092201A901F0DAFA00283FF44BAECD
:10D938009DF8043084F83830A1E6614B4268C3F89A
:10D948009420DA649BE65E4B027983F8982083F88A
:10D95800502094E65A4B4268C3F884208FE6584B0F
:10D968004268C3F8CC208AE6012B40F0A480554CCD
:10D978002421204603F050FA636A984201D0172008
:10D9880022E61C2104F1280003F046FA636C984251
:10D99800F5D14FF4807104F1480003F03DFAD4F852
:10D9A80048319842EBD1D42104F5A67003F034FA3B
:10D9B800D4F820329842E2D1002104F5097003F02E
:10D9C8002BFAD4F824329842D9D14FF4607104F577
:10D9D8000A7003F021FAD4F8A8359842CFD114215F
:10D9E80004F2AC5003F018FAD4F8C0359842C6D106
:10D9F800334E2146304640F2C45203F0F7F9204630
:10DA080040F2C452002103F005FA95F81B3485F85A
:10DA1800E833736FC5F8EC3396F87D3085F8F83342
:10DA280040F20123A5F8FA33274B96F819019B6DAC
:10DA3800984724E68379012B3FF6C5AD204B426811
:10DA48004068C3F82C2100F0BDFE48E61C4B426834
:10DA5800C3F8902013E61A4B027983F81F210EE6CB
:10DA6800174B8288A3F8882009E6154B8288A3F80B
:10DA78008A2004E6124B8288A3F8D020FFE5104BD9
:10DA88008288A3F8D220FAE50D4B93F848200AB112
:10DA9800062A12D1A288A3F8A025F0E5084B93F82E
:10DAA80048200AB1062A08D16268C3F8A425E6E529
:10DAB80000F098FBDBE5012086E5182084E500BF2F
:10DAC80028170020641100209C4301082DE9F04329
:10DAD80087B00023ADF800300646002800F0EE803D
:10DAE8000361FEF747FD20B10124204607B0BDE8D9
:10DAF800F08300F065FD0028F6D100F05BFD0146DB
:10DB080018B96F48142203F085F96E4D95F89134D1
:10DB1800012243F0040385F8552485F891343378BD
:10DB28008DF804300021013B8DF80520ADF8061072
:10DB38000C2B00F2BB80DFE803F007B9B9B9798292
:10DB4800B9B990B9AD9AA900D5F8407317F0200774
:10DB5800CAD196F80480B8F1020F46D1DFF868817F
:10DB68005A4CFEF763F896F9051098F848003A46BB
:10DB780001F00FFA88F83900B37988F83830384658
:10DB880007238DF80530FDF7E5FFFF2304F58670C0
:10DB9800A5F80C31C5F8084185F8047103F04EF872
:10DBA80004F58A7003F004F83846FDF72DFE0446A4
:10DBB800002839D096F9051098F84800012201F09C
:10DBC800E8F988F83900D5F894343361002C71D01D
:10DBD80000F0F0FC002888D195F8913485F81A04F3
:10DBE80060F3820385F891347FE7B8F1010F4FF0B5
:10DBF8000204E8D1DFF8D0908DF8144099F8480075
:10DC080089F81D7102A901F065F9337989F8303175
:10DC18008DF805708DF80680FDF7C4FC95F89134F1
:10DC280043F0100385F891340024CCE700226946BC
:10DC3800022000F0F3FA0028F6D01324C3E7244B9F
:10DC4800B288DB6B96F90C10B0689847D5F840336A
:10DC580043F00203C5F84033E6E702A90D2000F0BF
:10DC680053FB0028E0D0002269460D20E1E7164B5F
:10DC780093F81831D3B9347904F0070000F0ABFAFF
:10DC88008DF80040012269461020D2E7002269463B
:10DC98001220CEE78DF8072000F08EFA044638B936
:10DCA80000F087FA204600F089FABDE702248AE7E7
:10DCB800012488E701A800F0D1FB16E7032414E744
:10DCC80040210020EC1C002028170020EE1C00201A
:10DCD8009C4301082DE9F04F99B08046059118B989
:10DCE800032019B0BDE8F08F00230361FEF742FC62
:10DCF8000446002840F0A58046460FCE0EAD0FC55D
:10DD08001422524898F800A0B8F80C7098F90EB090
:10DD18004F4E214603F07EF84E4B012283F84124F2
:10DD280096F83021022A25460BD196F81821022AA6
:10DD380007D196F81E2122B9BAF1010F38BF4FF06A
:10DD4800010ABAF1010F2BD0BAF1030F2AD0BAF1A8
:10DD5800000F33D102229DF83C30DDF84090029349
:10DD680062F34715012496F87C108DF832100222D0
:10DD78000CA996F848008DF8302001F09DF896F827
:10DD88001A3196F830C196F81D1140B2002B63D0B5
:10DD9800BCF1010F57D1002955D1002C61D153E0B6
:10DDA8000422D8E70023DDF83C90BDF840709DF9C7
:10DDB80042B0029365F01F050124D4E74FF0000B31
:10DDC800D946CDF808B0CEE74FF0010084F81A0420
:10DDD800D2E005F29A420BA900F0D4FA002800F02C
:10DDE80015811320049B33871A4B002283F81A24C9
:10DDF80023E105F29A452A460BA900F0C3FA002848
:10DE0800EFD10B9B84F82801C4F82C5184F83031E9
:10DE1800FCE0B9F1000F00F0F980002A00F0F6806C
:10DE28004946E01C02F0E2FF94F8373201332380C0
:10DE3800ECE01220D6E70220D4E70720D4E713202D
:10DE4800D2E701204DE7FCB90220F6E02C210020A2
:10DE580028170020EC1C0020002CF5D05845B8BF2E
:10DE6800584696F87C308DF82000052296F8480030
:10DE78008DF8223008A901F032F800283FF430AFBD
:10DE88009DF8203086F839306F4A704BD2F89804E4
:10DE9800D3F8904038B105F087FA6C4B84423CBF08
:10DEA800002283F83A20198F1A8F93F830010491D1
:10DEB800996A099152BA0028BFD093F81B0100B99A
:10DEC800186393F81801ADF85820013893F87C20AE
:10DED80093F81A411491D0F1000BD3F888108DF8FB
:10DEE8005B204BEB000B93F8482093F83A0093F82B
:10DEF80068308DF85A3009AB0093554B03904FF0BA
:10DF080001008DF84C0015918DF85C20A3F12F01CC
:10DF1800A3F1300213A88DF84D4000F0DBF8039B05
:10DF28004FEA0B1B4BEA431B00264BEA801B4BEACC
:10DF3800C413B145444C039308BF37463A46494693
:10DF480004F59C70CDE90A669B46268084F81A641D
:10DF580002F04CFFE9B2A570C5F34215FAB2042DE0
:10DF68003A4E039B84F837223FF42EAF072D3FF437
:10DF780050AF022D7FF45FAF364D84F80D110420A9
:10DF8800029984F80401FF2084F80C0184F8281110
:10DF980084F81431D6F8E410C4F8085105F59B73D9
:10DFA8000AA8C4F8101184F83021C4F82C3100F004
:10DFB80011FC00287FF43DAF0A9BA4F844040BA889
:10DFC800A4F81631C4F84C3400F0D0F900287FF4D6
:10DFD80008AF0B9BD3B196F93900FDF7F7FA94F81F
:10DFE8003732002B3FF405AF0B9B0F2B3FF6F1AEFA
:10DFF80005F58B720BA90F2000F0C4F900287FF4F7
:10E00800F0AE0B9B63F3030B84F814B10598FDF78E
:10E01800FBFB00287FF4E6AE099B86F83A00B36262
:10E0280000F080F900287FF40AAF94F8913484F85E
:10E0380040A443F0010384F89134034BD3F894349B
:10E04800C8F810304DE600BFEC1C0020281700204F
:10E0580090170020EE1C002037B50B4D8DF80400FA
:10E0680004460F2295F8480001A900F038FF40B196
:10E07800064A85F81C4192F8913443F0200382F84F
:10E08800913403B030BD00BF28170020EC1C0020DD
:10E0980010B5FFF7C1F8044688B90A4805F0BEF97B
:10E0A800094805F0BBF9094805F0B8F900F094F8FB
:10E0B800FDF7BCFD064BDB6A9847204610BD0124DE
:10E0C800FBE700BF542000206C20002084200020A3
:10E0D8009C4301082DE9F04F8BB047780093149BBF
:10E0E80090F90C8090F90D6090F80EB08A4641685E
:10E0F800196004469146002F58D002238DF810303D
:10E1080004A9C37B007C8DF8123000F0D5FEB4F86A
:10E1180008C0618943B26068984545466144B8BF04
:10E128001D46604534BF00270127884209D30A21CC
:10E138008DF81010207C019304A900F0BDFE019B0E
:10E1480046B2B4F808C0608961680CEB400E7145AE
:10E1580019D3A1EB0C01B1FBF0FC00FB1C1191B928
:10E16800984503DC2378CBB94FF0010B21238DF8B8
:10E178001030207CE37B8DF8115004A98DF8123003
:10E1880000F09AFE45B2009B8AF80050384689F89C
:10E19800006083F800B00BB0BDE8F08F0223207C4C
:10E1A8008DF8243006A900F095FEDDE74546EAE73C
:10E1B8007047704770477047002070477047704736
:10E1C80070470020704700207047002070470020EB
:10E1D80070470020704770477047704702207047AB
:10E1E8000220704702207047704700207047704730
:10E1F800704700207047002070477047704770478D
:10E2080010B5054C4FF403722046002102F002FEBF
:10E218000020C4E9000010BD082200202DE9F843C1
:10E228008146904600293CD01F4C2023224604F109
:10E23800100012F8017F6FBB8242FAD11B4E33687F
:10E24800013403B93460736803B11C60002525608C
:10E25800C4F8088074601FFA88F284F80490601D7E
:10E2680002F0C4FDB9F1110F4FF0000398BF104D33
:10E278006373D6F8083298BF25FA09F503F101034C
:10E2880098BF05F0010543442573C6F8083238469F
:10E29800BDE8F883013B13F0FF030446C6D102270B
:10E2A800F5E70127F3E700BF0F220020082200202E
:10E2B8002007020010B518B3124A1368984204D117
:10E2C80003681360002305E00B46002BFAD0196899
:10E2D8008842F9D15168884208BF53600BB1016880
:10E2E8001960D2F808328168013B00245B1A046087
:10E2F8002146C2F80832102202F08CFD204610BDDB
:10E308000120FCE708220020054B1B6813B11A798D
:10E318008242FAD1002B0B600CBF0320002070470B
:10E328000822002010B5054B186800B910BD037B02
:10E3380004680BB9FFF7BEFF2046F6E70822002065
:10E3480038B5084B084C186800B938BD037905681A
:10E35800112B05D824FA03F3DB0701D5FFF7AAFF31
:10E368002846F1E7082200202007020028B1044BC4
:10E37800D3F808320360002070470120704700BFBF
:10E38800082200202DE9F04107460E46154642B303
:10E3980039B3154B1C6800232CB93046FFF7E6FF4C
:10E3A8000020BDE8F081A268F91A0132914215D324
:10E3B8002279EA54581C22895FFA80F8611D55FABF
:10E3C80080F002F013FDA368246898445FFA88F38C
:10E3D800E2E720462568FFF76DFF2C46002CF8D1B0
:10E3E800DBE70120DDE700BF082200200238C0B2C9
:10E3F80011289ABF014B185C00207047B33C0108F4
:10E4080030B50B4B93F820200446084672B1002122
:10E418001C330578A54208D001319842CDB214BF0B
:10E4280004301038AA42F4D8002030BD1046FCE76A
:10E438001424002010B5084C00232060142204F195
:10E448000C00FF2184F82030C4E9010002F0E2FC4E
:10E45800012384F8213010BD1424002010B50E4A81
:10E4680092F82010042915D8936804781C70447811
:10E478005C70C478807898700131DC7082F8201064
:10E4880002F11C018B4214BF043302F10C039360A8
:10E49800012010BD0020FCE714240020094B93F84C
:10E4A800200068B15A6803F11C018A4200F1FF306C
:10E4B80014BF043203F10C0283F820005A600120D3
:10E4C800704700BF1424002010B5074B93F8202094
:10E4D8000446084632B15968FFF792FF10B101238C
:10E4E8004470837010BD00BF1424002008B5064B8B
:10E4F80093F820202AB15968FFF782FF08B14078C5
:10E5080008BD0120FCE700BF1424002030B50A4AEA
:10E5180092F82010536882F8210061B191680124B3
:10E528001C32DD78587005B99C70934214BF0433CF
:10E53800103B9942F5D130BD1424002008B5044B96
:10E548005968FFF75DFF003818BF012008BD00BFFC
:10E5580014240020F7B50422154E044600210DEBC3
:10E56800020096F8207002F055FC0025EBB29F429D
:10E5780001D803B0F0BD7368197821705A786270B9
:10E58800987838B1336820469B689847FFF786FF2C
:10E598000135EBE7DB788DF804108DF805208DF850
:10E5A8000730FFF77BFF01A8FFF758FFF0E700BF30
:10E5B80014240020014B93F82000704714240020F5
:10E5C800034B93F82000042894BF002001207047D3
:10E5D800142400201FB50024CDE90244C41F8DF87F
:10E5E80000408DF801100C0AADF80420090C120C3B
:10E5F8008DF803108DF806208DF8073002461B0AA7
:10E60800012168468DF802408DF8083002F05DFA65
:10E61800002818BF0E2004B010BD2DE9F04188B0C5
:10E6280090460D460F9A0746002847D0002401213E
:10E63800CDE904448DF810109DF838108DF81510A8
:10E64800ADF81630190CCDE900441B0ECDE9024493
:10E658008DF81930ADF81A20130C120E07948DF8A6
:10E6680018108DF81C308DF81D20E3B21E01002D06
:10E67800F6B203DC002008B0BDE8F08101331021B8
:10E688008DF81F3042466B460DEB010002F0B3F9DE
:10E698000346A8B9102D28463E44A8BF1020694655
:10E6A800327811F801CB013382EA0C02984206F85D
:10E6B800012BF5DC103D2DB20134D6E70920DAE74D
:10E6C8000E20D8E70138032815D8DFE800F0020843
:10E6D8000C100A4B1B681B690B6000207047074B26
:10E6E8001B685B69F8E7054B1B689B69F4E7034BFC
:10E6F8001B68DB69F0E70520704700BF382400205D
:10E708002DE9F041C4B00C464A9E17461D46804686
:10E71800B8B3B1F5807F36D84FF4887200216846C7
:10E7280002F078FB492300934FF48073ADF804306E
:10E738002B0C8DF80830330CADF80650ADF80A6094
:10E748008DF80C3022460023414604A82D0E360EC3
:10E758008DF80E308DF809508DF80D608DF80F404A
:10E7680002F044FB04F110014B9A3B4689B268461B
:10E7780002F02BF910B1012818BF0E2044B0BDE8F3
:10E78800F0810920FAE70D20F8E7000010B590B1F4
:10E798000A4C28220021206002F03CFB2368084A2A
:10E7A8001A6000204FF0FF32C3E90302C3E90522D3
:10E7B800C3E9072210BD0820FCE700BF3824002069
:10E7C80000010101024B1B6818600020704700BF60
:10E7D8003824002030B1044B1B68DB680133036028
:10E7E80000207047092070473824002013B5002303
:10E7F8000C460193CAB101A9FFF764FF18B9019B40
:10E80800591C02D1146002B010BD99B2611A0029D6
:10E8180001DD5C18F6E702D113600720F3E71B0C53
:10E828001B0403F580331C44ECE70920EBE70000E8
:10E8380028B1044B1B681C33436200207047092031
:10E84800704700BF382400201FB5044600B30023DA
:10E8580003A8039302F090F9104ABDF80C3012682F
:10E8680020469380E38200F05EFA98B904F1180319
:10E87800009321680123132202F09CF860B9204616
:10E8880000F051FA003818BF0120000104B010BD93
:10E898000920FBE71020F9E70E20F7E738240020CD
:10E8A800F0B5054687B01C4613B9092007B0F0BD7E
:10E8B8002E4E3368DB68834255D894F82020002A0E
:10E8C8000CBF08220922834205D3204600F05FFAD4
:10E8D80068B11020EAE7002301900093A36894F838
:10E8E8002810606AFFF799FE0028EED0DEE723794A
:10E8F8002168B4F808C0A768043B9AB20029D4D0AC
:10E90800B2F5807F2DD8ADF80EC08DF817304FEADC
:10E91800174C04F12C033F0E8DF8117000932F0C47
:10E9280008234FF0490EADF80C008DF814708DF8DF
:10E9380016002F0E0DEB0300CDF808E08DF810C07F
:10E94800ADF812508DF8157002F034F808B10E20A9
:10E95800ACE7204600F01BFA0028BAD13368DD6026
:10E96800A4E70D20A2E70620A0E700BF3824002076
:10E978002DE9FF410A9D80460F4616461C46002D8C
:10E988005AD0002303A910460393FFF79BFE18B142
:10E99800062004B0BDE8F081039B9C4201D80133F6
:10E9A800F6D1284600F064F9002847D1264B1A789A
:10E9B800424503D01A79424542D10120AA68BA4299
:10E9C80040D103EB8002EB6A92F801802979CDE906
:10E9D80000430439927828683B4689B2FFF790FED5
:10E9E8000028D6D195F820300194002B4FF0010370
:10E9F800009314BF4246082295F82810686A3B46DF
:10EA0800FFF70BFE0028C4D1013E032EC1D8DFE872
:10EA180006F002070B0F0D4B1B681C611C62B8E760
:10EA28000A4B1B685C61F9E7084B1B689C61F5E7BA
:10EA3800064B1B68DC61ACE70920AAE70F20A8E7B2
:10EA48000B20A6E70220A4E7A40800203824002011
:10EA58001FB50B294FF00003CDE90033CDE9023390
:10EA68000A4607D00C2914D00A2910D00A2005B06C
:10EA78005DF804FB012802D120238DF80030002125
:10EA8800684602F022F8002818BF0E20EFE730236E
:10EA9800F3E70B21F4E7000038B5054602F010F85B
:10EAA800044610B10E24204638BD002DFBD1094B79
:10EAB8001B680B219878FFF7CBFF0028F2D10C21B7
:10EAC800FFF7C6FF0028EDD10A21FFF7C1FF002894
:10EAD800E9D0E7E7382400202DE9F04380468FB0DD
:10EAE8000C461746002A6BD0002969D00025294614
:10EAF8001D2206A8059504F0A7FE8DF81350344D85
:10EB08002B680DF114099E88CDF804900DF11303BC
:10EB180002933B7900933B6832462146404601F018
:10EB2800F0FF00284ED138683A79494602F05EF97C
:10EB3800384600F04FF8002846D13C7AFA79BB797C
:10EB4800240444EA02241C432B689A6894423DD961
:10EB58009C609DF813000B21FFF77AFF034658BB12
:10EB68000C21FFF775FF034630BB0A21FFF770FF42
:10EB7800034608BB7B7ABA7AFF7A3F0447EA022742
:10EB88001F433A46334621460920FFF723FD034633
:10EB980090B933463A4621460820FFF71BFD034645
:10EBA80050B92A689DF8131091700021D1604FF078
:10EBB800FF31C2E90411916118460FB0BDE8F08336
:10EBC8000923F9E70E23F7E70F23F5E70323F3E714
:10EBD8003824002010B50446002845D001680029D3
:10EBE80042D011F8013B43710322063002F0FEF8CF
:10EBF8002046032250F8091B043102F0F7F8216877
:10EC0800CB79E3600A7A43EA0223E3604A7A43EA6B
:10EC18000243E3608A7A43EA0263E360CB7A2374AF
:10EC28000B7B63742379212B1AD110220D3104F147
:10EC3800120002F0DBF81D222168501C8B5C636215
:10EC4800085C43EA0023901C6362085C033243EAD1
:10EC5800004363628A5C43EA02636362002010BD7A
:10EC6800112B03DC0D22E7E70220F8E70120F6E785
:10EC780010B50446002854D00168002951D00B78FB
:10EC880043714B7883608A7843EA02238360CA78A9
:10EC980043EA024383600A7943EA026383604B795B
:10ECA80003738B79C381CA7943EA0223027BC38148
:10ECB80002F00F020831103002F098F8237B00228E
:10ECC80003F00F0384F8202084F82820227903F128
:10ECD8000800111A04290DDD21680933043AD21AF3
:10ECE800085C84F82000D2B2606A84F828201944AD
:10ECF80002F07CF8237922681A44002012F8043CB8
:10ED0800E36212F8031C43EA0123E36212F8021CCF
:10ED180043EA0143E36212F8012C43EA0263E36227
:10ED280010BD0220FCE710B5044660B3036853B376
:10ED38000279162A29D942791A700146082251F80F
:10ED4800060B013002F05CF82146082251F80E0B40
:10ED5800093002F055F82368E28A5A74E38A226877
:10ED68001B0A93742368A269DA74A36922681B0AD0
:10ED780013752368628B5A752368E27E9A75172388
:10ED88002371002010BD0120FCE70220FAE738B506
:10ED98000446002863D00168002960D0037B90F8FE
:10EDA800282003F00F03002A57D1083320790432B2
:10EDB8001344984255D363790B702368A2685A703C
:10EDC800A36822681B0A937023686289DA70236833
:10EDD800E27A1A712368227B5A712368E2899A7150
:10EDE800E38922681B0A2146D371227B51F8100B54
:10EDF80002F00F02083001F0F9FF237B94F8282075
:10EE080003F00F0303F108052AB1226894F82010D3
:10EE1800515503F10905206894F82820616A2844AF
:10EE280001F0E4FF94F828302268E16A2B44D154B9
:10EE38005A1CE16A206892B2090A81549A1C216816
:10EE4800E08D92B28854DA1C216894F82F0092B2AF
:10EE5800043388542371002038BD0933A6E7012004
:10EE6800FAE70220F8E70000024B1A8810431880DE
:10EE7800704700BF3C24002008B5074B1B883BB1F6
:10EE8800FEF7CAF9002814BF6FF00200002008BD81
:10EE98006FF00100FBE700BF3C24002010B5034BD6
:10EEA80000241C80FEF7AEF9204610BD3C2400204B
:10EEB800B0FA80F04009704782B018B9084602B02D
:10EEC80000F0CAB8002002B0704710B9084600F038
:10EED80077B9704710B9084600F08EB970470346F5
:10EEE800084611460BB900F0E5B90020704710B983
:10EEF800084600F06DBD704710B9084600F006BA24
:10EF08000020704710B40446084611461A46019B73
:10EF180014B910BC00F014BA10BC70470346084678
:10EF280011460BB900F03EBA0020704710B40446F1
:10EF3800084611461A4614B910BC00F0ABBA0020B6
:10EF480010BC704730B40546084611461A46DDE93C
:10EF580002341DB9029430BC00F02ABB002030BC3A
:10EF6800704710B9084600F0DBBB0020704710B9A5
:10EF7800084600F06BBD0020704710B9084600F045
:10EF8800EABB0020704710B9084600F0E7BB002034
:10EF980070470346084611460BB900F001BC002033
:10EFA800704710B40446084611461A46019B14B926
:10EFB80010BC00F0F7BB092010BC704710B4044621
:10EFC800084611461A4614B910BC00F061BDC8B213
:10EFD80010BC70470048704701000102064B10B58D
:10EFE8001B6A0446984730B10448054B20449842B0
:10EFF8008CBF0020012010BD9C43010840C220C9DD
:10F0080080B92A00F0B5114B85B00C4610491F563F
:10F01800054601F04BF80F4BE4B25E6A072D4FF03E
:10F028000103CDE9024301460AD105220023CDE9B7
:10F0380000234FF47A727A431846B04705B0F0BD02
:10F0480008220020CDE900203A46F5E7803D010876
:10F05800603D01089C4301081FB500230093037815
:10F06800013B372B21D8DFE803F01C242020201E89
:10F07800202020204143454E2055585B5E61642086
:10F088006C1E6E73787A20207D8126202020202017
:10F09800202020202020202083858A2020838A2069
:10F0A8008C90C3780BB102230093009805B05DF8EB
:10F0B80004FB8378F6E743788DF8043005238DF850
:10F0C80005308378003B18BF01235B008DF80630BC
:10F0D80010238DF80730304B1B6801A803F55872D0
:10F0E800CDE9022300F0C2FF0090DEE74023DBE712
:10F0F8002023D9E7827890F9013012B9274AD35CE6
:10F10800D2E7274AFBE7827890F90130002AF8D144
:10F11800244AF4E740F6B833C6E74FF47A73C3E7F6
:10F128004FF4FA63C0E741F28833BDE741F27073E8
:10F13800BAE71D484FF47A7101F03CFE00F5FA6019
:10F14800D2E71A4BB0E7144B1B6803F55873ABE7CB
:10F15800114B1B6803F55B73A6E71023A4E70E4B5E
:10F168001B68A1E74FF0834300939EE7104BFBE732
:10F17800104B99E740F21113ADF8003095E70323DF
:10F1880092E790F901300C4AB9E70C4990F901006F
:10F1980000F08CFFA8E700BF44240020553D01087B
:10F1A800453D01084D3D010818FCFFFF00EA063700
:10F1B8009A99094040F70937803D0108603D0108E8
:10F1C80037B50B4B02781B680C2101FB02335B7AC5
:10F1D80003EB4304074B1D6803690093C368427837
:10F1E800816805EBC40000F0DDFC03B030BD00BF52
:10F1F800442400204024002070B586B0027B64239C
:10F20800ADF80030012A4FF00003CDE90133CDE914
:10F2180003338DF802308DF8143030D0022A39D0FB
:10F228005ABB03684BB343683BB31F4D80682B60E0
:10F238001E4B18226946186001F0D8FD1C4B2C683B
:10F2480093E807000C3384E8070093E8070004F10B
:10F258000C06032386E80700A4F86C33012204F5A2
:10F268005B7104F5587000F08EFC2B684FF6B07295
:10F27800A3F878230522C3F87C2306B070BD0A4999
:10F2880008684360036100F55B7100F5587000F091
:10F298007AFCF2E7044B1B68B3F86023B3F86C13ED
:10F2A8000A43A3F86023E8E7442400204024002010
:10F2B800383A010808B503460A2924D8DFE801F0DE
:10F2C80006232323230B161B23212100BDE8084016
:10F2D8000068FFF783BE90F900009978052271B99C
:10F2E80000F011FC003818BF012008BD052293F971
:10F2F80000000021F4E790F900005978EEE70221B8
:10F30800EEE70722F3E70020EFE7000008B50279EF
:10F318001AB1012A0BD0002008BD084B01681B68F0
:10F32800012203F5587000F02EFC0120F4E7034B8E
:10F3380001681B6803F55B70F5E700BF44240020F3
:10F34800F7B50528144D1C46A8BF052058700E4671
:10F358002946174600F0AAFE94F90130A070072B41
:10F3680013D1322000F0A2FD0C4BDB6D0546984707
:10F3780004F10C0208340346019200943A463146DF
:10F38800284600F098FD03B0F0BD054A55F8231053
:10F39800D05C00F083FDE7E7603D01089C4301086D
:10F3A800803D01082DE9F04F344F90F901607B68EA
:10F3B800D0F804908BB00446884698470546002844
:10F3C80059D1E37C73B92E4A2378126803EB4303BF
:10F3D800990002EB8303D3F80490B9F1000F01D12F
:10F3E80052F80190274B484613F906B0FB68984736
:10F3F800A37C2289D7F818A00993072E28D10023C7
:10F408000121CDE90223204A0693CDE90431CDE953
:10F4180007330521CDE900214FF47A7202FB0BF284
:10F428004CF250311846D047637C13B3174B995DA3
:10F438007B6D0D31C9B228469847E07C3246494673
:10F4480000F046FE88F8006001200BB0BDE8F08FA0
:10F45800002101250823CDE90013CDE90715CDE9E1
:10F468000511CDE903110292A1782B465A46284688
:10F47800D9E7074BDBE70020E7E700BF9C4301081B
:10F4880044240020803D0108854501004D3D0108C8
:10F49800553D01082DE9F04F8DB090F90130DFF8A6
:10F4A800FCA0DFF8FC90CDE90A123E4A12F903B03D
:10F4B8000278DAF800300C2505FB02333A4A5B7A09
:10F4C800126803EB430302EBC303044693F90210EB
:10F4D80090F9020000F0E5FD3449064694F9010070
:10F4E80000F0E4FDA26861688046304600F00BFD3C
:10F4F8002178DAF80020D9F80C30694307465058CB
:10F508009847D9F81C309C4694F901300025072B00
:10F518004FF47A63CDE90753CDE905552DD1012381
:10F52800CDE903530523CDE901534FF47A7303FB67
:10F538000BF300933946434646F2A812284667461D
:10F54800B8472378DAF800200C214B4394F90110CE
:10F55800D05800F0DFFDA18994F90100FFF752FDB2
:10F568000B9B217B1860D9F85430284698470A9B92
:10F5780001201E700DB0BDE8F08F01200823CDE9F1
:10F588000350CDE901032A46CDF800B0654643464D
:10F598003946A84701200546D3E700BF4424002088
:10F5A8009C430108803D010840240020603D01087B
:10F5B8002DE9F04F8FB0002405468A4691469846BB
:10F5C8000494ADF81440ADF8024007264FF0010B43
:10F5D8002B7AA34206D9686804A9204400F0F6FBF8
:10F5E80000285ED102238DF8083002A86B7A8DF8C6
:10F5F8000A30FFF731FDAB7A8DF81D309DF81130D8
:10F608008DF81E309DF812308DF81F309DF810309F
:10F618008DF82030EB7A8DF821302B7B8DF8223055
:10F628006B7B8DF8233010238DF81C608DF8243007
:10F638003A4E8DF82C000DF102030A9305238DF83C
:10F648002D3033680C930723ADF834302B680693BC
:10F658000DF1120204AB0DF1110106A800F0D0FB68
:10F66800072805460BD130680C22002100F5587098
:10F6780001F0D0FB3368BDF80220A3F860239DF8A1
:10F6880011308AF800309DF8123089F800309DF862
:10F69800103088F80030189B28461C700FB0BDE861
:10F6A800F08F9DF81330BDF81470ADF80270204447
:10F6B800C4B2F3B917B3194A0020116807260246E5
:10F6C8004FF00C0C062B1BD10CFB00FE51F80EE082
:10F6D800BEF1000F04D00BFA00F23A4397B20122B0
:10F6E80001301028EED1002A3FF472AFADF8027055
:10F6F8006EE75A1E042A01D9062BDCD0062667E7D6
:10F7080047FA00FE1EF0010FEAD00CFB00FE51F88C
:10F718000EE0BEF1000F08BF0626E1E744240020F2
:10F7280038B505464068FFF759FC0522841D0021BD
:10F7380095F90000E4B200F0E6F908B904F0FD0418
:10F7480095F901000722002100F0DDF908B904F05D
:10F75800FB04204638BD00207047000010B5037830
:10F768000F2B044618D84068FFF738FC22780B495D
:10F7780002EB42020968831C01EB820051F8222047
:10F78800DBB21AB903F0FD0358B210BD032B06BF54
:10F79800626842600223F7E70020F6E7442400206D
:10F7A800022070472DE9F04FDFF838810446D8F879
:10F7B800000099B08946174600211E4601220323FE
:10F7C80000F55870CDE90611CDE908118DF814102F
:10F7D8008DF81510ADF8163000F0B7F938B9D8F82B
:10F7E8000020B2F8603343F00303A2F86033D8F87E
:10F7F8000020637A8DF8283002F55871CDE90B1294
:10F80800394A94F9083012680D920DF116020F92D8
:10F818002268109262681192D4E90301A27A8DF8E5
:10F82800482001228DF8492013AA82E803001025F8
:10F83800227DE18A8DF8293018468DF85420ADF8DC
:10F848003850FFF7DFFB0AAB17930DF1150316903D
:10F8580000933146019705AB06AA10A800F0C2FB39
:10F86800064698BB9DF81410204F013901F0A2FA02
:10F878001F4B1B690393C4B24FF00C0B04F16003D8
:10F888006B44D8F8000013F848AC9DF814300BFB13
:10F898000AFC01343946B4FBF3F203FB1244D0F8F6
:10F8A8007C33B0F9782350F80C00DDF80CC0E4B2D2
:10F8B800E04728B189F800A0304619B0BDE8F08FBC
:10F8C800013D15F0FF05D9D10D26F5E70C2801BF3C
:10F8D800D8F80020B2F8603343F00303A2F860338D
:10F8E800EAE700BF4424002040240020400D030024
:10F8F8009C430108F8B50679012E054648D90F2E14
:10F9080048D80368187A40F303000522002140B262
:10F9180000F0F9F82B680446187A40F30310052222
:10F92800002140B200F0EFF8B8B1B4FA84F46409E9
:10F9380029680B7A086843F3030243F303135BB2A5
:10F9480052B29A42C8BF0124FFF748FB80F0010376
:10F95800DBB224B10533D8B2F8BD0124E8E7DBB93E
:10F968000E4F29683B6806EB460003EB80000C222B
:10F9780001F03CFA3A680C2303FB062320465C722C
:10F98800B2F860130123B3400B43A2F86033E3E7F6
:10F998000620E1E70320DFE70420DDE74424002018
:10F9A80010B4017801290ED9084B18680C234B4371
:10F9B800C4180022C250C4E9012200F5587010BCD6
:10F9C800102200F0A9B8002010BC70474424002081
:10F9D8002DE9F04186B050238DF81430037A102BAE
:10F9E800074630D14368DD7B6DBB0224A8466426F8
:10F9F800062C14D87A68535D03932A44517843EA55
:10FA080001230393927843EA02437343CDE9033811
:10FA180063B968468DF80040FFF7C2FF0DE0CDF8E6
:10FA28000C808DF81480CDF81080F2E703AB01A8A4
:10FA380001938DF80840FFF75DFF0134E4B2102C04
:10FA480005F10305D4D106B0BDE8F0811FB5026801
:10FA58000379116849B901A88DF80430FFF7A0FFB0
:10FA680078B1032005B05DF804FB02A802928DF876
:10FA78000C30FFF73FFF042805D0052805D00028E3
:10FA8800EFD00020EEE70220ECE70120EAE70000D3
:10FA9800C90020B9034B0B449856C0B27047024BBB
:10FAA800F9E700BF053D0108C53C0108F0B59A42D9
:10FAB800069D03DB9DF914309A4220DD0020F0BD3D
:10FAC80003EB430331F814C005EB830300264CFA1B
:10FAD80006F7FF0707D51F7A07F00F0E964502DCD9
:10FAE800B2EB171F0DDD0136102E03F10C03EED11A
:10FAF8000134E4B22301DBB29842E1D8DEE7002406
:10FB0800F8E70120DBE7884204DB9042CCBF002005
:10FB1800012070470020704710B51409B4EB111F7D
:10FB280003464FEA11100ED391420CD202B201F0F3
:10FB38000F0133F81240012000FA01F124EA010113
:10FB480023F8121010BD0020FCE7F0B528B100EB37
:10FB5800410501270020914200D3F0BD002435F86B
:10FB680002CB234607FA04F636EA0C0608BF01332F
:10FB780004F1010408BFDBB2102CF3D118440131A1
:10FB8800C0B2C9B2E7E710B500B149B910BD31F844
:10FB9800134020F813400133DCB2A242F7D8F5E74E
:10FBA8000023F9E782B030B504880493D2B9B3F5DD
:10FBB800616F15D349F6AF2542F21072AB4298BF78
:10FBC8004FF47A72944238BF14466143BDE830401E
:10FBD800C3688B428CBF5B1A0023C36002B07047B6
:10FBE8006422EFE7012C38BF0124EEE72DE9F04F3E
:10FBF8008FB01546199F03939DF8603007930C4604
:10FC0800804603F0C7FB6A4A0590A7F5F633303BF8
:10FC1800B3FBF2F3534303F5F63B0493182313FBAA
:10FC280005430BF1300B069300254FF0FF3A069B76
:10FC38009C4207D1002D14BF50464FF0FF300FB043
:10FC4800BDE8F08FBDF96830ADF8243009991997EF
:10FC58003846089703F02EFB2688B8F1000F5FD1CD
:10FC6800B7F5616F5AD349F6AF2242F21073974243
:10FC780098BF4FF47A739E4238BF1E46642E59D1FE
:10FC8800DFF83091A060A1680CA803F035FB0D9B4C
:10FC98000093DDE908120C9B0AA803F08CFA039A7A
:10FCA8000A9B0AB9079A2AB122694A4502D1424AEF
:10FCB80093420ED9414BC4F80C909F4209D90023B6
:10FCC800ADF82C300B99CDF828B0584603F0F2FA6D
:10FCD800A060606808B9C4F80C90C4F81090B8F136
:10FCE800000F04D003F060FBE3680344E360D4E949
:10FCF80003329342059B88BFE26063601B9BE16807
:10FD08007343994204D20398E8B9B8F1000F1AD0A6
:10FD180001231D442375EDB2183488E76423AAE74C
:10FD2800039B0BB9234BE360012EDFF8889038BFA3
:10FD38000126CEE7B6F57A7F0ABFDFF88490DFF8B0
:10FD48008490A0609FE700209342207506D85B1A34
:10FD58009A4505F1010528BF9A46EDB2B8F1000FA2
:10FD6800DAD1642E184AADF82C801DD049F6B0239C
:10FD7800B6F57A7F18BF1346974281BF049A02F5F9
:10FD8800A83202F5C0729B180A931A9B00930AAE18
:10FD980096E80600199B304603F00DFA96E8030032
:10FDA80003F088FA8246B7E74FF46163E4E700BFDF
:10FDB8008051010040771B007F5101002FEC0100AA
:10FDC80080A81201002E930230EC01000378032B67
:10FDD80014D1437803F00F021B098A704B708378A3
:10FDE8008B80C27843EA02238B800379C3F3021223
:10FDF80003F00F03CA700B7005207047002070478E
:10FE08002DE9F3479A464379057990F907609146B9
:10FE1800044690F906208846D3B190F90870002D61
:10FE280037D00F2A1BD194F909200F2E27D194F926
:10FE38000A00072D02D1002F08BF012788F80020EB
:10FE480089F8000028468AF8007002B0BDE8F087FB
:10FE580090F90B7090F9092090F90A60DFE7A3691F
:10FE6800019394F91530009394F914302169207B9B
:10FE7800FFF71CFE0028D8D105F0FD05D5E794F959
:10FE88001D00B042D5DC94F91C30B34203DA05F00A
:10FE9800FB053046D2E73046CBE70000024B03FAB9
:10FEA80000F0B0FBF1F0704740420F004FF4FA53F6
:10FEB800B3FBF0F0704730B54FF47A750C1F6A4306
:10FEC80000FB042252001EBF00F1FF341219B2FBDE
:10FED800F0F2914238BF1146039A116082004843FC
:10FEE8001CBF013040084FF47A71121A01FB13232A
:10FEF800002BCABF03F2E73393FBF1F1B3FBF1F137
:10FF0800049B196030BD38B5400014460D46F1F722
:10FF18007DFD01462846F1F7C7FC2146F1F7C4FCF0
:10FF2800F1F7B6FB03F0DCFCF1F792FC40B238BD08
:10FF38002DE9F74F019300239C469E46048A1E0133
:10FF4800F6B2B44246D906EB46054FEA4309AD007E
:10FF58000024476837F809702741FF0729D58768C3
:10FF680007EB050A7F5927B3077837B9476927B1DF
:10FF780037F809702741FF071BD59AF8087090F9E0
:10FF880001B047F303084FFA88F8D84511DC47F366
:10FF980003177FB25F450CDB9AF8097007EB470837
:10FFA800C76807EBC8073F7D5FB90CF1010C5FFA22
:10FFB8008CFC0134102C05F10C05CAD10133DBB2DD
:10FFC800BCE70EF1010706EB040801F80E805FFAA2
:10FFD80087FEEEE7019B82F800E083F800C003B0DB
:10FFE800BDE8F08F2DE9FF4704464068DDE90C675E
:08FFF8001D468A46914603F004
:020000040801F1
:10000000D7F923681B1A3B604FF0000801233370B7
:1000100085F80080636813B12368834224D8D4F83C
:100020001CC0CAF80080A3699CF800E00393D4E9DF
:10003000030101AB83E80300237D0093DCF80C107F
:10004000237A627A7046FFF7D5FD334638602A4638
:10005000E0694946FFF770FF2B782BB1C7F80080A5
:10006000002004B0BDE8F0873378002B0CBF0C20D3
:100070000B20F6E737B590F9002090F90250954231
:1000800004460FD0013A52B295420BD0A3680193B7
:1000900094F9013000936168E0782B46FFF70AFD80
:1000A0000028EFD0104603B030BD8842B8BF0846E4
:1000B0007047000051F82000054B984205D0054BD1
:1000C000C31A58425841400070470120704700BF92
:1000D00090D0030020A1070005281FB50ED80C4BB7
:1000E00053F820300093CDE901120A4B0122002180
:1000F000022002F06BFE05B05DF804FBCDE90012B2
:10010000054B01220021022002F060FEF3E700BF50
:10011000F43D0108883D0108A73D010807B5054BDE
:10012000CDE9000101220021022002F04FFE03B0C0
:100130005DF804FBC33D010810B510220446002100
:10014000F13000F06BFE0021C4F814112046F022BB
:10015000BDE8104000F062BE02460846102100F0E3
:10016000A5B92DE9F0430446D0F8140185B00E4638
:10017000154604F2011988B3C0F1100890454746AE
:1001800028BF1746BAB2484400F034FED4F8143100
:100190003B440F2BC4F814312DD9A8452BD204F1C0
:1001A000F00304F5807113F8012F187C8B4282EA6A
:1001B00000021A70F7D104F1F10810224146684696
:1001C00000F018FE22466946684600F0F1F9102258
:1001D0006946404600F00EFE3E44ED1B04F5807873
:1001E00004F1F107102D09D8AAB23146484600F0B3
:1001F00001FEC4F8145105B0BDE8F08304F1F0032A
:10020000711E13F8012F11F8010F434582EA000215
:100210001A70F6D110223946684600F0EBFD2246EE
:100220006946684600F0C4F910226946384600F075
:10023000E1FD1036103DD5E7F0B589B00C4610222F
:1002400000210546684600F0E9FD224669466846F9
:1002500000F0AEF99DF90030002B6A464FF0000126
:1002600043DA137812F8010F01315B0043EAD0132F
:100270000F2902F8013CF4D19DF80F305B0083F0A8
:100280008703D4F81401DBB210288DF80F303BD16E
:1002900004F58073694604F5887013F8016F11F84E
:1002A000012B984282EA06021A70F6D104F1F0039B
:1002B00004F5807113F8012F187C8B4282EA00024A
:1002C0001A70F7D110220DEB020004F1F10100F0D9
:1002D00091FD2246294604A800F06AF91022002167
:1002E000684600F09BFD09B0F0BD137812F8010FCD
:1002F00001315B0043EAD0130F2902F8013CF4D12D
:100300009DF80F305B00BCE79DF90030002B6A467A
:100310004FF0000137DA137812F8016F01315B00FA
:1003200043EAD6130F2902F8013CF4D19DF80F30AF
:100330005B0083F08703471CDBB28DF80F30102F72
:1003400004EB0003C0F10F064FF0800288BF0026C7
:1003500000F5817083F801210021324620443E449B
:1003600003F076FAC4F8146104F58073694604F565
:10037000887013F8016F11F8012B984282EA060287
:100380001A70F6D192E7137812F8016F01315B0011
:1003900043EAD6130F2902F8013CF4D19DF80F303F
:1003A0005B00C8E70A780378534003704A784378C3
:1003B000534043708A78837853408370CA78C378F7
:1003C0005340C3700A790379534003714A794379E2
:1003D000534043718A79837953408371CA79C379D1
:1003E0005340C3710A7A037A534003724A7A437ABC
:1003F000534043728A7A837A53408372CA7AC37AAB
:100400005340C3720A7B037B534003734A7B437B95
:10041000534043738A7B837B53408373CA7BC37B84
:100420005340C373704710B50B7814786340037062
:1004300054784B786340437094788B786340837032
:10044000D478CB786340C37014790B79634003711F
:1004500054794B796340437194798B79634083710C
:10046000D479CB796340C371147A0B7A63400372F9
:10047000547A4B7A634043728B7A947A63408372E6
:10048000D47ACB7A6340C372147B0B7B63400373D3
:10049000547B4B7B63404373947B8B7B63408373C0
:1004A000CB7BD27B5340C37310BD0000A1F110037E
:1004B000DBB2102B2DE9F047044604D83A4820FA65
:1004C00003F3DB0705D4002382F8F030FF20BDE8FA
:1004D000F087561E254615F8013B06F8013F631BC1
:1004E0000B4413F0FF00F6D101F11C039B005FFAEF
:1004F00083FCC3F30313013BDFF8B09082F8F030C4
:10050000884653184FF0010EB8FBF1FA01FB1A8A26
:100510001AF0FF0A13F8047C13F8036C13F8025C5A
:1005200013F8014C30D119F806A019F8056019F834
:10053000045019F807404FEADE1707EB47078EEA29
:100540000A0A07EBC7074FEA4E0EFFB25FFA8EFEAC
:1005500087EA0E0E574692F800A087EA0A071F7036
:1005600057787E405E70967875409D70D57808F11A
:1005700004085FFA88F86C40C445DC7002F104029C
:1005800003F10403C0D8A2E71829E4D9BAF1100F87
:10059000E1D1DFF818A01AF807701AF806601AF807
:1005A00005501AF80440D6E7010101000C4001088B
:1005B0002DE9F04FA3B092F8F0301D911B920193FA
:1005C000002B00F0538101461EA8FFF72CFF1B9B58
:1005D000A74CA84DA84E10330293002303939DF817
:1005E0007C0004909DF886000590205C06909DF8A4
:1005F0007B000790205C089004989DF881C0205CE7
:10060000099014F80C000A909DF880000B909DF85A
:1006100085009DF878809DF87DE09DF882A09DF88A
:1006200087900C909DF87A00029B1C9314F80A2086
:1006300014F8093014F8081014F80E700D90205CAE
:100640000E909DF87F000F90205C10900B98205C1E
:1006500011900C98205C12909DF8840013909DF8E6
:10066000790014909DF87E001590205C16909DF8FE
:1006700083001790205C18901398205C19901498B0
:10068000205C1A900398013003900298DDF804B0C2
:10069000103002909DF80C00834536D88DF8781004
:1006A0008DF87A2009990E9A8DF87C108DF88220A9
:1006B0001199069A8DF880108DF87E201999169A56
:1006C0008DF884108DF886200A99189A8DF87D107F
:1006D0008DF887201299109A8DF87B301B9B8DF82E
:1006E00081108DF883201A99089A1D988DF885102D
:1006F0008DF87F201EA903EB0B128DF87970FFF7A0
:1007000092FE002023B0BDE8F08F15F808B082EA11
:1007100003008BEA000016F80EB080EA0B008DF89B
:10072000780015F80E004B40434016F80A0043408D
:100730008DF8793081EA070315F80A10594016F848
:100740000930594016F808308DF87A107A40534035
:1007500015F8092053408DF87B30089A069B5340CA
:10076000049AAA5C534016F80C2053408DF87C3054
:10077000DDE908325A4015F80C305340059AB25C56
:1007800053408DF87D30DDE909325A40059BEB5C22
:100790005340079AB25C53408DF87E30069B0A9A0C
:1007A0005340049AB25C5A40079BEB5C5A408DF868
:1007B0007F200E9B109A53400B9AAA5C53400C9AD0
:1007C000B25C53408DF88030DDE910325A400C9B0A
:1007D000EB5C53400D9AB25C53408DF88130DDE9FB
:1007E00011325A400D9BEB5C53400F9AB25C534060
:1007F0008DF88230129A0E9B53400B9AB25C5A408D
:100800000F9BEB5C1C995A408DF88320169B189A1D
:100810005340139AAA5C5340149AB25C53408DF82B
:100820008430DDE918325A40149BEB5C5340159A32
:10083000B25C53408DF88530DDE919325A40159B82
:10084000EB5C5340179AB25C53408DF886301A9A8D
:10085000169B5340139AB25C5340179AAA5C1EA889
:1008600053408DF88730FFF79DFDB8E6FF2049E73C
:100870000C4001080C3F01080C3E010808B538B1D6
:10088000044A05491060D82200F0B4FA002008BDDF
:100890000220FCE7482400203C4501080A4B1A6866
:1008A00070B5002302F1180503EB03142E5D864298
:1008B00004D1183422440A60002070BD01330B2B90
:1008C000F2D10320F9E700BF482400202DE9F041D0
:1008D000CCB00646DDF8488117461C460D4631B3BC
:1008E000B8F1000F23D006A8FFF726FC204601A987
:1008F000FFF7D4FF0446B0B9019906A80131FFF70C
:100900002BFC26B11022314606A8FFF72AFC3A46F6
:10091000294606A8FFF725FC06A902A8FFF78CFCCC
:10092000029BC8F8003020464CB0BDE8F08102249C
:10093000F9E7000030B595B013A90446FFF7AEFF04
:10094000002830D11B4B0C2101FB00F2D5189A5C1A
:10095000A2422AD1139B1A7C1092DA7B0F929A7BC7
:100960000E925A7B0D921A7B0C92DA7A0B929A7A3B
:100970000A925A7A09921A7A0892DA7907929A793F
:1009800006925A7905921A790492DA7803929A7843
:1009900002925B7801930022AB6800931146064BEC
:1009A000022002F013FA15B030BD01300B28CBD174
:1009B000F9E700BF844201080C41010810B40B2B79
:1009C000019C03D8019410BCFFF780BF032010BC2A
:1009D000704730B50D4685B01446014668B103AA8C
:1009E000002000922A460390FFF770FF18B9039881
:1009F000001B18BF012005B030BD0220FBE72DE928
:100A0000F0430D46BFB014469946804620B31BB351
:100A100011F00F0122D1F02201A800F0FFF92046C9
:100A20006946FFF73BFF044648B9009801AA102128
:100A30000130FFF73BFD2E46AF1BFFB21EB920462B
:100A40003FB0BDE8F08301AA09EB070108EB0700FE
:100A5000FFF7AEFD103EEFE70224F0E70524EEE7D6
:100A6000F0B5184E3468024685B00846002304F1FC
:100A7000180103EB03154F5D97421ED10D2A05F1B6
:100A8000190513D10023CDE90033CDE902330C223F
:100A900010216B46FFF7B3FF044630681022694609
:100AA000284400F0A7F9204605B0F0BD0146102209
:100AB000601900F09FF90024F5E701330B2BD8D122
:100AC0000324F0E74824002009B1FFF7C9BF022042
:100AD00070471FB51446A0B10C2A01D10B2912D1C1
:100AE0000023CDE90033CDE902330A466B461021DD
:100AF000FFF785FF18B969462046FFF7B1FF04B03C
:100B000010BD0220FBE70320F9E7F8B51E46DDE93A
:100B100007479DF818505BB354B34FB3212D29D824
:100B200019462A46204600F065F90122631C691E19
:100B3000B018FFF764FFF8B9E37ADB093B70EBB953
:100B40006319204613F8012C13F8021C120642EA1E
:100B5000014213F8041C0A4313F8031C012342EA60
:100B60000122291FFFF735FF003818BF0120F8BD0B
:100B70000220FCE70520FAE70720F8E70420F6E763
:100B800010B5044628B1044B5B69984720600020EB
:100B900010BD0220FCE700BF9C43010808B50146D8
:100BA00030B1044B0822186800F024F9002008BD79
:100BB0000220FCE74824002008B530B1044B08228D
:100BC000196800F017F9002008BD0220FCE700BFFB
:100BD000482400207FB5124E0023044602A801934A
:100BE0000D46FFF7E9FF33685B6901936CB102AA18
:100BF000082312F8011B41B9013B13F0FF03F8D1A0
:100C000002A8A04702A8FFF7C9FF35B1019B23B98D
:100C100001A8A8473368019A5A61002004B070BD4A
:100C20004824002008B5014638B1054B1868082251
:100C3000104400F0DFF8002008BD0220FCE700BFF0
:100C40004824002008B538B1044B19680822114423
:100C500000F0D0F8002008BD0220FCE74824002066
:100C6000034B1B6802280CBF1961596100207047B3
:100C70004824002049B1064B1B68D3E9042302280D
:100C800008BF13460B60002070470220704700BF6A
:100C90004824002030B58FB0002405460CA80994E4
:100CA000FFF78AFF9DF8373007939DF8363006939B
:100CB0009DF8353005939DF8343004939DF833301A
:100CC00003939DF8323002939DF8313001939DF8E3
:100CD00030300093224621461E4B022002F076F867
:100CE0000AA8FFF7AFFF9DF82F3007939DF82E302D
:100CF00006939DF82D3005939DF82C3004939DF8B4
:100D00002B3003939DF82A3002939DF829300193EC
:100D10009DF82830009322460F4B2146022002F016
:100D200055F809A92846FFF7A5FF9DF8243003933D
:100D30009DF8253002939DF8263001939DF82730C9
:100D400000932246054B2146022002F03FF80FB0E7
:100D500030BD00BF68410108A6410108E441010817
:100D600008B50020FFF7E6FD0120FFF7E3FD0920AD
:100D7000FFF7E0FD0820FFF7DDFD0020FFF78AFF09
:100D8000002008BD10B504460B20FFF7D3FD0C2052
:100D9000FFF7D0FD0920FFF7CDFD0820FFF7CAFDC2
:100DA0000A20FFF7C7FD2046FFF774FF002010BDA3
:100DB000014B1860704700BFAC0800200B4A30B5EB
:100DC00014680B4D43F2390305FB04331360091A11
:100DD0006FF00042B3FBF2F2C2EBC27201319B1A18
:100DE00093FBF1F201FB1233184430BDAC08002034
:100DF0006D4EC64101380A44914200D1704711F846
:100E0000013B00F8013FF7E710440A44914200D14A
:100E1000704711F8013B00F8013DF7E702F018BDFB
:100E200030B530B10A4D01444FF0FF33814201D15A
:100E3000D84330BD10F8012B5340082243F300047F
:100E4000013A2C4092B284EA5303002AF6D1EDE72E
:100E50002083B8ED01207047054B4FF400529A6291
:100E6000044B1B6813B15B6803B11847704700BFA0
:100E700000040048D8240020054B4FF480529A62A9
:100E8000044B1B6813B1DB6803B11847704700BF00
:100E900000040048D824002001207047012070473A
:100EA00001F03EB901F02CB910B501F00FFE0E2192
:100EB000044640F61F1001F023F92046012101F0FD
:100EC000EFFDBDE8104001F0CDBA000070B50C4E4A
:100ED00001EB40030D46B3654FF6FF710023044656
:100EE0001A46084601F054FB96F85600002101F01E
:100EF000D7FD29462046BDE8704001F08BBA00BFFF
:100F00007C24002010B5044601F0A0FE01281CD16D
:100F100001F0A4FE34B11248214602F00BFB104848
:100F200002F0CEFA0F4C104B00214FF48052A16515
:100F30009A6194F8560001F0B3FD63786BB16FF0DD
:100F40007F40BDE8104001F049BA002340F2622121
:100F50001A46084601F01CFBDCE7A0688001F0E7B8
:100F60004C2400207C24002000040048002001F0D4
:100F7000B5B9000008B501F0BDF80438C0B20328C7
:100F800096BF024B0020185C08BD00BF66430108F5
:100F900008B501F0B0FD033008BD01F03FB901F024
:100FA000FFB808B501F0F6FC08BD000038B50D46E5
:100FB000144601F053FB284601F088FD0E2105463A
:100FC00040F61F1001F09CF828460121074D01F062
:100FD00067FD01F047FA4FF47A716143284602F049
:100FE000A9FA2846BDE8384002F06ABA6424002015
:100FF00001F034BB08B5084B002193F8560001F00E
:101000004FFD00234FF4C0711A46084601F0C0FAA4
:10101000BDE8084001F01ABA7C24002010B504464F
:1010200001F014FE01281CD101F018FE34B1124861
:10103000214602F07FFA104802F042FA0F4C104BA2
:1010400000214FF48052A1659A6194F8560001F096
:1010500027FD63786BB16FF07F40BDE8104001F071
:1010600073B9002340F262211A46084601F090FA53
:10107000DCE7A0688001F0E74C2400207C240020FD
:101080000004004808B54FF0040001F00DF9BDE878
:1010900008400220F1F748BD08B500231A4619465A
:1010A000184601F075FABDE8084001F063B9000088
:1010B0001D4B73B51D4D186000241D486C70C5E9AB
:1010C0000144AC6501F08EFAAC8101F0F9F92146DA
:1010D000204601F041FC21460422012001F0F2FAF1
:1010E000144E154D4FF6FF7123462246084601F077
:1010F0004FFAFFF7C7FF2246104B00944FF0FF3125
:10110000304602F031F90E4B009422464FF0FF3189
:10111000284602F029F9304602F084F9284602B048
:10112000BDE8704002F07EB9D82400207C24002065
:10113000E5200108642400204C240020590E0108F9
:10114000790E01080128084805D1084BC1771970AC
:101150000E3001F09DBB437D012B03D1034B817504
:101160001970F5E7704700BF7C240020B00800200C
:101170000D4B10B5044618735873012000F016F893
:101180005CB134214FF4E86000F0BAFF4421BDE8BF
:10119000104040F2417000F0B3BF14214FF4E860FA
:1011A00000F0AEFF2421F2E77C24002038B5114C7A
:1011B0000546207001F057FD052D04D8DFE805F045
:1011C000090B03171709032001F066FA0023637364
:1011D00038BD0020F8E7012001F05EFA207B637B38
:1011E0008342F5D06073BDE83840FFF7C1BF0220ED
:1011F000EAE700BF7C2400202DE9F0431E4687B0BB
:1012000000230546CDE901330C46174601F01DFDCC
:10121000032D5BD8DFE815F07A00C1000C01040053
:10122000A27C082A69D8A16801A801F0D5FE21682E
:10123000002962D042F210729142E37C874D50D86F
:101240000322AA7385F83820E96385F844304FF00B
:1012500002086368A17DDB002B820423AB74A37CAE
:10126000DB00EB7402294FF000032B75637D02D085
:10127000227D022A46D103F10F02D2B2012A01D9FE
:10128000012B3AD1764B774A196803944FF0010944
:1012900003A88DF8149001F0D5FC70BB287685F872
:1012A00017906875FFF762FE4046FFF77FFF6E48B4
:1012B00001F082FA6D4801F0EBFA01A800F080FF1E
:1012C000208A00F051FFA08900F096FF384601F017
:1012D000FDFB624C84F8560001F0BCFC6660002007
:1012E0000DE04FF00008E963890885F80E8085F865
:1012F000388085F844302964ABE74FF0FF3007B001
:10130000BDE8F083EB7529766A75CBE72368002B7F
:10131000F3D0A27C082AF0D8504DA16801A801F0B2
:101320005BFE002385F838302268EA63E27C85F8AA
:101330004420A269AB732A646268D2002A82042224
:10134000AA74A27C2B75D200EA74A27D022A02D074
:10135000237D022B1CD1627D02F10F03DBB2012B36
:1013600001D9012AC9D13E4B3E4A196803944FF076
:10137000010803A88DF8148001F064FC0028BCD19A
:10138000287685F817806875FFF7F0FD00208CE758
:10139000617DE9752A766B75F6E7304D012185F898
:1013A0003810227885F85020637885F85130A3787A
:1013B00085F85230E3788B4202D0022B03D03BB940
:1013C00085F8533004E00B3A012A29D885F85310E8
:1013D0004FF0010885F80E80A388AB83A379AB7723
:1013E000E37985F82030237A85F82130FFF7BEFDB8
:1013F0004046FFF7DBFE1C4801F0DEF91B4801F018
:1014000047FA95F85130062B40F689000AD100F0D2
:1014100087FE00F0FB0140F6890000F071FE55E701
:101420000023CDE700F07CFE40F00401C9B2F2E7F2
:101430002368013BB3F57A7FBFF45FAF0320FFF76A
:10144000B5FE0648022380F83830236883641623EB
:1014500080F84C30383001F0AFF937E77C240020B9
:10146000D824002064240020B42400208A240020F2
:10147000F0B51E4687B00023CDE901331446074678
:101480000D4601F0E2FB002C724C16BF0123002335
:101490000026637027B1012F7AD0002007B0F0BD7D
:1014A000AB68002B00F0D280EB68002B00F0CE8000
:1014B000AA7F082A00F2CA80296901A801F08CFDE0
:1014C0002868003818BF012000F0D6FF84F8387073
:1014D000AB68E36395F8203084F84430686801F025
:1014E00057FBA77384F84500EB68DB002382EB7F92
:1014F000A374AB7FDB00E37495F82130237595F876
:101500002230002B3ED12A7D95F82410A2750229A5
:1015100095F8232001D0022B36D102F10F03DBB264
:10152000012B02D9012A40F0918000238DF814305C
:10153000494B4A4A1968049503A801F083FB002827
:1015400040F0848001232076E3756075FFF70EFD7F
:101550000020FFF72BFE424801F02EF9414801F030
:1015600097F901A800F02CFEA88B00F0FDFD288B58
:1015700000F042FE4FF4FA53AA687343B3FBF2F350
:10158000A3608AE7FF22BFE7E27521766375DDE796
:101590002B8E002B5AD095F83230A86A012B0CBF45
:1015A0002F7DFF27003818BF012000F065FFF0B243
:1015B00000F06EFF012184F8381095F82C2084F893
:1015C000502095F82D3084F8513095F82E3084F85D
:1015D000523095F82F308B4202D0022B03D03BB90A
:1015E00084F8533004E00B3A012A27D884F85310CA
:1015F0002B8EA38395F83230A3770126AB8E2384FC
:10160000A673E777FFF7B2FC3046FFF7CFFD14482B
:1016100001F0D2F8134801F03BF994F82130B342BD
:1016200040F236700CD100F07BFD00F0FB0140F27F
:10163000367000F065FD4FF6FF73A1E70023CFE79A
:1016400000F06EFD40F00401C9B2F0E74FF0FF304A
:1016500024E700BF7C240020D82400204C24002054
:10166000B42400208A2400202DE9F04F85B0824662
:101670000E9DBDF840809DF844709DF84890019102
:1016800093461E4601F0E1FABAF1010F524C54D0D4
:10169000BAF1040F00F09180BAF1000F3AD10B2299
:1016A000304684F8442084F838A0E56301F070FAED
:1016B0004FEAC803B9F1000F238241F604036382A5
:1016C0000CBF0123F223E37587F001070123237682
:1016D00084F84500C4F840B084F80EA084F814A043
:1016E0006775FFF743FC5046FFF760FD04F13800D3
:1016F00001F062F804F10E0001F0CAF8374A1068F0
:10170000516802AB03C302A800F05AFD40F2FF107B
:1017100000F02AFD019801F0D9F90E2184F8560055
:1017200040F61F1000F0ECFC94F8560001F092FA1D
:10173000169B636005B0BDE8F08F294984F838A096
:10174000EAB2895D84F8502076BB0B3D012D8CBF39
:1017500000250125053A012A04D8B8F10C0F38BF3D
:101760004FF00C081F4B9DF83C201B7884F8535019
:10177000E37701259DF8543084F8511084F8522005
:1017800084F82130A573A4F81C80A77784F82090F2
:10179000FFF7ECFB2846FFF709FD134801F00CF8B2
:1017A000124801F075F8B5E7012E04D1A5F10C033C
:1017B0005D425D41CEE70025CCE75046FFF7F6FCE1
:1017C000022384F8383004F138001623A56484F825
:1017D0004C3000F0F1FF9DE77C240020503A0108D6
:1017E00098430108B0080020B42400208A24002077
:1017F0002DE9F04F87B0DFF8B4B29DF864A09DF8F2
:101800004C90029314469DF854309DF85020BDF83A
:101810004880039205468BF801A0BDF8446001930F
:101820000F4601F012FABAF1000F18BF4FF000088E
:10183000DFF87CA2039AB9F1000F08BFFF22012D47
:101840008AF8002000F0C880052D48D0002D40F017
:10185000C080284600F010FE0B2238468BF844204A
:101860008BF83850CBF83C4001F092F9019B8BF893
:10187000450041F60402002BABF812209AF8002034
:101880008BF816200CBF0122F2228BF81720F600ED
:10189000012289F001098BF818208BF80E50ABF863
:1018A00010608BF814508BF81590FFF75FFB2846FB
:1018B000FFF77CFC0BF1380000F07EFF0BF10E000F
:1018C00000F0E6FF7B490868496804AA03C204A83F
:1018D00000F076FC40F2FF1000F046FC71E00120C1
:1018E00000F0CAFD09224FF000098BF84420384669
:1018F0004FF44872CBF840208BF83890CBF83C403E
:1019000001F046F94FF48052ABF812209AF800200B
:101910008BF845008BF8162028460122F6008BF83C
:1019200017208BF80E90ABF81060ABF814908BF882
:101930001890FFF73BFC0BF1380000F03DFF0BF176
:101940000E0000F0A5FF5B498868C96804AA03C2BD
:1019500004A800F035FC40F2FF1000F005FC40F652
:10196000B80000F0DDFB00F0EF0140F6B80000F039
:10197000C7FB042140F6B90000F0C2FB40F69B0013
:1019800000F0CEFB00F0E30141F0080140F69B00BF
:1019900000F0B6FB40F2D16000F0C2FB40F018014D
:1019A000C9B240F2D16000F0ABFB40F2AC6000F095
:1019B000B7FB00F08F0141F0500140F2AC6000F045
:1019C0009FFB4FF4FA5202FB08F2B2FBF4F2CBF8A1
:1019D000082007B0BDE8F08F002000F04DFD36492B
:1019E0008BF83850E2B2C95D8BF85020002F4DD1F2
:1019F0000B3C012C8CBF00240124053A012A02D89B
:101A00000C2E38BF0C26029B9AF800208BF852301F
:101A10008BF85340019B8BF81F2001249DF8602018
:101A20008BF821208BF851108BF820308BF80E406A
:101A3000ABF81C608BF81E90FFF798FA2046FFF772
:101A4000B5FB1E4800F0B8FE1D4800F021FF5FFA0C
:101A500088F000F01DFD40F6A30000F061FB00EAF5
:101A6000040140F6A30000F04BFB9BF82120A242AA
:101A700040F2367013D100F053FB00F0FB0140F24E
:101A8000367000F03DFB4FF6FF72A0E7012F04D146
:101A9000A4F10C035C425C41AFE70024ADE700F029
:101AA0003FFB40F00401C9B2E9E700BF7C240020FD
:101AB000B0080020503A010898430108B4240020DF
:101AC0008A240020F0B58BB00D46044617461E460A
:101AD000FFF74CFA0020FFF769FB204600F0BEFD3F
:101AE00000240123CDE9084303234FF4167229464D
:101AF0002046CDE90644CDE90444CDE90244CDE9D0
:101B000000532346FFF774FE2046FFF787FAFFF7DE
:101B10003FFAF1F709F801F041FC0446204601F0D4
:101B200047FCB04205D30124FFF720FA20460BB052
:101B3000F0BD00F02FFF8742F0DA0024F4E7000048
:101B4000F7B500230C4640F201211A460646084626
:101B500000F01EFD644B654D4FF400529A6195F8FC
:101B60005600012100F09CFF2B78012B40F68900E4
:101B700013D195F85130062B0FD100F0D1FA00F0B7
:101B8000FB0140F6890000F0BBFA2B78042B6CD8DF
:101B9000DFE803F0524B527F090000F0C1FA40F039
:101BA0000401C9B2EDE7524A731E1046C6F101079F
:101BB0004FF0000CF9188C426FDC0022E70013464E
:101BC000BA4271D19A0142EAC3125B0183F0200349
:101BD0001343661C0355F6B202234648AB73AE7638
:101BE00000F056FE0021F12000F08AFA0021F020DA
:101BF00000F086FAAB6C642B70D17021F32000F0FA
